 java

 Timestamp is f05fb8d7 (reproducible build file hash)

 Preferred load address is 0000000180000000

 Start         Length     Name                   Class
 0001:00000000 00016760H .text$mn                CODE
 0001:00016760 00000036H .text$mn$00             CODE
 0001:00016796 00000092H .text$x                 CODE
 0002:00000000 00000a80H .idata$5                DATA
 0002:00000a80 00000038H .00cfg                  DATA
 0002:00000ab8 00000008H .CRT$XCA                DATA
 0002:00000ac0 00000008H .CRT$XCZ                DATA
 0002:00000ac8 00000008H .CRT$XIA                DATA
 0002:00000ad0 00000008H .CRT$XIZ                DATA
 0002:00000ad8 00000008H .CRT$XPA                DATA
 0002:00000ae0 00000008H .CRT$XPZ                DATA
 0002:00000ae8 00000008H .CRT$XTA                DATA
 0002:00000af0 00000010H .CRT$XTZ                DATA
 0002:00000af8 00000000H .gehcont$y              DATA
 0002:00000af8 00000000H .gfids$y                DATA
 0002:00000b00 00002200H .rdata                  DATA
 0002:00002d00 00000000H .rdata$CastGuardVftablesA DATA
 0002:00002d00 00000000H .rdata$CastGuardVftablesC DATA
 0002:00002d00 000000b8H .rdata$voltmd           DATA
 0002:00002db8 00000330H .rdata$zzzdbg           DATA
 0002:000030e8 00000008H .rtc$IAA                DATA
 0002:000030f0 00000008H .rtc$IZZ                DATA
 0002:000030f8 00000008H .rtc$TAA                DATA
 0002:00003100 00000008H .rtc$TZZ                DATA
 0002:00003108 00000ce4H .xdata                  DATA
 0002:00003dec 00000020H .didat$2                DATA
 0002:00003e0c 00000024H .didat$3                DATA
 0002:00003e30 00000018H .didat$4                DATA
 0002:00003e48 00000030H .didat$6                DATA
 0002:00003e78 00000018H .didat$7                DATA
 0002:00003e90 00003eb8H .edata                  DATA
 0002:00007d48 00000118H .idata$2                DATA
 0002:00007e60 00000018H .idata$3                DATA
 0002:00007e78 00000a80H .idata$4                DATA
 0002:000088f8 00001b74H .idata$6                DATA
 0003:00000000 000013a0H .data                   DATA
 0003:000013a0 00000020H .didat$5                DATA
 0003:000013c0 000008d0H .bss                    DATA
 0004:00000000 00000ff0H .pdata                  DATA
 0005:00000000 00000060H .rsrc$01                DATA
 0005:00000060 00000308H .rsrc$02                DATA

  Address         Publics by Value              Rva+Base               Lib:Object

 0000:00000000       __AbsoluteZero             0000000000000000     <absolute>
 0000:00000000       ___safe_se_handler_count   0000000000000000     <absolute>
 0000:00000000       ___safe_se_handler_table   0000000000000000     <absolute>
 0000:00000000       __arm64x_extra_rfe_table   0000000000000000     <absolute>
 0000:00000000       __arm64x_extra_rfe_table_size 0000000000000000     <absolute>
 0000:00000000       __arm64x_native_entrypoint 0000000000000000     <absolute>
 0000:00000000       __arm64x_redirection_metadata 0000000000000000     <absolute>
 0000:00000000       __arm64x_redirection_metadata_count 0000000000000000     <absolute>
 0000:00000000       __dynamic_value_reloc_table 0000000000000000     <absolute>
 0000:00000000       __enclave_config           0000000000000000     <absolute>
 0000:00000000       __guard_check_icall_a64n_fptr 0000000000000000     <absolute>
 0000:00000000       __guard_eh_cont_count      0000000000000000     <absolute>
 0000:00000000       __guard_eh_cont_table      0000000000000000     <absolute>
 0000:00000000       __guard_fids_count         0000000000000000     <absolute>
 0000:00000000       __guard_fids_table         0000000000000000     <absolute>
 0000:00000000       __guard_iat_count          0000000000000000     <absolute>
 0000:00000000       __guard_iat_table          0000000000000000     <absolute>
 0000:00000000       __guard_longjmp_count      0000000000000000     <absolute>
 0000:00000000       __guard_longjmp_table      0000000000000000     <absolute>
 0000:00000000       __hybrid_auxiliary_delayload_iat 0000000000000000     <absolute>
 0000:00000000       __hybrid_auxiliary_delayload_iat_copy 0000000000000000     <absolute>
 0000:00000000       __hybrid_auxiliary_iat     0000000000000000     <absolute>
 0000:00000000       __hybrid_auxiliary_iat_copy 0000000000000000     <absolute>
 0000:00000000       __hybrid_code_map          0000000000000000     <absolute>
 0000:00000000       __hybrid_code_map_count    0000000000000000     <absolute>
 0000:00000000       __hybrid_image_info_bitfield 0000000000000000     <absolute>
 0000:00000000       __x64_code_ranges_to_entry_points 0000000000000000     <absolute>
 0000:00000000       __x64_code_ranges_to_entry_points_count 0000000000000000     <absolute>
 0000:00000100       __guard_flags              0000000000000100     <absolute>
 0000:00000000       __ImageBase                0000000180000000     <linker-defined>
 0001:00000000       Java_java_security_AccessController_doPrivileged__Ljava_security_PrivilegedAction_2 0000000180001000 f   AccessController.obj
 0001:00000018       Java_java_security_AccessController_doPrivileged__Ljava_security_PrivilegedAction_2Ljava_security_AccessControlContext_2 0000000180001018 f   AccessController.obj
 0001:0000002c       Java_java_security_AccessController_doPrivileged__Ljava_security_PrivilegedExceptionAction_2 000000018000102c f   AccessController.obj
 0001:00000044       Java_java_security_AccessController_doPrivileged__Ljava_security_PrivilegedExceptionAction_2Ljava_security_AccessControlContext_2 0000000180001044 f   AccessController.obj
 0001:00000058       Java_java_security_AccessController_getInheritedAccessControlContext 0000000180001058 f   AccessController.obj
 0001:00000060       Java_java_security_AccessController_getStackAccessControlContext 0000000180001060 f   AccessController.obj
 0001:00000068       Java_java_lang_reflect_Array_get 0000000180001068 f   Array.obj
 0001:00000074       Java_java_lang_reflect_Array_getBoolean 0000000180001074 f   Array.obj
 0001:00000088       Java_java_lang_reflect_Array_getByte 0000000180001088 f   Array.obj
 0001:0000009c       Java_java_lang_reflect_Array_getChar 000000018000109c f   Array.obj
 0001:000000b0       Java_java_lang_reflect_Array_getDouble 00000001800010b0 f   Array.obj
 0001:000000d8       Java_java_lang_reflect_Array_getFloat 00000001800010d8 f   Array.obj
 0001:00000100       Java_java_lang_reflect_Array_getInt 0000000180001100 f   Array.obj
 0001:00000114       Java_java_lang_reflect_Array_getLength 0000000180001114 f   Array.obj
 0001:0000011c       Java_java_lang_reflect_Array_getLong 000000018000111c f   Array.obj
 0001:00000130       Java_java_lang_reflect_Array_getShort 0000000180001130 f   Array.obj
 0001:00000144       Java_java_lang_reflect_Array_multiNewArray 0000000180001144 f   Array.obj
 0001:00000150       Java_java_lang_reflect_Array_newArray 0000000180001150 f   Array.obj
 0001:0000015c       Java_java_lang_reflect_Array_set 000000018000115c f   Array.obj
 0001:00000170       Java_java_lang_reflect_Array_setBoolean 0000000180001170 f   Array.obj
 0001:00000198       Java_java_lang_reflect_Array_setByte 0000000180001198 f   Array.obj
 0001:000001c0       Java_java_lang_reflect_Array_setChar 00000001800011c0 f   Array.obj
 0001:000001ec       Java_java_lang_reflect_Array_setDouble 00000001800011ec f   Array.obj
 0001:00000210       Java_java_lang_reflect_Array_setFloat 0000000180001210 f   Array.obj
 0001:0000023c       Java_java_lang_reflect_Array_setInt 000000018000123c f   Array.obj
 0001:00000264       Java_java_lang_reflect_Array_setLong 0000000180001264 f   Array.obj
 0001:00000288       Java_java_lang_reflect_Array_setShort 0000000180001288 f   Array.obj
 0001:000002b4       Java_java_util_concurrent_atomic_AtomicLong_VMSupportsCS8 00000001800012b4 f   AtomicLong.obj
 0001:000002bc       Java_jdk_internal_loader_BootLoader_getSystemPackageLocation 00000001800012bc f   BootLoader.obj
 0001:000002c4       Java_jdk_internal_loader_BootLoader_getSystemPackageNames 00000001800012c4 f   BootLoader.obj
 0001:000002cc       Java_jdk_internal_loader_BootLoader_setBootLoaderUnnamedModule0 00000001800012cc f   BootLoader.obj
 0001:000002d4       Java_java_lang_Class_forName0 00000001800012d4 f   Class.obj
 0001:00000430       Java_java_lang_Class_getPrimitiveClass 0000000180001430 f   Class.obj
 0001:000004ac       Java_java_lang_Class_isAssignableFrom 00000001800014ac f   Class.obj
 0001:000004d8       Java_java_lang_Class_isInstance 00000001800014d8 f   Class.obj
 0001:000004f4       Java_java_lang_Class_registerNatives 00000001800014f4 f   Class.obj
 0001:0000051c       Java_java_lang_ClassLoader_00024NativeLibrary_findEntry 000000018000151c f   ClassLoader.obj
 0001:000005b4       Java_java_lang_ClassLoader_00024NativeLibrary_load0 00000001800015b4 f   ClassLoader.obj
 0001:000007d0       Java_java_lang_ClassLoader_00024NativeLibrary_unload 00000001800017d0 f   ClassLoader.obj
 0001:00000888       Java_java_lang_ClassLoader_defineClass1 0000000180001888 f   ClassLoader.obj
 0001:00000a38       Java_java_lang_ClassLoader_defineClass2 0000000180001a38 f   ClassLoader.obj
 0001:00000bb4       Java_java_lang_ClassLoader_findBootstrapClass 0000000180001bb4 f   ClassLoader.obj
 0001:00000c70       Java_java_lang_ClassLoader_findBuiltinLib 0000000180001c70 f   ClassLoader.obj
 0001:00000dc8       Java_java_lang_ClassLoader_findLoadedClass0 0000000180001dc8 f   ClassLoader.obj
 0001:00000dd8       Java_java_lang_ClassLoader_registerNatives 0000000180001dd8 f   ClassLoader.obj
 0001:00001034       Java_java_io_Console_echo  0000000180002034 f   Console_md.obj
 0001:000010c8       Java_java_io_Console_encoding 00000001800020c8 f   Console_md.obj
 0001:00001130       Java_java_io_Console_istty 0000000180002130 f   Console_md.obj
 0001:000011ac       __local_stdio_printf_options 00000001800021ac f i Console_md.obj
 0001:000011b4       sprintf                    00000001800021b4 f i Console_md.obj
 0001:0000120c       Java_jdk_internal_reflect_ConstantPool_getClassAt0 000000018000220c f   ConstantPool.obj
 0001:00001214       Java_jdk_internal_reflect_ConstantPool_getClassAtIfLoaded0 0000000180002214 f   ConstantPool.obj
 0001:0000121c       Java_jdk_internal_reflect_ConstantPool_getClassRefIndexAt0 000000018000221c f   ConstantPool.obj
 0001:00001224       Java_jdk_internal_reflect_ConstantPool_getDoubleAt0 0000000180002224 f   ConstantPool.obj
 0001:0000122c       Java_jdk_internal_reflect_ConstantPool_getFieldAt0 000000018000222c f   ConstantPool.obj
 0001:00001234       Java_jdk_internal_reflect_ConstantPool_getFieldAtIfLoaded0 0000000180002234 f   ConstantPool.obj
 0001:0000123c       Java_jdk_internal_reflect_ConstantPool_getFloatAt0 000000018000223c f   ConstantPool.obj
 0001:00001244       Java_jdk_internal_reflect_ConstantPool_getIntAt0 0000000180002244 f   ConstantPool.obj
 0001:0000124c       Java_jdk_internal_reflect_ConstantPool_getLongAt0 000000018000224c f   ConstantPool.obj
 0001:00001254       Java_jdk_internal_reflect_ConstantPool_getMemberRefInfoAt0 0000000180002254 f   ConstantPool.obj
 0001:0000125c       Java_jdk_internal_reflect_ConstantPool_getMethodAt0 000000018000225c f   ConstantPool.obj
 0001:00001264       Java_jdk_internal_reflect_ConstantPool_getMethodAtIfLoaded0 0000000180002264 f   ConstantPool.obj
 0001:0000126c       Java_jdk_internal_reflect_ConstantPool_getNameAndTypeRefIndexAt0 000000018000226c f   ConstantPool.obj
 0001:00001274       Java_jdk_internal_reflect_ConstantPool_getNameAndTypeRefInfoAt0 0000000180002274 f   ConstantPool.obj
 0001:0000127c       Java_jdk_internal_reflect_ConstantPool_getSize0 000000018000227c f   ConstantPool.obj
 0001:00001284       Java_jdk_internal_reflect_ConstantPool_getStringAt0 0000000180002284 f   ConstantPool.obj
 0001:0000128c       Java_jdk_internal_reflect_ConstantPool_getTagAt0 000000018000228c f   ConstantPool.obj
 0001:00001294       Java_jdk_internal_reflect_ConstantPool_getUTF8At0 0000000180002294 f   ConstantPool.obj
 0001:0000129c       Java_java_lang_Double_doubleToRawLongBits 000000018000229c f   Double.obj
 0001:000012a8       Java_java_lang_Double_longBitsToDouble 00000001800022a8 f   Double.obj
 0001:000012b4       Java_java_lang_reflect_Executable_getParameters0 00000001800022b4 f   Executable.obj
 0001:000012bc       Java_java_lang_reflect_Executable_getTypeAnnotationBytes0 00000001800022bc f   Executable.obj
 0001:000012c4       Java_java_lang_reflect_Field_getTypeAnnotationBytes0 00000001800022c4 f   Field.obj
 0001:000012cc       Java_java_io_FileCleanable_cleanupClose0 00000001800022cc f   FileDescriptor_md.obj
 0001:000012fc       Java_java_io_FileDescriptor_close0 00000001800022fc f   FileDescriptor_md.obj
 0001:00001304       Java_java_io_FileDescriptor_getAppend 0000000180002304 f   FileDescriptor_md.obj
 0001:00001304       Java_java_lang_StringUTF16_isBigEndian 0000000180002304 f   String.obj
 0001:00001308       Java_java_io_FileDescriptor_getHandle 0000000180002308 f   FileDescriptor_md.obj
 0001:00001338       Java_java_io_FileDescriptor_initIDs 0000000180002338 f   FileDescriptor_md.obj
 0001:000013c4       Java_java_io_FileDescriptor_sync 00000001800023c4 f   FileDescriptor_md.obj
 0001:00001408       Java_java_io_FileInputStream_available0 0000000180002408 f   FileInputStream.obj
 0001:000014bc       Java_java_io_FileInputStream_initIDs 00000001800024bc f   FileInputStream.obj
 0001:000014e4       Java_java_io_FileInputStream_open0 00000001800024e4 f   FileInputStream.obj
 0001:00001500       Java_java_io_FileInputStream_read0 0000000180002500 f   FileInputStream.obj
 0001:0000150c       Java_java_io_FileInputStream_readBytes 000000018000250c f   FileInputStream.obj
 0001:00001530       Java_java_io_FileInputStream_skip0 0000000180002530 f   FileInputStream.obj
 0001:00001610       Java_java_io_FileOutputStream_initIDs 0000000180002610 f   FileOutputStream_md.obj
 0001:00001638       Java_java_io_FileOutputStream_open0 0000000180002638 f   FileOutputStream_md.obj
 0001:00001660       Java_java_io_FileOutputStream_write 0000000180002660 f   FileOutputStream_md.obj
 0001:0000167c       Java_java_io_FileOutputStream_writeBytes 000000018000267c f   FileOutputStream_md.obj
 0001:000016a8       Java_java_lang_Float_floatToRawIntBits 00000001800026a8 f   Float.obj
 0001:000016b4       Java_java_lang_Float_intBitsToFloat 00000001800026b4 f   Float.obj
 0001:000016c0       EnumCalendarInfoProc       00000001800026c0 f   HostLocaleProviderAdapter_md.obj
 0001:000016fc       Java_sun_util_locale_provider_HostLocaleProviderAdapterImpl_getAmPmStrings 00000001800026fc f   HostLocaleProviderAdapter_md.obj
 0001:00001834       Java_sun_util_locale_provider_HostLocaleProviderAdapterImpl_getCalendarDataValue 0000000180002834 f   HostLocaleProviderAdapter_md.obj
 0001:000018b8       Java_sun_util_locale_provider_HostLocaleProviderAdapterImpl_getCalendarDisplayStrings 00000001800028b8 f   HostLocaleProviderAdapter_md.obj
 0001:00001984       Java_sun_util_locale_provider_HostLocaleProviderAdapterImpl_getCalendarID 0000000180002984 f   HostLocaleProviderAdapter_md.obj
 0001:000019ec       Java_sun_util_locale_provider_HostLocaleProviderAdapterImpl_getCurrencySymbol 00000001800029ec f   HostLocaleProviderAdapter_md.obj
 0001:00001ab0       Java_sun_util_locale_provider_HostLocaleProviderAdapterImpl_getDateTimePattern 0000000180002ab0 f   HostLocaleProviderAdapter_md.obj
 0001:00001bbc       Java_sun_util_locale_provider_HostLocaleProviderAdapterImpl_getDecimalSeparator 0000000180002bbc f   HostLocaleProviderAdapter_md.obj
 0001:00001c68       Java_sun_util_locale_provider_HostLocaleProviderAdapterImpl_getDefaultLocale 0000000180002c68 f   HostLocaleProviderAdapter_md.obj
 0001:00001cdc       Java_sun_util_locale_provider_HostLocaleProviderAdapterImpl_getDisplayString 0000000180002cdc f   HostLocaleProviderAdapter_md.obj
 0001:00001dcc       Java_sun_util_locale_provider_HostLocaleProviderAdapterImpl_getEras 0000000180002dcc f   HostLocaleProviderAdapter_md.obj
 0001:00001dec       Java_sun_util_locale_provider_HostLocaleProviderAdapterImpl_getGroupingSeparator 0000000180002dec f   HostLocaleProviderAdapter_md.obj
 0001:00001e98       Java_sun_util_locale_provider_HostLocaleProviderAdapterImpl_getInfinity 0000000180002e98 f   HostLocaleProviderAdapter_md.obj
 0001:00001f5c       Java_sun_util_locale_provider_HostLocaleProviderAdapterImpl_getInternationalCurrencySymbol 0000000180002f5c f   HostLocaleProviderAdapter_md.obj
 0001:00002020       Java_sun_util_locale_provider_HostLocaleProviderAdapterImpl_getMinusSign 0000000180003020 f   HostLocaleProviderAdapter_md.obj
 0001:000020cc       Java_sun_util_locale_provider_HostLocaleProviderAdapterImpl_getMonetaryDecimalSeparator 00000001800030cc f   HostLocaleProviderAdapter_md.obj
 0001:00002178       Java_sun_util_locale_provider_HostLocaleProviderAdapterImpl_getMonths 0000000180003178 f   HostLocaleProviderAdapter_md.obj
 0001:000021b8       Java_sun_util_locale_provider_HostLocaleProviderAdapterImpl_getNaN 00000001800031b8 f   HostLocaleProviderAdapter_md.obj
 0001:0000227c       Java_sun_util_locale_provider_HostLocaleProviderAdapterImpl_getNumberPattern 000000018000327c f   HostLocaleProviderAdapter_md.obj
 0001:00002324       Java_sun_util_locale_provider_HostLocaleProviderAdapterImpl_getPerMill 0000000180003324 f   HostLocaleProviderAdapter_md.obj
 0001:000023d0       Java_sun_util_locale_provider_HostLocaleProviderAdapterImpl_getPercent 00000001800033d0 f   HostLocaleProviderAdapter_md.obj
 0001:0000247c       Java_sun_util_locale_provider_HostLocaleProviderAdapterImpl_getShortMonths 000000018000347c f   HostLocaleProviderAdapter_md.obj
 0001:000024bc       Java_sun_util_locale_provider_HostLocaleProviderAdapterImpl_getShortWeekdays 00000001800034bc f   HostLocaleProviderAdapter_md.obj
 0001:00002500       Java_sun_util_locale_provider_HostLocaleProviderAdapterImpl_getWeekdays 0000000180003500 f   HostLocaleProviderAdapter_md.obj
 0001:00002544       Java_sun_util_locale_provider_HostLocaleProviderAdapterImpl_getZeroDigit 0000000180003544 f   HostLocaleProviderAdapter_md.obj
 0001:000025f0       Java_sun_util_locale_provider_HostLocaleProviderAdapterImpl_initialize 00000001800035f0 f   HostLocaleProviderAdapter_md.obj
 0001:000026a4       Java_sun_util_locale_provider_HostLocaleProviderAdapterImpl_isNativeDigit 00000001800036a4 f   HostLocaleProviderAdapter_md.obj
 0001:00002728       enumCalendarInfoWrapper    0000000180003728 f   HostLocaleProviderAdapter_md.obj
 0001:000027a8       getCalendarID              00000001800037a8 f   HostLocaleProviderAdapter_md.obj
 0001:00002818       getCalendarInfoWrapper     0000000180003818 f   HostLocaleProviderAdapter_md.obj
 0001:000028a8       getErasImpl                00000001800038a8 f   HostLocaleProviderAdapter_md.obj
 0001:00002b30       getFixPart                 0000000180003b30 f   HostLocaleProviderAdapter_md.obj
 0001:00002bf4       getLocaleInfoWrapper       0000000180003bf4 f   HostLocaleProviderAdapter_md.obj
 0001:00002c64       getNumberPart              0000000180003c64 f   HostLocaleProviderAdapter_md.obj
 0001:00002e24       getNumberPattern           0000000180003e24 f   HostLocaleProviderAdapter_md.obj
 0001:00002fd4       replaceCalendarArrayElems  0000000180003fd4 f   HostLocaleProviderAdapter_md.obj
 0001:000031e8       Java_java_lang_Module_addExports0 00000001800041e8 f   Module.obj
 0001:00003290       Java_java_lang_Module_addExportsToAll0 0000000180004290 f   Module.obj
 0001:00003320       Java_java_lang_Module_addExportsToAllUnnamed0 0000000180004320 f   Module.obj
 0001:000033b0       Java_java_lang_Module_addReads0 00000001800043b0 f   Module.obj
 0001:000033bc       Java_java_lang_Module_defineModule0 00000001800043bc f   Module.obj
 0001:000034f4       Java_jdk_internal_reflect_NativeConstructorAccessorImpl_newInstance0 00000001800044f4 f   NativeAccessors.obj
 0001:00003500       Java_jdk_internal_reflect_NativeMethodAccessorImpl_invoke0 0000000180004500 f   NativeAccessors.obj
 0001:00003514       Java_java_lang_Object_getClass 0000000180004514 f   Object.obj
 0001:00003538       Java_java_lang_Object_registerNatives 0000000180004538 f   Object.obj
 0001:00003550       Java_java_io_ObjectInputStream_bytesToDoubles 0000000180004550 f   ObjectInputStream.obj
 0001:000036c0       Java_java_io_ObjectInputStream_bytesToFloats 00000001800046c0 f   ObjectInputStream.obj
 0001:000037f4       Java_java_io_ObjectOutputStream_doublesToBytes 00000001800047f4 f   ObjectOutputStream.obj
 0001:000039b8       Java_java_io_ObjectOutputStream_floatsToBytes 00000001800049b8 f   ObjectOutputStream.obj
 0001:00003b14       Java_java_io_ObjectStreamClass_hasStaticInitializer 0000000180004b14 f   ObjectStreamClass.obj
 0001:00003c18       Java_java_io_ObjectStreamClass_initNative 0000000180004c18 f   ObjectStreamClass.obj
 0001:00003c50       Java_java_lang_ProcessEnvironment_environmentBlock 0000000180004c50 f   ProcessEnvironment_md.obj
 0001:00003dc0       Java_java_lang_ProcessHandleImpl_00024Info_info0 0000000180004dc0 f   ProcessHandleImpl_win.obj
 0001:00003e30       Java_java_lang_ProcessHandleImpl_00024Info_initIDs 0000000180004e30 f   ProcessHandleImpl_win.obj
 0001:00003f40       Java_java_lang_ProcessHandleImpl_destroy0 0000000180004f40 f   ProcessHandleImpl_win.obj
 0001:00003fac       Java_java_lang_ProcessHandleImpl_getCurrentPid0 0000000180004fac f   ProcessHandleImpl_win.obj
 0001:00003fc0       Java_java_lang_ProcessHandleImpl_getProcessPids0 0000000180004fc0 f   ProcessHandleImpl_win.obj
 0001:00004290       Java_java_lang_ProcessHandleImpl_initNative 0000000180005290 f   ProcessHandleImpl_win.obj
 0001:00004290       _guard_check_icall_nop     0000000180005290 f   MSVCRT:guard_support.obj
 0001:00004294       Java_java_lang_ProcessHandleImpl_isAlive0 0000000180005294 f   ProcessHandleImpl_win.obj
 0001:000042f4       Java_java_lang_ProcessHandleImpl_parent0 00000001800052f4 f   ProcessHandleImpl_win.obj
 0001:000043f0       Java_java_lang_ProcessHandleImpl_waitForProcessExit0 00000001800053f0 f   ProcessHandleImpl_win.obj
 0001:000048e4       Java_java_lang_ProcessImpl_closeHandle 00000001800058e4 f   ProcessImpl_md.obj
 0001:000048f0       Java_java_lang_ProcessImpl_create 00000001800058f0 f   ProcessImpl_md.obj
 0001:00004a84       Java_java_lang_ProcessImpl_getExitCodeProcess 0000000180005a84 f   ProcessImpl_md.obj
 0001:00004ab8       Java_java_lang_ProcessImpl_getProcessId0 0000000180005ab8 f   ProcessImpl_md.obj
 0001:00004ac4       Java_java_lang_ProcessImpl_getStillActive 0000000180005ac4 f   ProcessImpl_md.obj
 0001:00004acc       Java_java_lang_ProcessImpl_isProcessAlive 0000000180005acc f   ProcessImpl_md.obj
 0001:00004af0       Java_java_lang_ProcessImpl_openForAtomicAppend 0000000180005af0 f   ProcessImpl_md.obj
 0001:00004b7c       Java_java_lang_ProcessImpl_terminateProcess 0000000180005b7c f   ProcessImpl_md.obj
 0001:00004b8c       Java_java_lang_ProcessImpl_waitForInterruptibly 0000000180005b8c f   ProcessImpl_md.obj
 0001:00004bd4       Java_java_lang_ProcessImpl_waitForTimeoutInterruptibly 0000000180005bd4 f   ProcessImpl_md.obj
 0001:00004cd0       os_error_message           0000000180005cd0 f   ProcessImpl_md.obj
 0001:00005098       swprintf                   0000000180006098 f i ProcessImpl_md.obj
 0001:00005214       Java_java_io_RandomAccessFile_getFilePointer 0000000180006214 f   RandomAccessFile.obj
 0001:000052bc       Java_java_io_RandomAccessFile_initIDs 00000001800062bc f   RandomAccessFile.obj
 0001:000052e4       Java_java_io_RandomAccessFile_length 00000001800062e4 f   RandomAccessFile.obj
 0001:00005388       Java_java_io_RandomAccessFile_open0 0000000180006388 f   RandomAccessFile.obj
 0001:000053e0       Java_java_io_RandomAccessFile_read0 00000001800063e0 f   RandomAccessFile.obj
 0001:000053ec       Java_java_io_RandomAccessFile_readBytes 00000001800063ec f   RandomAccessFile.obj
 0001:00005410       Java_java_io_RandomAccessFile_seek0 0000000180006410 f   RandomAccessFile.obj
 0001:000054c8       Java_java_io_RandomAccessFile_setLength 00000001800064c8 f   RandomAccessFile.obj
 0001:000055b0       Java_java_io_RandomAccessFile_write0 00000001800065b0 f   RandomAccessFile.obj
 0001:000055d0       Java_java_io_RandomAccessFile_writeBytes 00000001800065d0 f   RandomAccessFile.obj
 0001:000055f8       Java_java_lang_ref_Reference_getAndClearReferencePendingList 00000001800065f8 f   Reference.obj
 0001:00005600       Java_java_lang_ref_Reference_hasReferencePendingList 0000000180006600 f   Reference.obj
 0001:00005608       Java_java_lang_ref_Reference_waitForReferencePendingList 0000000180006608 f   Reference.obj
 0001:00005610       Java_jdk_internal_reflect_Reflection_areNestMates 0000000180006610 f   Reflection.obj
 0001:0000561c       Java_jdk_internal_reflect_Reflection_getCallerClass__ 000000018000661c f   Reflection.obj
 0001:00005624       Java_jdk_internal_reflect_Reflection_getClassAccessFlags 0000000180006624 f   Reflection.obj
 0001:0000562c       Java_java_lang_Runtime_availableProcessors 000000018000662c f   Runtime.obj
 0001:00005634       Java_java_lang_Runtime_freeMemory 0000000180006634 f   Runtime.obj
 0001:0000563c       Java_java_lang_Runtime_gc  000000018000663c f   Runtime.obj
 0001:00005644       Java_java_lang_Runtime_maxMemory 0000000180006644 f   Runtime.obj
 0001:0000564c       Java_java_lang_Runtime_totalMemory 000000018000664c f   Runtime.obj
 0001:00005654       Java_java_lang_SecurityManager_getClassContext 0000000180006654 f   SecurityManager.obj
 0001:00005718       Java_java_lang_Shutdown_beforeHalt 0000000180006718 f   Shutdown.obj
 0001:00005720       Java_java_lang_Shutdown_halt0 0000000180006720 f   Shutdown.obj
 0001:00005728       Java_jdk_internal_misc_Signal_findSignal0 0000000180006728 f   Signal.obj
 0001:000057a4       Java_jdk_internal_misc_Signal_handle0 00000001800067a4 f   Signal.obj
 0001:000057b0       Java_jdk_internal_misc_Signal_raise0 00000001800067b0 f   Signal.obj
 0001:000057b8       Java_java_lang_StackStreamFactory_00024AbstractStackWalker_callStackWalk 00000001800067b8 f   StackStreamFactory.obj
 0001:000057c0       Java_java_lang_StackStreamFactory_00024AbstractStackWalker_fetchStackFrames 00000001800067c0 f   StackStreamFactory.obj
 0001:000057c8       Java_java_lang_StackStreamFactory_checkStackWalkModes 00000001800067c8 f   StackStreamFactory.obj
 0001:000057c8       __acrt_initialize          00000001800067c8 f   MSVCRT:ucrt_stubs.obj
 0001:000057c8       __acrt_thread_attach       00000001800067c8 f   MSVCRT:ucrt_stubs.obj
 0001:000057c8       __acrt_thread_detach       00000001800067c8 f   MSVCRT:ucrt_stubs.obj
 0001:000057c8       __acrt_uninitialize        00000001800067c8 f   MSVCRT:ucrt_stubs.obj
 0001:000057c8       __acrt_uninitialize_critical 00000001800067c8 f   MSVCRT:ucrt_stubs.obj
 0001:000057c8       __scrt_stub_for_acrt_initialize 00000001800067c8 f   MSVCRT:ucrt_stubs.obj
 0001:000057c8       __scrt_stub_for_acrt_thread_attach 00000001800067c8 f   MSVCRT:ucrt_stubs.obj
 0001:000057c8       __scrt_stub_for_acrt_thread_detach 00000001800067c8 f   MSVCRT:ucrt_stubs.obj
 0001:000057c8       __scrt_stub_for_acrt_uninitialize 00000001800067c8 f   MSVCRT:ucrt_stubs.obj
 0001:000057c8       __scrt_stub_for_acrt_uninitialize_critical 00000001800067c8 f   MSVCRT:ucrt_stubs.obj
 0001:000057c8       __vcrt_initialize          00000001800067c8 f   MSVCRT:ucrt_stubs.obj
 0001:000057c8       __vcrt_thread_attach       00000001800067c8 f   MSVCRT:ucrt_stubs.obj
 0001:000057c8       __vcrt_thread_detach       00000001800067c8 f   MSVCRT:ucrt_stubs.obj
 0001:000057c8       __vcrt_uninitialize        00000001800067c8 f   MSVCRT:ucrt_stubs.obj
 0001:000057c8       __vcrt_uninitialize_critical 00000001800067c8 f   MSVCRT:ucrt_stubs.obj
 0001:000057cc       Java_java_lang_StackTraceElement_initStackTraceElement 00000001800067cc f   StackTraceElement.obj
 0001:000057d8       Java_java_lang_StackTraceElement_initStackTraceElements 00000001800067d8 f   StackTraceElement.obj
 0001:000057e4       Java_java_lang_StrictMath_IEEEremainder 00000001800067e4 f   StrictMath.obj
 0001:000057fc       Java_java_lang_StrictMath_acos 00000001800067fc f   StrictMath.obj
 0001:0000580c       Java_java_lang_StrictMath_asin 000000018000680c f   StrictMath.obj
 0001:0000581c       Java_java_lang_StrictMath_atan 000000018000681c f   StrictMath.obj
 0001:0000582c       Java_java_lang_StrictMath_atan2 000000018000682c f   StrictMath.obj
 0001:00005844       Java_java_lang_StrictMath_cos 0000000180006844 f   StrictMath.obj
 0001:00005854       Java_java_lang_StrictMath_cosh 0000000180006854 f   StrictMath.obj
 0001:00005864       Java_java_lang_StrictMath_expm1 0000000180006864 f   StrictMath.obj
 0001:00005874       Java_java_lang_StrictMath_log 0000000180006874 f   StrictMath.obj
 0001:00005884       Java_java_lang_StrictMath_log10 0000000180006884 f   StrictMath.obj
 0001:00005894       Java_java_lang_StrictMath_log1p 0000000180006894 f   StrictMath.obj
 0001:000058a4       Java_java_lang_StrictMath_sin 00000001800068a4 f   StrictMath.obj
 0001:000058b4       Java_java_lang_StrictMath_sinh 00000001800068b4 f   StrictMath.obj
 0001:000058c4       Java_java_lang_StrictMath_sqrt 00000001800068c4 f   StrictMath.obj
 0001:000058d4       Java_java_lang_StrictMath_tan 00000001800068d4 f   StrictMath.obj
 0001:000058e4       Java_java_lang_StrictMath_tanh 00000001800068e4 f   StrictMath.obj
 0001:000058f4       Java_java_lang_String_intern 00000001800068f4 f   String.obj
 0001:000058fc       Java_java_lang_StringCoding_err 00000001800068fc f   StringCoding.obj
 0001:00005a18       Java_java_lang_System_identityHashCode 0000000180006a18 f   System.obj
 0001:00005a20       Java_java_lang_System_initProperties 0000000180006a20 f   System.obj
 0001:00006f44       Java_java_lang_System_mapLibraryName 0000000180007f44 f   System.obj
 0001:00007084       Java_java_lang_System_registerNatives 0000000180008084 f   System.obj
 0001:0000709c       Java_java_lang_System_setErr0 000000018000809c f   System.obj
 0001:000070f8       Java_java_lang_System_setIn0 00000001800080f8 f   System.obj
 0001:00007154       Java_java_lang_System_setOut0 0000000180008154 f   System.obj
 0001:000071b0       fillI18nProps              00000001800081b0 f   System.obj
 0001:00007588       Java_java_lang_Thread_registerNatives 0000000180008588 f   Thread.obj
 0001:000075a0       Java_java_lang_Throwable_fillInStackTrace 00000001800085a0 f   Throwable.obj
 0001:000075b8       Java_java_util_TimeZone_getSystemGMTOffsetID 00000001800085b8 f   TimeZone.obj
 0001:00007604       Java_java_util_TimeZone_getSystemTimeZoneID 0000000180008604 f   TimeZone.obj
 0001:00007708       findJavaTZ_md              0000000180008708 f   TimeZone_md.obj
 0001:00007790       getGMTOffsetID             0000000180008790 f   TimeZone_md.obj
 0001:000080e8       Java_jdk_internal_misc_VM_getRuntimeArguments 00000001800090e8 f   VM.obj
 0001:000080f0       Java_jdk_internal_misc_VM_initialize 00000001800090f0 f   VM.obj
 0001:00008140       Java_jdk_internal_misc_VM_initializeFromArchive 0000000180009140 f   VM.obj
 0001:00008148       Java_jdk_internal_misc_VM_latestUserDefinedLoader0 0000000180009148 f   VM.obj
 0001:00008150       Java_jdk_internal_vm_VMSupport_getVMTemporaryDirectory 0000000180009150 f   VMSupport.obj
 0001:00008158       Java_jdk_internal_vm_VMSupport_initAgentProperties 0000000180009158 f   VMSupport.obj
 0001:00008160       Java_jdk_internal_misc_VM_getegid 0000000180009160 f   VM_md.obj
 0001:00008160       Java_jdk_internal_misc_VM_geteuid 0000000180009160 f   VM_md.obj
 0001:00008160       Java_jdk_internal_misc_VM_getgid 0000000180009160 f   VM_md.obj
 0001:00008160       Java_jdk_internal_misc_VM_getuid 0000000180009160 f   VM_md.obj
 0001:00008168       Java_sun_io_Win32ErrorMode_setErrorMode 0000000180009168 f   Win32ErrorMode.obj
 0001:0000817c       Java_sun_security_provider_NativeSeedGenerator_nativeGenerateSeed 000000018000917c f   WinCAPISeedGenerator.obj
 0001:0000825c       Java_java_io_WinNTFileSystem_canonicalize0 000000018000925c f   WinNTFileSystem_md.obj
 0001:000083d0       Java_java_io_WinNTFileSystem_canonicalizeWithPrefix0 00000001800093d0 f   WinNTFileSystem_md.obj
 0001:0000858c       Java_java_io_WinNTFileSystem_checkAccess 000000018000958c f   WinNTFileSystem_md.obj
 0001:00008608       Java_java_io_WinNTFileSystem_createDirectory 0000000180009608 f   WinNTFileSystem_md.obj
 0001:00008650       Java_java_io_WinNTFileSystem_createFileExclusively 0000000180009650 f   WinNTFileSystem_md.obj
 0001:00008724       Java_java_io_WinNTFileSystem_delete0 0000000180009724 f   WinNTFileSystem_md.obj
 0001:00008794       Java_java_io_WinNTFileSystem_getBooleanAttributes 0000000180009794 f   WinNTFileSystem_md.obj
 0001:000087fc       Java_java_io_WinNTFileSystem_getDriveDirectory 00000001800097fc f   WinNTFileSystem_md.obj
 0001:00008884       Java_java_io_WinNTFileSystem_getLastModifiedTime 0000000180009884 f   WinNTFileSystem_md.obj
 0001:0000893c       Java_java_io_WinNTFileSystem_getLength 000000018000993c f   WinNTFileSystem_md.obj
 0001:00008ab4       Java_java_io_WinNTFileSystem_getNameMax0 0000000180009ab4 f   WinNTFileSystem_md.obj
 0001:00008b7c       Java_java_io_WinNTFileSystem_getSpace0 0000000180009b7c f   WinNTFileSystem_md.obj
 0001:00008c40       Java_java_io_WinNTFileSystem_initIDs 0000000180009c40 f   WinNTFileSystem_md.obj
 0001:00008cc0       Java_java_io_WinNTFileSystem_list 0000000180009cc0 f   WinNTFileSystem_md.obj
 0001:00008ff8       Java_java_io_WinNTFileSystem_listRoots0 0000000180009ff8 f   WinNTFileSystem_md.obj
 0001:00009000       Java_java_io_WinNTFileSystem_rename0 000000018000a000 f   WinNTFileSystem_md.obj
 0001:00009094       Java_java_io_WinNTFileSystem_setLastModifiedTime 000000018000a094 f   WinNTFileSystem_md.obj
 0001:00009160       Java_java_io_WinNTFileSystem_setPermission 000000018000a160 f   WinNTFileSystem_md.obj
 0001:00009240       Java_java_io_WinNTFileSystem_setReadOnly 000000018000a240 f   WinNTFileSystem_md.obj
 0001:0000936c       getFinalAttributes         000000018000a36c f   WinNTFileSystem_md.obj
 0001:0000941c       getFinalAttributesIfReparsePoint 000000018000a41c f   WinNTFileSystem_md.obj
 0001:00009788       canonicalize               000000018000a788 f   canonicalize_md.obj
 0001:00009bfc       getPrefixed                000000018000abfc f   canonicalize_md.obj
 0001:00009c94       lastErrorReportable        000000018000ac94 f   canonicalize_md.obj
 0001:00009d24       wcanonicalize              000000018000ad24 f   canonicalize_md.obj
 0001:0000a048       wcanonicalizeWithPrefix    000000018000b048 f   canonicalize_md.obj
 0001:0000a1f8       JNI_OnLoad                 000000018000b1f8 f   check_version.obj
 0001:0000a288       readBytes                  000000018000b288 f   io_util.obj
 0001:0000a42c       readSingle                 000000018000b42c f   io_util.obj
 0001:0000a4dc       throwFileNotFoundException 000000018000b4dc f   io_util.obj
 0001:0000a588       writeBytes                 000000018000b588 f   io_util.obj
 0001:0000a748       writeSingle                000000018000b748 f   io_util.obj
 0001:0000a804       currentDir                 000000018000b804 f   io_util_md.obj
 0001:0000a86c       currentDirLength           000000018000b86c f   io_util_md.obj
 0001:0000a918       fileDescriptorClose        000000018000b918 f   io_util_md.obj
 0001:0000a9ac       fileOpen                   000000018000b9ac f   io_util_md.obj
 0001:0000aa78       fileToNTPath               000000018000ba78 f   io_util_md.obj
 0001:0000aaa4       handleAppend               000000018000baa4 f   io_util_md.obj
 0001:0000aaec       handleAvailable            000000018000baec f   io_util_md.obj
 0001:0000abdc       handleGetLength            000000018000bbdc f   io_util_md.obj
 0001:0000ac00       handleLseek                000000018000bc00 f   io_util_md.obj
 0001:0000ac48       handleRead                 000000018000bc48 f   io_util_md.obj
 0001:0000ac8c       handleSetLength            000000018000bc8c f   io_util_md.obj
 0001:0000ae0c       handleSync                 000000018000be0c f   io_util_md.obj
 0001:0000ae30       handleWrite                000000018000be30 f   io_util_md.obj
 0001:0000ae68       pathToNTPath               000000018000be68 f   io_util_md.obj
 0001:0000afdc       prefixAbpath               000000018000bfdc f   io_util_md.obj
 0001:0000b084       winFileHandleOpen          000000018000c084 f   io_util_md.obj
 0001:0000b178       GetJavaProperties          000000018000c178 f   java_props_md.obj
 0001:0000b858       GetStringPlatform          000000018000c858 f   java_props_md.obj
 0001:0000baa0       __local_stdio_scanf_options 000000018000caa0 f i java_props_md.obj
 0001:0000bbc0       getEncodingFromLangID      000000018000cbc0 f   java_props_md.obj
 0001:0000bddc       getHomeFromShell32         000000018000cddc f   java_props_md.obj
 0001:0000be98       getJavaIDFromLangID        000000018000ce98 f   java_props_md.obj
 0001:0000bf8c       sscanf                     000000018000cf8c f i java_props_md.obj
 0001:0000bfd8       JDK_GetVersionInfo0        000000018000cfd8 f   jdk_util.obj
 0001:0000c000       JDK_InitJvmHandle          000000018000d000 f   jdk_util_md.obj
 0001:0000c028       JDK_LoadSystemLibrary      000000018000d028 f   jdk_util_md.obj
 0001:0000c0f8       jio_fprintf                000000018000d0f8 f   jio.obj
 0001:0000c11c       jio_snprintf               000000018000d11c f   jio.obj
 0001:0000c13c       Canonicalize               000000018000d13c f   jni_util.obj
 0001:0000c150       GetStringPlatformChars     000000018000d150 f   jni_util.obj
 0001:0000c158       InitializeEncoding         000000018000d158 f   jni_util.obj
 0001:0000c3b0       JNU_CallMethodByName       000000018000d3b0 f   jni_util.obj
 0001:0000c3d4       JNU_CallMethodByNameV      000000018000d3d4 f   jni_util.obj
 0001:0000c61c       JNU_CallStaticMethodByName 000000018000d61c f   jni_util.obj
 0001:0000c810       JNU_ClassClass             000000018000d810 f   jni_util.obj
 0001:0000c890       JNU_ClassObject            000000018000d890 f   jni_util.obj
 0001:0000c910       JNU_ClassString            000000018000d910 f   jni_util.obj
 0001:0000c990       JNU_ClassThrowable         000000018000d990 f   jni_util.obj
 0001:0000ca10       JNU_CopyObjectArray        000000018000da10 f   jni_util.obj
 0001:0000cab0       JNU_Equals                 000000018000dab0 f   jni_util.obj
 0001:0000cb34       JNU_GetEnv                 000000018000db34 f   jni_util.obj
 0001:0000cb50       JNU_GetFieldByName         000000018000db50 f   jni_util.obj
 0001:0000cd24       JNU_GetStaticFieldByName   000000018000dd24 f   jni_util.obj
 0001:0000cef0       JNU_GetStringPlatformChars 000000018000def0 f   jni_util.obj
 0001:0000cf64       JNU_IsInstanceOfByName     000000018000df64 f   jni_util.obj
 0001:0000cfec       JNU_MonitorWait            000000018000dfec f   jni_util.obj
 0001:0000d084       JNU_NewObjectByName        000000018000e084 f   jni_util.obj
 0001:0000d11c       JNU_NewStringPlatform      000000018000e11c f   jni_util.obj
 0001:0000d1cc       JNU_Notify                 000000018000e1cc f   jni_util.obj
 0001:0000d254       JNU_NotifyAll              000000018000e254 f   jni_util.obj
 0001:0000d2dc       JNU_PrintClass             000000018000e2dc f   jni_util.obj
 0001:0000d3ac       JNU_PrintString            000000018000e3ac f   jni_util.obj
 0001:0000d428       JNU_ReleaseStringPlatformChars 000000018000e428 f   jni_util.obj
 0001:0000d434       JNU_SetFieldByName         000000018000e434 f   jni_util.obj
 0001:0000d5f0       JNU_SetStaticFieldByName   000000018000e5f0 f   jni_util.obj
 0001:0000d7b0       JNU_ThrowArrayIndexOutOfBoundsException 000000018000e7b0 f   jni_util.obj
 0001:0000d7c0       JNU_ThrowByName            000000018000e7c0 f   jni_util.obj
 0001:0000d7f8       JNU_ThrowByNameWithLastError 000000018000e7f8 f   jni_util.obj
 0001:0000d8a4       JNU_ThrowByNameWithMessageAndLastError 000000018000e8a4 f   jni_util.obj
 0001:0000da60       JNU_ThrowClassNotFoundException 000000018000ea60 f   jni_util.obj
 0001:0000da70       JNU_ThrowIOException       000000018000ea70 f   jni_util.obj
 0001:0000da80       JNU_ThrowIOExceptionWithLastError 000000018000ea80 f   jni_util.obj
 0001:0000da90       JNU_ThrowIllegalAccessError 000000018000ea90 f   jni_util.obj
 0001:0000daa0       JNU_ThrowIllegalAccessException 000000018000eaa0 f   jni_util.obj
 0001:0000dab0       JNU_ThrowIllegalArgumentException 000000018000eab0 f   jni_util.obj
 0001:0000dac0       JNU_ThrowInstantiationException 000000018000eac0 f   jni_util.obj
 0001:0000dad0       JNU_ThrowInternalError     000000018000ead0 f   jni_util.obj
 0001:0000dae0       JNU_ThrowNoSuchFieldError  000000018000eae0 f   jni_util.obj
 0001:0000daf0       JNU_ThrowNoSuchFieldException 000000018000eaf0 f   jni_util.obj
 0001:0000db00       JNU_ThrowNoSuchMethodError 000000018000eb00 f   jni_util.obj
 0001:0000db10       JNU_ThrowNoSuchMethodException 000000018000eb10 f   jni_util.obj
 0001:0000db20       JNU_ThrowNullPointerException 000000018000eb20 f   jni_util.obj
 0001:0000db30       JNU_ThrowNumberFormatException 000000018000eb30 f   jni_util.obj
 0001:0000db40       JNU_ThrowOutOfMemoryError  000000018000eb40 f   jni_util.obj
 0001:0000db50       JNU_ThrowStringIndexOutOfBoundsException 000000018000eb50 f   jni_util.obj
 0001:0000db60       JNU_ToString               000000018000eb60 f   jni_util.obj
 0001:0000dba0       NewStringPlatform          000000018000eba0 f   jni_util.obj
 0001:0000dba8       fprintf                    000000018000eba8 f i jni_util.obj
 0001:0000e7b0       buildJniFunctionName       000000018000f7b0 f   jni_util_md.obj
 0001:0000e86c       getErrorString             000000018000f86c f   jni_util_md.obj
 0001:0000e890       getLastErrorString         000000018000f890 f   jni_util_md.obj
 0001:0000e93c       getProcessHandle           000000018000f93c f   jni_util_md.obj
 0001:0000e948       VerifyClassCodes           000000018000f948 f   verify_stub.obj
 0001:0000e950       VerifyClassCodesForMajorVersion 000000018000f950 f   verify_stub.obj
 0001:0000e960       jacos                      000000018000f960 f   fdlibm:w_acos.obj
 0001:0000e980       jasin                      000000018000f980 f   fdlibm:w_asin.obj
 0001:0000e9a0       jatan                      000000018000f9a0 f   fdlibm:s_atan.obj
 0001:0000eea0       jatan2                     000000018000fea0 f   fdlibm:w_atan2.obj
 0001:0000eed0       jcos                       000000018000fed0 f   fdlibm:s_cos.obj
 0001:0000f060       jsin                       0000000180010060 f   fdlibm:s_sin.obj
 0001:0000f200       jtan                       0000000180010200 f   fdlibm:s_tan.obj
 0001:0000f2e0       jcosh                      00000001800102e0 f   fdlibm:w_cosh.obj
 0001:0000f300       jsinh                      0000000180010300 f   fdlibm:w_sinh.obj
 0001:0000f320       jtanh                      0000000180010320 f   fdlibm:s_tanh.obj
 0001:0000f4e0       jlog                       00000001800104e0 f   fdlibm:w_log.obj
 0001:0000f500       jlog10                     0000000180010500 f   fdlibm:w_log10.obj
 0001:0000f520       jsqrt                      0000000180010520 f   fdlibm:w_sqrt.obj
 0001:0000f540       jremainder                 0000000180010540 f   fdlibm:w_remainder.obj
 0001:0000f570       jexpm1                     0000000180010570 f   fdlibm:s_expm1.obj
 0001:0000fbc0       jlog1p                     0000000180010bc0 f   fdlibm:s_log1p.obj
 0001:000100e0       __ieee754_acos             00000001800110e0 f   fdlibm:e_acos.obj
 0001:000106d0       __ieee754_asin             00000001800116d0 f   fdlibm:e_asin.obj
 0001:00010bf0       jfabs                      0000000180011bf0 f   fdlibm:s_fabs.obj
 0001:00010c10       __ieee754_atan2            0000000180011c10 f   fdlibm:e_atan2.obj
 0001:00011040       __ieee754_rem_pio2         0000000180012040 f   fdlibm:e_rem_pio2.obj
 0001:000117f0       __kernel_sin               00000001800127f0 f   fdlibm:k_sin.obj
 0001:00011960       __kernel_cos               0000000180012960 f   fdlibm:k_cos.obj
 0001:00011b40       __kernel_tan               0000000180012b40 f   fdlibm:k_tan.obj
 0001:00012170       __ieee754_cosh             0000000180013170 f   fdlibm:e_cosh.obj
 0001:00012350       __ieee754_sinh             0000000180013350 f   fdlibm:e_sinh.obj
 0001:00012560       __ieee754_log              0000000180013560 f   fdlibm:e_log.obj
 0001:000129f0       __ieee754_log10            00000001800139f0 f   fdlibm:e_log10.obj
 0001:00012b70       __ieee754_sqrt             0000000180013b70 f   fdlibm:e_sqrt.obj
 0001:00013010       __ieee754_remainder        0000000180014010 f   fdlibm:e_remainder.obj
 0001:00013240       __kernel_rem_pio2          0000000180014240 f   fdlibm:k_rem_pio2.obj
 0001:00013f80       __ieee754_exp              0000000180014f80 f   fdlibm:e_exp.obj
 0001:00014320       __ieee754_fmod             0000000180015320 f   fdlibm:e_fmod.obj
 0001:000148d0       jfloor                     00000001800158d0 f   fdlibm:s_floor.obj
 0001:00014b00       scalbn                     0000000180015b00 f   fdlibm:s_scalbn.obj
 0001:00014ce0       copysign                   0000000180015ce0 f   fdlibm:s_copysign.obj
 0001:00014d0b       JVM_DoPrivileged           0000000180015d0b f   jvm:jvm.dll
 0001:00014d11       JVM_GetInheritedAccessControlContext 0000000180015d11 f   jvm:jvm.dll
 0001:00014d17       JVM_GetStackAccessControlContext 0000000180015d17 f   jvm:jvm.dll
 0001:00014d1d       JVM_GetArrayLength         0000000180015d1d f   jvm:jvm.dll
 0001:00014d23       JVM_GetArrayElement        0000000180015d23 f   jvm:jvm.dll
 0001:00014d29       JVM_GetPrimitiveArrayElement 0000000180015d29 f   jvm:jvm.dll
 0001:00014d2f       JVM_SetArrayElement        0000000180015d2f f   jvm:jvm.dll
 0001:00014d35       JVM_SetPrimitiveArrayElement 0000000180015d35 f   jvm:jvm.dll
 0001:00014d3b       JVM_NewArray               0000000180015d3b f   jvm:jvm.dll
 0001:00014d41       JVM_NewMultiArray          0000000180015d41 f   jvm:jvm.dll
 0001:00014d47       JVM_SupportsCX8            0000000180015d47 f   jvm:jvm.dll
 0001:00014d4d       JVM_GetSystemPackage       0000000180015d4d f   jvm:jvm.dll
 0001:00014d53       JVM_GetSystemPackages      0000000180015d53 f   jvm:jvm.dll
 0001:00014d59       JVM_SetBootLoaderUnnamedModule 0000000180015d59 f   jvm:jvm.dll
 0001:00014d5f       JVM_InitClassName          0000000180015d5f f   jvm:jvm.dll
 0001:00014d65       JVM_GetClassInterfaces     0000000180015d65 f   jvm:jvm.dll
 0001:00014d6b       JVM_IsInterface            0000000180015d6b f   jvm:jvm.dll
 0001:00014d71       JVM_GetClassSigners        0000000180015d71 f   jvm:jvm.dll
 0001:00014d77       JVM_SetClassSigners        0000000180015d77 f   jvm:jvm.dll
 0001:00014d7d       JVM_GetProtectionDomain    0000000180015d7d f   jvm:jvm.dll
 0001:00014d83       JVM_IsArrayClass           0000000180015d83 f   jvm:jvm.dll
 0001:00014d89       JVM_IsPrimitiveClass       0000000180015d89 f   jvm:jvm.dll
 0001:00014d8f       JVM_GetClassModifiers      0000000180015d8f f   jvm:jvm.dll
 0001:00014d95       JVM_GetDeclaredClasses     0000000180015d95 f   jvm:jvm.dll
 0001:00014d9b       JVM_GetDeclaringClass      0000000180015d9b f   jvm:jvm.dll
 0001:00014da1       JVM_GetSimpleBinaryName    0000000180015da1 f   jvm:jvm.dll
 0001:00014da7       JVM_GetClassSignature      0000000180015da7 f   jvm:jvm.dll
 0001:00014dad       JVM_GetClassAnnotations    0000000180015dad f   jvm:jvm.dll
 0001:00014db3       JVM_GetClassTypeAnnotations 0000000180015db3 f   jvm:jvm.dll
 0001:00014db9       JVM_GetClassDeclaredMethods 0000000180015db9 f   jvm:jvm.dll
 0001:00014dbf       JVM_GetClassDeclaredFields 0000000180015dbf f   jvm:jvm.dll
 0001:00014dc5       JVM_GetClassDeclaredConstructors 0000000180015dc5 f   jvm:jvm.dll
 0001:00014dcb       JVM_GetNestHost            0000000180015dcb f   jvm:jvm.dll
 0001:00014dd1       JVM_GetNestMembers         0000000180015dd1 f   jvm:jvm.dll
 0001:00014dd7       JVM_GetClassConstantPool   0000000180015dd7 f   jvm:jvm.dll
 0001:00014ddd       JVM_DesiredAssertionStatus 0000000180015ddd f   jvm:jvm.dll
 0001:00014de3       JVM_GetEnclosingMethodInfo 0000000180015de3 f   jvm:jvm.dll
 0001:00014de9       JVM_FindPrimitiveClass     0000000180015de9 f   jvm:jvm.dll
 0001:00014def       JVM_FindClassFromCaller    0000000180015def f   jvm:jvm.dll
 0001:00014df5       JVM_AssertionStatusDirectives 0000000180015df5 f   jvm:jvm.dll
 0001:00014dfb       JVM_LoadLibrary            0000000180015dfb f   jvm:jvm.dll
 0001:00014e01       JVM_UnloadLibrary          0000000180015e01 f   jvm:jvm.dll
 0001:00014e07       JVM_FindLibraryEntry       0000000180015e07 f   jvm:jvm.dll
 0001:00014e0d       JVM_IsSupportedJNIVersion  0000000180015e0d f   jvm:jvm.dll
 0001:00014e13       JVM_FindClassFromBootLoader 0000000180015e13 f   jvm:jvm.dll
 0001:00014e19       JVM_FindLoadedClass        0000000180015e19 f   jvm:jvm.dll
 0001:00014e1f       JVM_DefineClassWithSource  0000000180015e1f f   jvm:jvm.dll
 0001:00014e25       JVM_ConstantPoolGetSize    0000000180015e25 f   jvm:jvm.dll
 0001:00014e2b       JVM_ConstantPoolGetClassAt 0000000180015e2b f   jvm:jvm.dll
 0001:00014e31       JVM_ConstantPoolGetClassAtIfLoaded 0000000180015e31 f   jvm:jvm.dll
 0001:00014e37       JVM_ConstantPoolGetClassRefIndexAt 0000000180015e37 f   jvm:jvm.dll
 0001:00014e3d       JVM_ConstantPoolGetMethodAt 0000000180015e3d f   jvm:jvm.dll
 0001:00014e43       JVM_ConstantPoolGetMethodAtIfLoaded 0000000180015e43 f   jvm:jvm.dll
 0001:00014e49       JVM_ConstantPoolGetFieldAt 0000000180015e49 f   jvm:jvm.dll
 0001:00014e4f       JVM_ConstantPoolGetFieldAtIfLoaded 0000000180015e4f f   jvm:jvm.dll
 0001:00014e55       JVM_ConstantPoolGetMemberRefInfoAt 0000000180015e55 f   jvm:jvm.dll
 0001:00014e5b       JVM_ConstantPoolGetNameAndTypeRefIndexAt 0000000180015e5b f   jvm:jvm.dll
 0001:00014e61       JVM_ConstantPoolGetNameAndTypeRefInfoAt 0000000180015e61 f   jvm:jvm.dll
 0001:00014e67       JVM_ConstantPoolGetIntAt   0000000180015e67 f   jvm:jvm.dll
 0001:00014e6d       JVM_ConstantPoolGetLongAt  0000000180015e6d f   jvm:jvm.dll
 0001:00014e73       JVM_ConstantPoolGetFloatAt 0000000180015e73 f   jvm:jvm.dll
 0001:00014e79       JVM_ConstantPoolGetDoubleAt 0000000180015e79 f   jvm:jvm.dll
 0001:00014e7f       JVM_ConstantPoolGetStringAt 0000000180015e7f f   jvm:jvm.dll
 0001:00014e85       JVM_ConstantPoolGetUTF8At  0000000180015e85 f   jvm:jvm.dll
 0001:00014e8b       JVM_ConstantPoolGetTagAt   0000000180015e8b f   jvm:jvm.dll
 0001:00014e91       JVM_GetMethodTypeAnnotations 0000000180015e91 f   jvm:jvm.dll
 0001:00014e97       JVM_GetMethodParameters    0000000180015e97 f   jvm:jvm.dll
 0001:00014e9d       JVM_GetFieldTypeAnnotations 0000000180015e9d f   jvm:jvm.dll
 0001:00014ea3       JVM_DefineModule           0000000180015ea3 f   jvm:jvm.dll
 0001:00014ea9       JVM_AddModuleExports       0000000180015ea9 f   jvm:jvm.dll
 0001:00014eaf       JVM_AddModuleExportsToAllUnnamed 0000000180015eaf f   jvm:jvm.dll
 0001:00014eb5       JVM_AddModuleExportsToAll  0000000180015eb5 f   jvm:jvm.dll
 0001:00014ebb       JVM_AddReadsModule         0000000180015ebb f   jvm:jvm.dll
 0001:00014ec1       JVM_InvokeMethod           0000000180015ec1 f   jvm:jvm.dll
 0001:00014ec7       JVM_NewInstanceFromConstructor 0000000180015ec7 f   jvm:jvm.dll
 0001:00014ecd       JVM_IHashCode              0000000180015ecd f   jvm:jvm.dll
 0001:00014ed3       JVM_MonitorWait            0000000180015ed3 f   jvm:jvm.dll
 0001:00014ed9       JVM_MonitorNotify          0000000180015ed9 f   jvm:jvm.dll
 0001:00014edf       JVM_MonitorNotifyAll       0000000180015edf f   jvm:jvm.dll
 0001:00014ee5       JVM_Clone                  0000000180015ee5 f   jvm:jvm.dll
 0001:00014eeb       JVM_GetThreadInterruptEvent 0000000180015eeb f   jvm:jvm.dll
 0001:00014ef1       JVM_GetAndClearReferencePendingList 0000000180015ef1 f   jvm:jvm.dll
 0001:00014ef7       JVM_HasReferencePendingList 0000000180015ef7 f   jvm:jvm.dll
 0001:00014efd       JVM_WaitForReferencePendingList 0000000180015efd f   jvm:jvm.dll
 0001:00014f03       JVM_GetCallerClass         0000000180015f03 f   jvm:jvm.dll
 0001:00014f09       JVM_GetClassAccessFlags    0000000180015f09 f   jvm:jvm.dll
 0001:00014f0f       JVM_AreNestMates           0000000180015f0f f   jvm:jvm.dll
 0001:00014f15       JVM_GC                     0000000180015f15 f   jvm:jvm.dll
 0001:00014f1b       JVM_TotalMemory            0000000180015f1b f   jvm:jvm.dll
 0001:00014f21       JVM_FreeMemory             0000000180015f21 f   jvm:jvm.dll
 0001:00014f27       JVM_MaxMemory              0000000180015f27 f   jvm:jvm.dll
 0001:00014f2d       JVM_ActiveProcessorCount   0000000180015f2d f   jvm:jvm.dll
 0001:00014f33       JVM_GetClassContext        0000000180015f33 f   jvm:jvm.dll
 0001:00014f39       JVM_BeforeHalt             0000000180015f39 f   jvm:jvm.dll
 0001:00014f3f       JVM_Halt                   0000000180015f3f f   jvm:jvm.dll
 0001:00014f45       JVM_RegisterSignal         0000000180015f45 f   jvm:jvm.dll
 0001:00014f4b       JVM_RaiseSignal            0000000180015f4b f   jvm:jvm.dll
 0001:00014f51       JVM_FindSignal             0000000180015f51 f   jvm:jvm.dll
 0001:00014f57       JVM_CallStackWalk          0000000180015f57 f   jvm:jvm.dll
 0001:00014f5d       JVM_MoreStackWalk          0000000180015f5d f   jvm:jvm.dll
 0001:00014f63       JVM_InitStackTraceElementArray 0000000180015f63 f   jvm:jvm.dll
 0001:00014f69       JVM_InitStackTraceElement  0000000180015f69 f   jvm:jvm.dll
 0001:00014f6f       JVM_InternString           0000000180015f6f f   jvm:jvm.dll
 0001:00014f75       JVM_CurrentTimeMillis      0000000180015f75 f   jvm:jvm.dll
 0001:00014f7b       JVM_NanoTime               0000000180015f7b f   jvm:jvm.dll
 0001:00014f81       JVM_ArrayCopy              0000000180015f81 f   jvm:jvm.dll
 0001:00014f87       JVM_InitProperties         0000000180015f87 f   jvm:jvm.dll
 0001:00014f8d       JVM_StartThread            0000000180015f8d f   jvm:jvm.dll
 0001:00014f93       JVM_StopThread             0000000180015f93 f   jvm:jvm.dll
 0001:00014f99       JVM_IsThreadAlive          0000000180015f99 f   jvm:jvm.dll
 0001:00014f9f       JVM_SuspendThread          0000000180015f9f f   jvm:jvm.dll
 0001:00014fa5       JVM_ResumeThread           0000000180015fa5 f   jvm:jvm.dll
 0001:00014fab       JVM_SetThreadPriority      0000000180015fab f   jvm:jvm.dll
 0001:00014fb1       JVM_Yield                  0000000180015fb1 f   jvm:jvm.dll
 0001:00014fb7       JVM_Sleep                  0000000180015fb7 f   jvm:jvm.dll
 0001:00014fbd       JVM_CurrentThread          0000000180015fbd f   jvm:jvm.dll
 0001:00014fc3       JVM_CountStackFrames       0000000180015fc3 f   jvm:jvm.dll
 0001:00014fc9       JVM_Interrupt              0000000180015fc9 f   jvm:jvm.dll
 0001:00014fcf       JVM_IsInterrupted          0000000180015fcf f   jvm:jvm.dll
 0001:00014fd5       JVM_HoldsLock              0000000180015fd5 f   jvm:jvm.dll
 0001:00014fdb       JVM_GetAllThreads          0000000180015fdb f   jvm:jvm.dll
 0001:00014fe1       JVM_SetNativeThreadName    0000000180015fe1 f   jvm:jvm.dll
 0001:00014fe7       JVM_DumpThreads            0000000180015fe7 f   jvm:jvm.dll
 0001:00014fed       JVM_FillInStackTrace       0000000180015fed f   jvm:jvm.dll
 0001:00014ff3       JVM_GetNanoTimeAdjustment  0000000180015ff3 f   jvm:jvm.dll
 0001:00014ff9       JVM_GetVmArguments         0000000180015ff9 f   jvm:jvm.dll
 0001:00014fff       JVM_InitializeFromArchive  0000000180015fff f   jvm:jvm.dll
 0001:00015005       JVM_LatestUserDefinedLoader 0000000180016005 f   jvm:jvm.dll
 0001:0001500b       JVM_InitAgentProperties    000000018001600b f   jvm:jvm.dll
 0001:00015011       JVM_GetTemporaryDirectory  0000000180016011 f   jvm:jvm.dll
 0001:00015017       JVM_GetInterfaceVersion    0000000180016017 f   jvm:jvm.dll
 0001:0001501d       jio_vsnprintf              000000018001601d f   jvm:jvm.dll
 0001:00015023       jio_vfprintf               0000000180016023 f   jvm:jvm.dll
 0001:00015029       VerifyClassname            0000000180016029 f   verify:verify.dll
 0001:0001502f       VerifyFixClassname         000000018001602f f   verify:verify.dll
 0001:00015035       __imp_load_SHGetFolderPathW 0000000180016035 f   shell32:SHELL32.dll
 0001:00015041       __tailMerge_shell32_dll    0000000180016041     shell32:SHELL32.dll
 0001:000150ba       __imp_load_SHGetKnownFolderPath 00000001800160ba f   shell32:SHELL32.dll
 0001:000150c6       SHGetKnownFolderPath       00000001800160c6 f   shell32:SHELL32.dll
 0001:000150cc       ?DloadAcquireSectionWriteAccess@@YAXXZ 00000001800160cc f i delayimp:delayhlp.obj
 0001:00015178       ?DloadGetSRWLockFunctionPointers@@YAEXZ 0000000180016178 f i delayimp:delayhlp.obj
 0001:00015218       ?DloadMakePermanentImageCommit@@YAXPEAX_K@Z 0000000180016218 f i delayimp:delayhlp.obj
 0001:000152b0       ?DloadObtainSection@@YAPEAXPEAK0@Z 00000001800162b0 f i delayimp:delayhlp.obj
 0001:0001534c       ?DloadProtectSection@@YAXKPEAK@Z 000000018001634c f i delayimp:delayhlp.obj
 0001:000153dc       ?DloadReleaseSectionWriteAccess@@YAXXZ 00000001800163dc f i delayimp:delayhlp.obj
 0001:00015470       __delayLoadHelper2         0000000180016470 f   delayimp:delayhlp.obj
 0001:00015746       ConvertSidToStringSidW     0000000180016746 f   advapi32:ADVAPI32.dll
 0001:0001574c       GetFileVersionInfoSizeW    000000018001674c f   version:VERSION.dll
 0001:00015752       GetFileVersionInfoW        0000000180016752 f   version:VERSION.dll
 0001:00015758       VerQueryValueW             0000000180016758 f   version:VERSION.dll
 0001:00015760       __GSHandlerCheck           0000000180016760 f   MSVCRT:gshandler.obj
 0001:00015780       __GSHandlerCheckCommon     0000000180016780 f   MSVCRT:gshandler.obj
 0001:000157f0       __security_check_cookie    00000001800167f0 f   MSVCRT:amdsecgs.obj
 0001:00015810       __raise_securityfailure    0000000180016810 f   MSVCRT:gs_report.obj
 0001:00015844       __report_gsfailure         0000000180016844 f   MSVCRT:gs_report.obj
 0001:00015918       __report_rangecheckfailure 0000000180016918 f   MSVCRT:gs_report.obj
 0001:0001592c       __report_securityfailure   000000018001692c f   MSVCRT:gs_report.obj
 0001:00015ac0       __chkstk                   0000000180016ac0 f   MSVCRT:chkstk.obj
 0001:00015ac0       _alloca_probe              0000000180016ac0 f   MSVCRT:chkstk.obj
 0001:00015b10       __GSHandlerCheck_SEH       0000000180016b10 f   MSVCRT:gshandlerseh.obj
 0001:00015eb8       _DllMainCRTStartup         0000000180016eb8 f   MSVCRT:dll_dllmain.obj
 0001:00015ef8       __security_init_cookie     0000000180016ef8 f   MSVCRT:gs_support.obj
 0001:00015fa4       DllMain                    0000000180016fa4 f   MSVCRT:dll_dllmain_stub.obj
 0001:00015fc8       ?__scrt_initialize_type_info@@YAXXZ 0000000180016fc8 f   MSVCRT:tncleanup.obj
 0001:00015fd8       ?__scrt_uninitialize_type_info@@YAXXZ 0000000180016fd8 f   MSVCRT:tncleanup.obj
 0001:00015fe4       __scrt_initialize_default_local_stdio_options 0000000180016fe4 f   MSVCRT:default_local_stdio_options.obj
 0001:00016000       __scrt_acquire_startup_lock 0000000180017000 f   MSVCRT:utility.obj
 0001:0001603c       __scrt_dllmain_after_initialize_c 000000018001703c f   MSVCRT:utility.obj
 0001:00016070       __scrt_dllmain_before_initialize_c 0000000180017070 f   MSVCRT:utility.obj
 0001:00016088       __scrt_dllmain_crt_thread_attach 0000000180017088 f   MSVCRT:utility.obj
 0001:000160b0       __scrt_dllmain_crt_thread_detach 00000001800170b0 f   MSVCRT:utility.obj
 0001:000160c8       __scrt_dllmain_exception_filter 00000001800170c8 f   MSVCRT:utility.obj
 0001:00016128       __scrt_dllmain_uninitialize_c 0000000180017128 f   MSVCRT:utility.obj
 0001:00016158       __scrt_dllmain_uninitialize_critical 0000000180017158 f   MSVCRT:utility.obj
 0001:0001616c       __scrt_initialize_crt      000000018001716c f   MSVCRT:utility.obj
 0001:000161b8       __scrt_initialize_onexit_tables 00000001800171b8 f   MSVCRT:utility.obj
 0001:00016244       __scrt_is_nonwritable_in_current_image 0000000180017244 f   MSVCRT:utility.obj
 0001:000162dc       __scrt_release_startup_lock 00000001800172dc f   MSVCRT:utility.obj
 0001:00016300       __scrt_uninitialize_crt    0000000180017300 f   MSVCRT:utility.obj
 0001:0001632c       __scrt_get_dyn_tls_init_callback 000000018001732c f   MSVCRT:dyn_tls_init.obj
 0001:00016334       __crt_debugger_hook        0000000180017334 f   MSVCRT:utility_desktop.obj
 0001:0001633c       __scrt_fastfail            000000018001733c f   MSVCRT:utility_desktop.obj
 0001:00016488       _RTC_Initialize            0000000180017488 f   MSVCRT:initsect.obj
 0001:000164c4       _RTC_Terminate             00000001800174c4 f   MSVCRT:initsect.obj
 0001:00016500       __isa_available_init       0000000180017500 f   MSVCRT:cpu_disp.obj
 0001:000166ac       _get_startup_argv_mode     00000001800176ac f   MSVCRT:argv_mode.obj
 0001:000166b4       __scrt_is_ucrt_dll_in_use  00000001800176b4 f   MSVCRT:ucrt_detection.obj
 0001:000166c0       CreateToolhelp32Snapshot   00000001800176c0 f   kernel32:KERNEL32.dll
 0001:000166c6       Process32First             00000001800176c6 f   kernel32:KERNEL32.dll
 0001:000166cc       Process32Next              00000001800176cc f   kernel32:KERNEL32.dll
 0001:000166d2       memset                     00000001800176d2 f   vcruntime:VCRUNTIME140.dll
 0001:000166d8       memcmp                     00000001800176d8 f   vcruntime:VCRUNTIME140.dll
 0001:000166de       wcsrchr                    00000001800176de f   vcruntime:VCRUNTIME140.dll
 0001:000166e4       strchr                     00000001800176e4 f   vcruntime:VCRUNTIME140.dll
 0001:000166ea       wcschr                     00000001800176ea f   vcruntime:VCRUNTIME140.dll
 0001:000166f0       memcpy                     00000001800176f0 f   vcruntime:VCRUNTIME140.dll
 0001:000166f6       strrchr                    00000001800176f6 f   vcruntime:VCRUNTIME140.dll
 0001:000166fc       __C_specific_handler       00000001800176fc f   vcruntime:VCRUNTIME140.dll
 0001:00016702       __std_type_info_destroy_list 0000000180017702 f   vcruntime:VCRUNTIME140.dll
 0001:00016708       strcpy                     0000000180017708 f   ucrt:api-ms-win-crt-string-l1-1-0.dll
 0001:0001670e       strlen                     000000018001770e f   ucrt:api-ms-win-crt-string-l1-1-0.dll
 0001:00016714       strcmp                     0000000180017714 f   ucrt:api-ms-win-crt-string-l1-1-0.dll
 0001:0001671a       strcat                     000000018001771a f   ucrt:api-ms-win-crt-string-l1-1-0.dll
 0001:00016720       _initterm                  0000000180017720 f   ucrt:api-ms-win-crt-runtime-l1-1-0.dll
 0001:00016726       _initterm_e                0000000180017726 f   ucrt:api-ms-win-crt-runtime-l1-1-0.dll
 0001:0001672c       _seh_filter_dll            000000018001772c f   ucrt:api-ms-win-crt-runtime-l1-1-0.dll
 0001:00016732       _configure_narrow_argv     0000000180017732 f   ucrt:api-ms-win-crt-runtime-l1-1-0.dll
 0001:00016738       _initialize_narrow_environment 0000000180017738 f   ucrt:api-ms-win-crt-runtime-l1-1-0.dll
 0001:0001673e       _initialize_onexit_table   000000018001773e f   ucrt:api-ms-win-crt-runtime-l1-1-0.dll
 0001:00016744       _execute_onexit_table      0000000180017744 f   ucrt:api-ms-win-crt-runtime-l1-1-0.dll
 0001:0001674a       _cexit                     000000018001774a f   ucrt:api-ms-win-crt-runtime-l1-1-0.dll
 0001:00016750       __scrt_stub_for_is_c_termination_complete 0000000180017750 f   MSVCRT:ucrt_stubs.obj
 0001:00016750       _is_c_termination_complete 0000000180017750 f   MSVCRT:ucrt_stubs.obj
 0001:00016770       _guard_dispatch_icall_nop  0000000180017770 f   MSVCRT:guard_dispatch.obj
 0001:00016790       _guard_xfg_dispatch_icall_nop 0000000180017790 f   MSVCRT:guard_xfg_dispatch.obj
 0002:00000000       __imp_CryptAcquireContextA 0000000180018000     advapi32:ADVAPI32.dll
 0002:00000008       __imp_RegQueryValueExW     0000000180018008     advapi32:ADVAPI32.dll
 0002:00000010       __imp_RegQueryValueExA     0000000180018010     advapi32:ADVAPI32.dll
 0002:00000018       __imp_RegQueryInfoKeyA     0000000180018018     advapi32:ADVAPI32.dll
 0002:00000020       __imp_RegOpenKeyExW        0000000180018020     advapi32:ADVAPI32.dll
 0002:00000028       __imp_RegOpenKeyExA        0000000180018028     advapi32:ADVAPI32.dll
 0002:00000030       __imp_RegEnumKeyExA        0000000180018030     advapi32:ADVAPI32.dll
 0002:00000038       __imp_RegCloseKey          0000000180018038     advapi32:ADVAPI32.dll
 0002:00000040       __imp_ConvertSidToStringSidW 0000000180018040     advapi32:ADVAPI32.dll
 0002:00000048       __imp_LookupAccountSidW    0000000180018048     advapi32:ADVAPI32.dll
 0002:00000050       __imp_GetTokenInformation  0000000180018050     advapi32:ADVAPI32.dll
 0002:00000058       __imp_OpenProcessToken     0000000180018058     advapi32:ADVAPI32.dll
 0002:00000060       __imp_CryptReleaseContext  0000000180018060     advapi32:ADVAPI32.dll
 0002:00000068       __imp_CryptGenRandom       0000000180018068     advapi32:ADVAPI32.dll
 0002:00000070       __imp_GetUserNameW         0000000180018070     advapi32:ADVAPI32.dll
 0002:00000078       \177ADVAPI32_NULL_THUNK_DATA 0000000180018078     advapi32:ADVAPI32.dll
 0002:00000080       __imp_GetStdHandle         0000000180018080     kernel32:KERNEL32.dll
 0002:00000088       __imp_GetFileType          0000000180018088     kernel32:KERNEL32.dll
 0002:00000090       __imp_GetConsoleCP         0000000180018090     kernel32:KERNEL32.dll
 0002:00000098       __imp_GetConsoleMode       0000000180018098     kernel32:KERNEL32.dll
 0002:000000a0       __imp_SetConsoleMode       00000001800180a0     kernel32:KERNEL32.dll
 0002:000000a8       __imp_CloseHandle          00000001800180a8     kernel32:KERNEL32.dll
 0002:000000b0       __imp_GetModuleHandleA     00000001800180b0     kernel32:KERNEL32.dll
 0002:000000b8       __imp_IsDebuggerPresent    00000001800180b8     kernel32:KERNEL32.dll
 0002:000000c0       __imp_InitializeSListHead  00000001800180c0     kernel32:KERNEL32.dll
 0002:000000c8       __imp_DisableThreadLibraryCalls 00000001800180c8     kernel32:KERNEL32.dll
 0002:000000d0       __imp_GetSystemTimeAsFileTime 00000001800180d0     kernel32:KERNEL32.dll
 0002:000000d8       __imp_GetCurrentThreadId   00000001800180d8     kernel32:KERNEL32.dll
 0002:000000e0       __imp_QueryPerformanceCounter 00000001800180e0     kernel32:KERNEL32.dll
 0002:000000e8       __imp_GetCurrentProcess    00000001800180e8     kernel32:KERNEL32.dll
 0002:000000f0       __imp_SetUnhandledExceptionFilter 00000001800180f0     kernel32:KERNEL32.dll
 0002:000000f8       __imp_UnhandledExceptionFilter 00000001800180f8     kernel32:KERNEL32.dll
 0002:00000100       __imp_RtlVirtualUnwind     0000000180018100     kernel32:KERNEL32.dll
 0002:00000108       __imp_RtlLookupFunctionEntry 0000000180018108     kernel32:KERNEL32.dll
 0002:00000110       __imp_RtlCaptureContext    0000000180018110     kernel32:KERNEL32.dll
 0002:00000118       __imp_LoadLibraryExA       0000000180018118     kernel32:KERNEL32.dll
 0002:00000120       __imp_GetModuleHandleW     0000000180018120     kernel32:KERNEL32.dll
 0002:00000128       __imp_FreeLibrary          0000000180018128     kernel32:KERNEL32.dll
 0002:00000130       __imp_VirtualQuery         0000000180018130     kernel32:KERNEL32.dll
 0002:00000138       __imp_VirtualProtect       0000000180018138     kernel32:KERNEL32.dll
 0002:00000140       __imp_RaiseException       0000000180018140     kernel32:KERNEL32.dll
 0002:00000148       __imp_FormatMessageA       0000000180018148     kernel32:KERNEL32.dll
 0002:00000150       __imp_LoadLibraryA         0000000180018150     kernel32:KERNEL32.dll
 0002:00000158       __imp_GetSystemDirectoryA  0000000180018158     kernel32:KERNEL32.dll
 0002:00000160       __imp_GetACP               0000000180018160     kernel32:KERNEL32.dll
 0002:00000168       __imp_IsValidCodePage      0000000180018168     kernel32:KERNEL32.dll
 0002:00000170       __imp_GetNativeSystemInfo  0000000180018170     kernel32:KERNEL32.dll
 0002:00000178       __imp_GetVersionExA        0000000180018178     kernel32:KERNEL32.dll
 0002:00000180       __imp_GetWindowsDirectoryA 0000000180018180     kernel32:KERNEL32.dll
 0002:00000188       __imp_GetSystemDirectoryW  0000000180018188     kernel32:KERNEL32.dll
 0002:00000190       __imp_GetSystemInfo        0000000180018190     kernel32:KERNEL32.dll
 0002:00000198       __imp_IsProcessorFeaturePresent 0000000180018198     kernel32:KERNEL32.dll
 0002:000001a0       __imp_GetTempPathW         00000001800181a0     kernel32:KERNEL32.dll
 0002:000001a8       __imp_GetCurrentDirectoryW 00000001800181a8     kernel32:KERNEL32.dll
 0002:000001b0       __imp_PeekConsoleInputA    00000001800181b0     kernel32:KERNEL32.dll
 0002:000001b8       __imp_GetNumberOfConsoleInputEvents 00000001800181b8     kernel32:KERNEL32.dll
 0002:000001c0       __imp_PeekNamedPipe        00000001800181c0     kernel32:KERNEL32.dll
 0002:000001c8       __imp_WriteFile            00000001800181c8     kernel32:KERNEL32.dll
 0002:000001d0       __imp_SetFilePointerEx     00000001800181d0     kernel32:KERNEL32.dll
 0002:000001d8       __imp_SetFilePointer       00000001800181d8     kernel32:KERNEL32.dll
 0002:000001e0       __imp_SetEndOfFile         00000001800181e0     kernel32:KERNEL32.dll
 0002:000001e8       __imp_ReadFile             00000001800181e8     kernel32:KERNEL32.dll
 0002:000001f0       __imp_GetFileSizeEx        00000001800181f0     kernel32:KERNEL32.dll
 0002:000001f8       __imp_GetDriveTypeW        00000001800181f8     kernel32:KERNEL32.dll
 0002:00000200       __imp_FlushFileBuffers     0000000180018200     kernel32:KERNEL32.dll
 0002:00000208       __imp_IsDBCSLeadByte       0000000180018208     kernel32:KERNEL32.dll
 0002:00000210       __imp_FindFirstFileA       0000000180018210     kernel32:KERNEL32.dll
 0002:00000218       __imp_GetModuleHandleExW   0000000180018218     kernel32:KERNEL32.dll
 0002:00000220       __imp_SetLastError         0000000180018220     kernel32:KERNEL32.dll
 0002:00000228       __imp_SetFileTime          0000000180018228     kernel32:KERNEL32.dll
 0002:00000230       __imp_SetFileAttributesW   0000000180018230     kernel32:KERNEL32.dll
 0002:00000238       __imp_RemoveDirectoryW     0000000180018238     kernel32:KERNEL32.dll
 0002:00000240       __imp_GetVolumePathNameW   0000000180018240     kernel32:KERNEL32.dll
 0002:00000248       __imp_GetVolumeInformationW 0000000180018248     kernel32:KERNEL32.dll
 0002:00000250       __imp_GetLogicalDrives     0000000180018250     kernel32:KERNEL32.dll
 0002:00000258       __imp_GetFullPathNameW     0000000180018258     kernel32:KERNEL32.dll
 0002:00000260       __imp_GetFileTime          0000000180018260     kernel32:KERNEL32.dll
 0002:00000268       __imp_GetFileInformationByHandle 0000000180018268     kernel32:KERNEL32.dll
 0002:00000270       __imp_GetFileAttributesExW 0000000180018270     kernel32:KERNEL32.dll
 0002:00000278       __imp_GetFileAttributesW   0000000180018278     kernel32:KERNEL32.dll
 0002:00000280       __imp_GetDiskFreeSpaceExW  0000000180018280     kernel32:KERNEL32.dll
 0002:00000288       __imp_FindNextFileW        0000000180018288     kernel32:KERNEL32.dll
 0002:00000290       __imp_FindFirstFileW       0000000180018290     kernel32:KERNEL32.dll
 0002:00000298       __imp_FindClose            0000000180018298     kernel32:KERNEL32.dll
 0002:000002a0       __imp_DeleteFileW          00000001800182a0     kernel32:KERNEL32.dll
 0002:000002a8       __imp_CreateDirectoryW     00000001800182a8     kernel32:KERNEL32.dll
 0002:000002b0       __imp_SetErrorMode         00000001800182b0     kernel32:KERNEL32.dll
 0002:000002b8       __imp_GetUserGeoID         00000001800182b8     kernel32:KERNEL32.dll
 0002:000002c0       __imp_GetGeoInfoA          00000001800182c0     kernel32:KERNEL32.dll
 0002:000002c8       __imp_GetLocaleInfoA       00000001800182c8     kernel32:KERNEL32.dll
 0002:000002d0       __imp_MultiByteToWideChar  00000001800182d0     kernel32:KERNEL32.dll
 0002:000002d8       __imp_GetDynamicTimeZoneInformation 00000001800182d8     kernel32:KERNEL32.dll
 0002:000002e0       __imp_GetTimeZoneInformation 00000001800182e0     kernel32:KERNEL32.dll
 0002:000002e8       __imp_GetConsoleWindow     00000001800182e8     kernel32:KERNEL32.dll
 0002:000002f0       __imp_WideCharToMultiByte  00000001800182f0     kernel32:KERNEL32.dll
 0002:000002f8       __imp_FormatMessageW       00000001800182f8     kernel32:KERNEL32.dll
 0002:00000300       __imp_GetProcessId         0000000180018300     kernel32:KERNEL32.dll
 0002:00000308       __imp_CreateProcessW       0000000180018308     kernel32:KERNEL32.dll
 0002:00000310       __imp_CreatePipe           0000000180018310     kernel32:KERNEL32.dll
 0002:00000318       __imp_SetHandleInformation 0000000180018318     kernel32:KERNEL32.dll
 0002:00000320       __imp_GetHandleInformation 0000000180018320     kernel32:KERNEL32.dll
 0002:00000328       __imp_CreateFileW          0000000180018328     kernel32:KERNEL32.dll
 0002:00000330       __imp_Process32Next        0000000180018330     kernel32:KERNEL32.dll
 0002:00000338       __imp_Process32First       0000000180018338     kernel32:KERNEL32.dll
 0002:00000340       __imp_CreateToolhelp32Snapshot 0000000180018340     kernel32:KERNEL32.dll
 0002:00000348       __imp_QueryFullProcessImageNameW 0000000180018348     kernel32:KERNEL32.dll
 0002:00000350       __imp_LocalFree            0000000180018350     kernel32:KERNEL32.dll
 0002:00000358       __imp_OpenProcess          0000000180018358     kernel32:KERNEL32.dll
 0002:00000360       __imp_GetExitCodeProcess   0000000180018360     kernel32:KERNEL32.dll
 0002:00000368       __imp_TerminateProcess     0000000180018368     kernel32:KERNEL32.dll
 0002:00000370       __imp_GetCurrentProcessId  0000000180018370     kernel32:KERNEL32.dll
 0002:00000378       __imp_GetProcessTimes      0000000180018378     kernel32:KERNEL32.dll
 0002:00000380       __imp_WaitForMultipleObjects 0000000180018380     kernel32:KERNEL32.dll
 0002:00000388       __imp_GetProcAddress       0000000180018388     kernel32:KERNEL32.dll
 0002:00000390       __imp_FreeEnvironmentStringsW 0000000180018390     kernel32:KERNEL32.dll
 0002:00000398       __imp_FreeEnvironmentStringsA 0000000180018398     kernel32:KERNEL32.dll
 0002:000003a0       __imp_GetEnvironmentStringsW 00000001800183a0     kernel32:KERNEL32.dll
 0002:000003a8       __imp_GetEnvironmentStrings 00000001800183a8     kernel32:KERNEL32.dll
 0002:000003b0       __imp_GetUserDefaultLCID   00000001800183b0     kernel32:KERNEL32.dll
 0002:000003b8       __imp_GetUserDefaultUILanguage 00000001800183b8     kernel32:KERNEL32.dll
 0002:000003c0       __imp_GetLastError         00000001800183c0     kernel32:KERNEL32.dll
 0002:000003c8       \177KERNEL32_NULL_THUNK_DATA 00000001800183c8     kernel32:KERNEL32.dll
 0002:000003d0       __imp_memset               00000001800183d0     vcruntime:VCRUNTIME140.dll
 0002:000003d8       __imp_memcmp               00000001800183d8     vcruntime:VCRUNTIME140.dll
 0002:000003e0       __imp_wcsrchr              00000001800183e0     vcruntime:VCRUNTIME140.dll
 0002:000003e8       __imp_strchr               00000001800183e8     vcruntime:VCRUNTIME140.dll
 0002:000003f0       __imp_wcschr               00000001800183f0     vcruntime:VCRUNTIME140.dll
 0002:000003f8       __imp_memcpy               00000001800183f8     vcruntime:VCRUNTIME140.dll
 0002:00000400       __imp___std_type_info_destroy_list 0000000180018400     vcruntime:VCRUNTIME140.dll
 0002:00000408       __imp___C_specific_handler 0000000180018408     vcruntime:VCRUNTIME140.dll
 0002:00000410       __imp_strrchr              0000000180018410     vcruntime:VCRUNTIME140.dll
 0002:00000418       \177VCRUNTIME140_NULL_THUNK_DATA 0000000180018418     vcruntime:VCRUNTIME140.dll
 0002:00000420       __imp_VerQueryValueW       0000000180018420     version:VERSION.dll
 0002:00000428       __imp_GetFileVersionInfoW  0000000180018428     version:VERSION.dll
 0002:00000430       __imp_GetFileVersionInfoSizeW 0000000180018430     version:VERSION.dll
 0002:00000438       \177VERSION_NULL_THUNK_DATA 0000000180018438     version:VERSION.dll
 0002:00000440       __imp_wcstombs             0000000180018440     ucrt:api-ms-win-crt-convert-l1-1-0.dll
 0002:00000448       __imp_mbstowcs_s           0000000180018448     ucrt:api-ms-win-crt-convert-l1-1-0.dll
 0002:00000450       __imp_wcstombs_s           0000000180018450     ucrt:api-ms-win-crt-convert-l1-1-0.dll
 0002:00000458       __imp__itoa_s              0000000180018458     ucrt:api-ms-win-crt-convert-l1-1-0.dll
 0002:00000460       __imp_atoi                 0000000180018460     ucrt:api-ms-win-crt-convert-l1-1-0.dll
 0002:00000468       \177api-ms-win-crt-convert-l1-1-0_NULL_THUNK_DATA 0000000180018468     ucrt:api-ms-win-crt-convert-l1-1-0.dll
 0002:00000470       __imp__wgetcwd             0000000180018470     ucrt:api-ms-win-crt-environment-l1-1-0.dll
 0002:00000478       __imp__wgetdcwd            0000000180018478     ucrt:api-ms-win-crt-environment-l1-1-0.dll
 0002:00000480       __imp__wgetenv             0000000180018480     ucrt:api-ms-win-crt-environment-l1-1-0.dll
 0002:00000488       \177api-ms-win-crt-environment-l1-1-0_NULL_THUNK_DATA 0000000180018488     ucrt:api-ms-win-crt-environment-l1-1-0.dll
 0002:00000490       __imp__wfullpath           0000000180018490     ucrt:api-ms-win-crt-filesystem-l1-1-0.dll
 0002:00000498       __imp__fullpath            0000000180018498     ucrt:api-ms-win-crt-filesystem-l1-1-0.dll
 0002:000004a0       __imp__wrename             00000001800184a0     ucrt:api-ms-win-crt-filesystem-l1-1-0.dll
 0002:000004a8       \177api-ms-win-crt-filesystem-l1-1-0_NULL_THUNK_DATA 00000001800184a8     ucrt:api-ms-win-crt-filesystem-l1-1-0.dll
 0002:000004b0       __imp_free                 00000001800184b0     ucrt:api-ms-win-crt-heap-l1-1-0.dll
 0002:000004b8       __imp_malloc               00000001800184b8     ucrt:api-ms-win-crt-heap-l1-1-0.dll
 0002:000004c0       __imp_realloc              00000001800184c0     ucrt:api-ms-win-crt-heap-l1-1-0.dll
 0002:000004c8       __imp_calloc               00000001800184c8     ucrt:api-ms-win-crt-heap-l1-1-0.dll
 0002:000004d0       \177api-ms-win-crt-heap-l1-1-0_NULL_THUNK_DATA 00000001800184d0     ucrt:api-ms-win-crt-heap-l1-1-0.dll
 0002:000004d8       __imp__isnan               00000001800184d8     ucrt:api-ms-win-crt-math-l1-1-0.dll
 0002:000004e0       \177api-ms-win-crt-math-l1-1-0_NULL_THUNK_DATA 00000001800184e0     ucrt:api-ms-win-crt-math-l1-1-0.dll
 0002:000004e8       __imp__initialize_narrow_environment 00000001800184e8     ucrt:api-ms-win-crt-runtime-l1-1-0.dll
 0002:000004f0       __imp__configure_narrow_argv 00000001800184f0     ucrt:api-ms-win-crt-runtime-l1-1-0.dll
 0002:000004f8       __imp__seh_filter_dll      00000001800184f8     ucrt:api-ms-win-crt-runtime-l1-1-0.dll
 0002:00000500       __imp__initialize_onexit_table 0000000180018500     ucrt:api-ms-win-crt-runtime-l1-1-0.dll
 0002:00000508       __imp__initterm            0000000180018508     ucrt:api-ms-win-crt-runtime-l1-1-0.dll
 0002:00000510       __imp_strerror_s           0000000180018510     ucrt:api-ms-win-crt-runtime-l1-1-0.dll
 0002:00000518       __imp__initterm_e          0000000180018518     ucrt:api-ms-win-crt-runtime-l1-1-0.dll
 0002:00000520       __imp__errno               0000000180018520     ucrt:api-ms-win-crt-runtime-l1-1-0.dll
 0002:00000528       __imp__cexit               0000000180018528     ucrt:api-ms-win-crt-runtime-l1-1-0.dll
 0002:00000530       __imp__execute_onexit_table 0000000180018530     ucrt:api-ms-win-crt-runtime-l1-1-0.dll
 0002:00000538       \177api-ms-win-crt-runtime-l1-1-0_NULL_THUNK_DATA 0000000180018538     ucrt:api-ms-win-crt-runtime-l1-1-0.dll
 0002:00000540       __imp___stdio_common_vsprintf 0000000180018540     ucrt:api-ms-win-crt-stdio-l1-1-0.dll
 0002:00000548       __imp___stdio_common_vfprintf 0000000180018548     ucrt:api-ms-win-crt-stdio-l1-1-0.dll
 0002:00000550       __imp___stdio_common_vswprintf 0000000180018550     ucrt:api-ms-win-crt-stdio-l1-1-0.dll
 0002:00000558       __imp___acrt_iob_func      0000000180018558     ucrt:api-ms-win-crt-stdio-l1-1-0.dll
 0002:00000560       __imp_fclose               0000000180018560     ucrt:api-ms-win-crt-stdio-l1-1-0.dll
 0002:00000568       __imp___stdio_common_vsscanf 0000000180018568     ucrt:api-ms-win-crt-stdio-l1-1-0.dll
 0002:00000570       __imp_fgets                0000000180018570     ucrt:api-ms-win-crt-stdio-l1-1-0.dll
 0002:00000578       __imp_fopen                0000000180018578     ucrt:api-ms-win-crt-stdio-l1-1-0.dll
 0002:00000580       \177api-ms-win-crt-stdio-l1-1-0_NULL_THUNK_DATA 0000000180018580     ucrt:api-ms-win-crt-stdio-l1-1-0.dll
 0002:00000588       __imp_iswctype             0000000180018588     ucrt:api-ms-win-crt-string-l1-1-0.dll
 0002:00000590       __imp__strdup              0000000180018590     ucrt:api-ms-win-crt-string-l1-1-0.dll
 0002:00000598       __imp_strcat               0000000180018598     ucrt:api-ms-win-crt-string-l1-1-0.dll
 0002:000005a0       __imp_strcmp               00000001800185a0     ucrt:api-ms-win-crt-string-l1-1-0.dll
 0002:000005a8       __imp_wcsncmp              00000001800185a8     ucrt:api-ms-win-crt-string-l1-1-0.dll
 0002:000005b0       __imp__wcsupr              00000001800185b0     ucrt:api-ms-win-crt-string-l1-1-0.dll
 0002:000005b8       __imp_wcscat               00000001800185b8     ucrt:api-ms-win-crt-string-l1-1-0.dll
 0002:000005c0       __imp_wcsncat              00000001800185c0     ucrt:api-ms-win-crt-string-l1-1-0.dll
 0002:000005c8       __imp_strncpy              00000001800185c8     ucrt:api-ms-win-crt-string-l1-1-0.dll
 0002:000005d0       __imp_wcslen               00000001800185d0     ucrt:api-ms-win-crt-string-l1-1-0.dll
 0002:000005d8       __imp_wcscpy               00000001800185d8     ucrt:api-ms-win-crt-string-l1-1-0.dll
 0002:000005e0       __imp_wcscmp               00000001800185e0     ucrt:api-ms-win-crt-string-l1-1-0.dll
 0002:000005e8       __imp__wcsdup              00000001800185e8     ucrt:api-ms-win-crt-string-l1-1-0.dll
 0002:000005f0       __imp_wcscat_s             00000001800185f0     ucrt:api-ms-win-crt-string-l1-1-0.dll
 0002:000005f8       __imp_toupper              00000001800185f8     ucrt:api-ms-win-crt-string-l1-1-0.dll
 0002:00000600       __imp_strlen               0000000180018600     ucrt:api-ms-win-crt-string-l1-1-0.dll
 0002:00000608       __imp_strcpy               0000000180018608     ucrt:api-ms-win-crt-string-l1-1-0.dll
 0002:00000610       __imp_isalpha              0000000180018610     ucrt:api-ms-win-crt-string-l1-1-0.dll
 0002:00000618       __imp_towupper             0000000180018618     ucrt:api-ms-win-crt-string-l1-1-0.dll
 0002:00000620       \177api-ms-win-crt-string-l1-1-0_NULL_THUNK_DATA 0000000180018620     ucrt:api-ms-win-crt-string-l1-1-0.dll
 0002:00000628       __imp_JVM_HasReferencePendingList 0000000180018628     jvm:jvm.dll
 0002:00000630       __imp_JVM_GetAndClearReferencePendingList 0000000180018630     jvm:jvm.dll
 0002:00000638       __imp_JVM_GetThreadInterruptEvent 0000000180018638     jvm:jvm.dll
 0002:00000640       __imp_JVM_Clone            0000000180018640     jvm:jvm.dll
 0002:00000648       __imp_JVM_MonitorNotifyAll 0000000180018648     jvm:jvm.dll
 0002:00000650       __imp_JVM_MonitorNotify    0000000180018650     jvm:jvm.dll
 0002:00000658       __imp_JVM_MonitorWait      0000000180018658     jvm:jvm.dll
 0002:00000660       __imp_JVM_IHashCode        0000000180018660     jvm:jvm.dll
 0002:00000668       __imp_JVM_NewInstanceFromConstructor 0000000180018668     jvm:jvm.dll
 0002:00000670       __imp_JVM_InvokeMethod     0000000180018670     jvm:jvm.dll
 0002:00000678       __imp_JVM_AddReadsModule   0000000180018678     jvm:jvm.dll
 0002:00000680       __imp_JVM_AddModuleExportsToAll 0000000180018680     jvm:jvm.dll
 0002:00000688       __imp_JVM_AddModuleExportsToAllUnnamed 0000000180018688     jvm:jvm.dll
 0002:00000690       __imp_JVM_AddModuleExports 0000000180018690     jvm:jvm.dll
 0002:00000698       __imp_JVM_DefineModule     0000000180018698     jvm:jvm.dll
 0002:000006a0       __imp_JVM_GetFieldTypeAnnotations 00000001800186a0     jvm:jvm.dll
 0002:000006a8       __imp_JVM_GetMethodParameters 00000001800186a8     jvm:jvm.dll
 0002:000006b0       __imp_JVM_GetMethodTypeAnnotations 00000001800186b0     jvm:jvm.dll
 0002:000006b8       __imp_JVM_ConstantPoolGetTagAt 00000001800186b8     jvm:jvm.dll
 0002:000006c0       __imp_JVM_ConstantPoolGetUTF8At 00000001800186c0     jvm:jvm.dll
 0002:000006c8       __imp_JVM_ConstantPoolGetStringAt 00000001800186c8     jvm:jvm.dll
 0002:000006d0       __imp_JVM_ConstantPoolGetDoubleAt 00000001800186d0     jvm:jvm.dll
 0002:000006d8       __imp_JVM_ConstantPoolGetFloatAt 00000001800186d8     jvm:jvm.dll
 0002:000006e0       __imp_JVM_ConstantPoolGetLongAt 00000001800186e0     jvm:jvm.dll
 0002:000006e8       __imp_JVM_ConstantPoolGetIntAt 00000001800186e8     jvm:jvm.dll
 0002:000006f0       __imp_JVM_ConstantPoolGetNameAndTypeRefInfoAt 00000001800186f0     jvm:jvm.dll
 0002:000006f8       __imp_JVM_ConstantPoolGetNameAndTypeRefIndexAt 00000001800186f8     jvm:jvm.dll
 0002:00000700       __imp_JVM_ConstantPoolGetMemberRefInfoAt 0000000180018700     jvm:jvm.dll
 0002:00000708       __imp_JVM_ConstantPoolGetFieldAtIfLoaded 0000000180018708     jvm:jvm.dll
 0002:00000710       __imp_JVM_ConstantPoolGetFieldAt 0000000180018710     jvm:jvm.dll
 0002:00000718       __imp_JVM_ConstantPoolGetMethodAtIfLoaded 0000000180018718     jvm:jvm.dll
 0002:00000720       __imp_JVM_ConstantPoolGetMethodAt 0000000180018720     jvm:jvm.dll
 0002:00000728       __imp_JVM_ConstantPoolGetClassRefIndexAt 0000000180018728     jvm:jvm.dll
 0002:00000730       __imp_JVM_ConstantPoolGetClassAtIfLoaded 0000000180018730     jvm:jvm.dll
 0002:00000738       __imp_JVM_ConstantPoolGetClassAt 0000000180018738     jvm:jvm.dll
 0002:00000740       __imp_JVM_ConstantPoolGetSize 0000000180018740     jvm:jvm.dll
 0002:00000748       __imp_JVM_DefineClassWithSource 0000000180018748     jvm:jvm.dll
 0002:00000750       __imp_JVM_FindLoadedClass  0000000180018750     jvm:jvm.dll
 0002:00000758       __imp_JVM_WaitForReferencePendingList 0000000180018758     jvm:jvm.dll
 0002:00000760       __imp_JVM_IsSupportedJNIVersion 0000000180018760     jvm:jvm.dll
 0002:00000768       __imp_JVM_FindLibraryEntry 0000000180018768     jvm:jvm.dll
 0002:00000770       __imp_JVM_DoPrivileged     0000000180018770     jvm:jvm.dll
 0002:00000778       __imp_JVM_LoadLibrary      0000000180018778     jvm:jvm.dll
 0002:00000780       __imp_JVM_AssertionStatusDirectives 0000000180018780     jvm:jvm.dll
 0002:00000788       __imp_JVM_FindClassFromCaller 0000000180018788     jvm:jvm.dll
 0002:00000790       __imp_JVM_FindPrimitiveClass 0000000180018790     jvm:jvm.dll
 0002:00000798       __imp_JVM_GetEnclosingMethodInfo 0000000180018798     jvm:jvm.dll
 0002:000007a0       __imp_JVM_DesiredAssertionStatus 00000001800187a0     jvm:jvm.dll
 0002:000007a8       __imp_JVM_GetClassConstantPool 00000001800187a8     jvm:jvm.dll
 0002:000007b0       __imp_JVM_GetNestMembers   00000001800187b0     jvm:jvm.dll
 0002:000007b8       __imp_JVM_GetNestHost      00000001800187b8     jvm:jvm.dll
 0002:000007c0       __imp_JVM_GetClassDeclaredConstructors 00000001800187c0     jvm:jvm.dll
 0002:000007c8       __imp_JVM_GetClassDeclaredFields 00000001800187c8     jvm:jvm.dll
 0002:000007d0       __imp_JVM_GetClassDeclaredMethods 00000001800187d0     jvm:jvm.dll
 0002:000007d8       __imp_JVM_GetClassTypeAnnotations 00000001800187d8     jvm:jvm.dll
 0002:000007e0       __imp_JVM_GetClassAnnotations 00000001800187e0     jvm:jvm.dll
 0002:000007e8       __imp_JVM_GetClassSignature 00000001800187e8     jvm:jvm.dll
 0002:000007f0       __imp_JVM_GetSimpleBinaryName 00000001800187f0     jvm:jvm.dll
 0002:000007f8       __imp_JVM_GetDeclaringClass 00000001800187f8     jvm:jvm.dll
 0002:00000800       __imp_JVM_GetDeclaredClasses 0000000180018800     jvm:jvm.dll
 0002:00000808       __imp_JVM_GetClassModifiers 0000000180018808     jvm:jvm.dll
 0002:00000810       __imp_JVM_IsPrimitiveClass 0000000180018810     jvm:jvm.dll
 0002:00000818       __imp_JVM_IsArrayClass     0000000180018818     jvm:jvm.dll
 0002:00000820       __imp_JVM_GetProtectionDomain 0000000180018820     jvm:jvm.dll
 0002:00000828       __imp_JVM_SetClassSigners  0000000180018828     jvm:jvm.dll
 0002:00000830       __imp_JVM_GetClassSigners  0000000180018830     jvm:jvm.dll
 0002:00000838       __imp_JVM_IsInterface      0000000180018838     jvm:jvm.dll
 0002:00000840       __imp_JVM_GetClassInterfaces 0000000180018840     jvm:jvm.dll
 0002:00000848       __imp_JVM_InitClassName    0000000180018848     jvm:jvm.dll
 0002:00000850       __imp_JVM_SetBootLoaderUnnamedModule 0000000180018850     jvm:jvm.dll
 0002:00000858       __imp_JVM_GetSystemPackages 0000000180018858     jvm:jvm.dll
 0002:00000860       __imp_JVM_GetSystemPackage 0000000180018860     jvm:jvm.dll
 0002:00000868       __imp_JVM_SupportsCX8      0000000180018868     jvm:jvm.dll
 0002:00000870       __imp_JVM_GetCallerClass   0000000180018870     jvm:jvm.dll
 0002:00000878       __imp_JVM_GetClassAccessFlags 0000000180018878     jvm:jvm.dll
 0002:00000880       __imp_JVM_AreNestMates     0000000180018880     jvm:jvm.dll
 0002:00000888       __imp_JVM_GC               0000000180018888     jvm:jvm.dll
 0002:00000890       __imp_JVM_TotalMemory      0000000180018890     jvm:jvm.dll
 0002:00000898       __imp_JVM_FreeMemory       0000000180018898     jvm:jvm.dll
 0002:000008a0       __imp_JVM_MaxMemory        00000001800188a0     jvm:jvm.dll
 0002:000008a8       __imp_JVM_ActiveProcessorCount 00000001800188a8     jvm:jvm.dll
 0002:000008b0       __imp_JVM_GetClassContext  00000001800188b0     jvm:jvm.dll
 0002:000008b8       __imp_JVM_BeforeHalt       00000001800188b8     jvm:jvm.dll
 0002:000008c0       __imp_JVM_Halt             00000001800188c0     jvm:jvm.dll
 0002:000008c8       __imp_JVM_RegisterSignal   00000001800188c8     jvm:jvm.dll
 0002:000008d0       __imp_JVM_RaiseSignal      00000001800188d0     jvm:jvm.dll
 0002:000008d8       __imp_JVM_FindSignal       00000001800188d8     jvm:jvm.dll
 0002:000008e0       __imp_JVM_CallStackWalk    00000001800188e0     jvm:jvm.dll
 0002:000008e8       __imp_JVM_MoreStackWalk    00000001800188e8     jvm:jvm.dll
 0002:000008f0       __imp_JVM_InitStackTraceElementArray 00000001800188f0     jvm:jvm.dll
 0002:000008f8       __imp_JVM_InitStackTraceElement 00000001800188f8     jvm:jvm.dll
 0002:00000900       __imp_JVM_InternString     0000000180018900     jvm:jvm.dll
 0002:00000908       __imp_JVM_CurrentTimeMillis 0000000180018908     jvm:jvm.dll
 0002:00000910       __imp_JVM_NanoTime         0000000180018910     jvm:jvm.dll
 0002:00000918       __imp_JVM_NewMultiArray    0000000180018918     jvm:jvm.dll
 0002:00000920       __imp_JVM_ArrayCopy        0000000180018920     jvm:jvm.dll
 0002:00000928       __imp_JVM_InitProperties   0000000180018928     jvm:jvm.dll
 0002:00000930       __imp_JVM_StartThread      0000000180018930     jvm:jvm.dll
 0002:00000938       __imp_JVM_StopThread       0000000180018938     jvm:jvm.dll
 0002:00000940       __imp_JVM_IsThreadAlive    0000000180018940     jvm:jvm.dll
 0002:00000948       __imp_JVM_SuspendThread    0000000180018948     jvm:jvm.dll
 0002:00000950       __imp_JVM_ResumeThread     0000000180018950     jvm:jvm.dll
 0002:00000958       __imp_JVM_NewArray         0000000180018958     jvm:jvm.dll
 0002:00000960       __imp_JVM_SetPrimitiveArrayElement 0000000180018960     jvm:jvm.dll
 0002:00000968       __imp_JVM_SetThreadPriority 0000000180018968     jvm:jvm.dll
 0002:00000970       __imp_JVM_Yield            0000000180018970     jvm:jvm.dll
 0002:00000978       __imp_JVM_Sleep            0000000180018978     jvm:jvm.dll
 0002:00000980       __imp_JVM_CurrentThread    0000000180018980     jvm:jvm.dll
 0002:00000988       __imp_JVM_CountStackFrames 0000000180018988     jvm:jvm.dll
 0002:00000990       __imp_JVM_SetArrayElement  0000000180018990     jvm:jvm.dll
 0002:00000998       __imp_JVM_GetPrimitiveArrayElement 0000000180018998     jvm:jvm.dll
 0002:000009a0       __imp_JVM_Interrupt        00000001800189a0     jvm:jvm.dll
 0002:000009a8       __imp_JVM_IsInterrupted    00000001800189a8     jvm:jvm.dll
 0002:000009b0       __imp_JVM_GetArrayElement  00000001800189b0     jvm:jvm.dll
 0002:000009b8       __imp_JVM_GetArrayLength   00000001800189b8     jvm:jvm.dll
 0002:000009c0       __imp_JVM_GetStackAccessControlContext 00000001800189c0     jvm:jvm.dll
 0002:000009c8       __imp_JVM_HoldsLock        00000001800189c8     jvm:jvm.dll
 0002:000009d0       __imp_JVM_GetAllThreads    00000001800189d0     jvm:jvm.dll
 0002:000009d8       __imp_JVM_SetNativeThreadName 00000001800189d8     jvm:jvm.dll
 0002:000009e0       __imp_JVM_DumpThreads      00000001800189e0     jvm:jvm.dll
 0002:000009e8       __imp_JVM_FillInStackTrace 00000001800189e8     jvm:jvm.dll
 0002:000009f0       __imp_JVM_GetNanoTimeAdjustment 00000001800189f0     jvm:jvm.dll
 0002:000009f8       __imp_JVM_GetVmArguments   00000001800189f8     jvm:jvm.dll
 0002:00000a00       __imp_JVM_InitializeFromArchive 0000000180018a00     jvm:jvm.dll
 0002:00000a08       __imp_JVM_LatestUserDefinedLoader 0000000180018a08     jvm:jvm.dll
 0002:00000a10       __imp_JVM_InitAgentProperties 0000000180018a10     jvm:jvm.dll
 0002:00000a18       __imp_JVM_GetTemporaryDirectory 0000000180018a18     jvm:jvm.dll
 0002:00000a20       __imp_JVM_GetInterfaceVersion 0000000180018a20     jvm:jvm.dll
 0002:00000a28       __imp_jio_vsnprintf        0000000180018a28     jvm:jvm.dll
 0002:00000a30       __imp_jio_vfprintf         0000000180018a30     jvm:jvm.dll
 0002:00000a38       __imp_JVM_GetInheritedAccessControlContext 0000000180018a38     jvm:jvm.dll
 0002:00000a40       __imp_JVM_FindClassFromBootLoader 0000000180018a40     jvm:jvm.dll
 0002:00000a48       __imp_JVM_UnloadLibrary    0000000180018a48     jvm:jvm.dll
 0002:00000a50       \177jvm_NULL_THUNK_DATA    0000000180018a50     jvm:jvm.dll
 0002:00000a58       __imp_VerifyFixClassname   0000000180018a58     verify:verify.dll
 0002:00000a60       __imp_VerifyClass          0000000180018a60     verify:verify.dll
 0002:00000a68       __imp_VerifyClassForMajorVersion 0000000180018a68     verify:verify.dll
 0002:00000a70       __imp_VerifyClassname      0000000180018a70     verify:verify.dll
 0002:00000a78       \177verify_NULL_THUNK_DATA 0000000180018a78     verify:verify.dll
 0002:00000a80       __guard_check_icall_fptr   0000000180018a80     MSVCRT:guard_support.obj
 0002:00000a88       __guard_xfg_check_icall_fptr 0000000180018a88     MSVCRT:guard_support.obj
 0002:00000a90       __guard_dispatch_icall_fptr 0000000180018a90     MSVCRT:guard_support.obj
 0002:00000a98       __guard_xfg_dispatch_icall_fptr 0000000180018a98     MSVCRT:guard_support.obj
 0002:00000aa0       __guard_xfg_table_dispatch_icall_fptr 0000000180018aa0     MSVCRT:guard_support.obj
 0002:00000aa8       __castguard_check_failure_os_handled_fptr 0000000180018aa8     MSVCRT:guard_support.obj
 0002:00000ab0       __guard_memcpy_fptr        0000000180018ab0     vcruntime:softmemtag.obj
 0002:00000ab8       __xc_a                     0000000180018ab8     MSVCRT:initializers.obj
 0002:00000ac0       __xc_z                     0000000180018ac0     MSVCRT:initializers.obj
 0002:00000ac8       __xi_a                     0000000180018ac8     MSVCRT:initializers.obj
 0002:00000ad0       __xi_z                     0000000180018ad0     MSVCRT:initializers.obj
 0002:00000ad8       __xp_a                     0000000180018ad8     MSVCRT:initializers.obj
 0002:00000ae0       __xp_z                     0000000180018ae0     MSVCRT:initializers.obj
 0002:00000ae8       __xt_a                     0000000180018ae8     MSVCRT:initializers.obj
 0002:00000af0       __xt_z                     0000000180018af0     MSVCRT:initializers.obj
 0002:00000b00       ??_C@_0O@LMKLDNGH@initClassName@ 0000000180018b00     Class.obj
 0002:00000b10       ??_C@_0BF@FOHFOJOB@?$CI?$CJLjava?1lang?1String?$DL@ 0000000180018b10     Class.obj
 0002:00000b28       ??_C@_0O@BCDKKCAE@getSuperclass@ 0000000180018b28     Class.obj
 0002:00000b38       ??_C@_0BE@IIFEGCLG@?$CI?$CJLjava?1lang?1Class?$DL@ 0000000180018b38     Class.obj
 0002:00000b50       ??_C@_0P@FLDOEJHK@getInterfaces0@ 0000000180018b50     Class.obj
 0002:00000b60       ??_C@_0BF@BNKCIMJP@?$CI?$CJ?$FLLjava?1lang?1Class?$DL@ 0000000180018b60     Class.obj
 0002:00000b78       ??_C@_0M@NAJCIFFF@isInterface@ 0000000180018b78     Class.obj
 0002:00000b84       ??_C@_03MMPFGPID@?$CI?$CJZ@ 0000000180018b84     Class.obj
 0002:00000b88       ??_C@_0L@NOPNAKKC@getSigners@ 0000000180018b88     Class.obj
 0002:00000b98       ??_C@_0BG@PFDHKCPA@?$CI?$CJ?$FLLjava?1lang?1Object?$DL@ 0000000180018b98     Class.obj
 0002:00000bb0       ??_C@_0L@MANCLNOL@setSigners@ 0000000180018bb0     Class.obj
 0002:00000bc0       ??_C@_0BH@JBNAJHIH@?$CI?$FLLjava?1lang?1Object?$DL?$CJV@ 0000000180018bc0     Class.obj
 0002:00000bd8       ??_C@_07LJDBDAGJ@isArray@  0000000180018bd8     Class.obj
 0002:00000be0       ??_C@_0M@DJOEILEB@isPrimitive@ 0000000180018be0     Class.obj
 0002:00000bf0       ??_C@_0N@MKAAFCEB@getModifiers@ 0000000180018bf0     Class.obj
 0002:00000c00       ??_C@_03KNBKCOBB@?$CI?$CJI@ 0000000180018c00     Class.obj
 0002:00000c08       ??_C@_0BD@BEKBHNDA@getDeclaredFields0@ 0000000180018c08     Class.obj
 0002:00000c20       ??_C@_0BO@KFNILMGC@?$CIZ?$CJ?$FLLjava?1lang?1reflect?1Field?$DL@ 0000000180018c20     Class.obj
 0002:00000c40       ??_C@_0BE@LOILJEHC@getDeclaredMethods0@ 0000000180018c40     Class.obj
 0002:00000c58       ??_C@_0BP@IIIKNIKA@?$CIZ?$CJ?$FLLjava?1lang?1reflect?1Method?$DL@ 0000000180018c58     Class.obj
 0002:00000c78       ??_C@_0BJ@KLPKFLFA@getDeclaredConstructors0@ 0000000180018c78     Class.obj
 0002:00000c98       ??_C@_0CE@FDMOFPI@?$CIZ?$CJ?$FLLjava?1lang?1reflect?1Construc@ 0000000180018c98     Class.obj
 0002:00000cc0       ??_C@_0BF@CGNPOFHG@getProtectionDomain0@ 0000000180018cc0     Class.obj
 0002:00000cd8       ??_C@_0CD@LEMBAENN@?$CI?$CJLjava?1security?1ProtectionDoma@ 0000000180018cd8     Class.obj
 0002:00000d00       ??_C@_0BE@CIFNAIBM@getDeclaredClasses0@ 0000000180018d00     Class.obj
 0002:00000d18       ??_C@_0BD@NHPDOJGF@getDeclaringClass0@ 0000000180018d18     Class.obj
 0002:00000d30       ??_C@_0BF@ODCBBOMF@getSimpleBinaryName0@ 0000000180018d30     Class.obj
 0002:00000d48       ??_C@_0BF@KFMFPKNK@getGenericSignature0@ 0000000180018d48     Class.obj
 0002:00000d60       ??_C@_0BC@CDJDGCDH@getRawAnnotations@ 0000000180018d60     Class.obj
 0002:00000d74       ??_C@_04LHPAGAEF@?$CI?$CJ?$FLB@ 0000000180018d74     Class.obj
 0002:00000d80       ??_C@_0BA@DLHKEBGM@getConstantPool@ 0000000180018d80     Class.obj
 0002:00000d90       ??_C@_0CG@OKGFDDJA@?$CI?$CJLjdk?1internal?1reflect?1Constan@ 0000000180018d90     Class.obj
 0002:00000db8       ??_C@_0BI@EOEBGMEG@desiredAssertionStatus0@ 0000000180018db8     Class.obj
 0002:00000dd0       ??_C@_0BF@CBMAAKJJ@?$CILjava?1lang?1Class?$DL?$CJZ@ 0000000180018dd0     Class.obj
 0002:00000de8       ??_C@_0BE@OLDEPMPN@getEnclosingMethod0@ 0000000180018de8     Class.obj
 0002:00000e00       ??_C@_0BG@CNILIFMJ@getRawTypeAnnotations@ 0000000180018e00     Class.obj
 0002:00000e18       ??_C@_0N@NMCDFPDB@getNestHost0@ 0000000180018e18     Class.obj
 0002:00000e28       ??_C@_0BA@DLOACIFG@getNestMembers0@ 0000000180018e28     Class.obj
 0002:00000e38       ??_C@_0BD@EELMJMNJ@retrieveDirectives@ 0000000180018e38     ClassLoader.obj
 0002:00000e50       ??_C@_0CI@FCANAINE@?$CI?$CJLjava?1lang?1AssertionStatusDir@ 0000000180018e50     ClassLoader.obj
 0002:00000e78       ??_C@_0CE@JCAGBDAJ@java?1lang?1ClassLoader$NativeLib@ 0000000180018e78     ClassLoader.obj
 0002:00000e9c       ??_C@_01LELAEKIP@J@        0000000180018e9c     ClassLoader.obj
 0002:00000ea0       ??_C@_06NCGDPKCC@handle@   0000000180018ea0     ClassLoader.obj
 0002:00000ea8       ??_C@_01JPJNBJEM@I@        0000000180018ea8     ClassLoader.obj
 0002:00000eb0       ??_C@_0L@FFGJFOPI@jniVersion@ 0000000180018eb0     ClassLoader.obj
 0002:00000ec0       ??_C@_0O@CNBBEDNA@_JNI_OnLoad?$EA8@ 0000000180018ec0     ClassLoader.obj
 0002:00000ed0       ??_C@_0L@OIKEFKEO@JNI_OnLoad@ 0000000180018ed0     ClassLoader.obj
 0002:00000ee0       ??_C@_0BA@LDELBKAG@_JNI_OnUnload?$EA8@ 0000000180018ee0     ClassLoader.obj
 0002:00000ef0       ??_C@_0N@LLELHEHJ@JNI_OnUnload@ 0000000180018ef0     ClassLoader.obj
 0002:00000f00       ??_C@_0CO@NLJCNFHA@unsupported?5JNI?5version?50x?$CF08X?5@ 0000000180018f00     ClassLoader.obj
 0002:00000f30       ??_C@_0BP@JABHMODJ@java?1lang?1UnsatisfiedLinkError@ 0000000180018f30     ClassLoader.obj
 0002:00000f4f       ??_C@_00CNPNBAHC@@         0000000180018f4f     ClassLoader.obj
 0002:00000f50       ??_C@_04HLONOPDM@?4dll@    0000000180018f50     ClassLoader.obj
 0002:00000f58       ??_C@_0CB@CKDHIJCP@NULL?5filename?5for?5native?5librar@ 0000000180018f58     ClassLoader.obj
 0002:00000f7c       ??_C@_04BOOCJOME@ms?$CFd@  0000000180018f7c     Console_md.obj
 0002:00000f84       ??_C@_04LDGHIPEL@cp?$CFd@  0000000180018f84     Console_md.obj
 0002:00000f90       ??_C@_0BG@NEFMNKJA@GetConsoleMode?5failed@ 0000000180018f90     Console_md.obj
 0002:00000fa8       ??_C@_0BG@CBAKADNB@SetConsoleMode?5failed@ 0000000180018fa8     Console_md.obj
 0002:00000fc0       ??_C@_02ENHFDPNM@fd@       0000000180018fc0     FileDescriptor_md.obj
 0002:00000fc4       ??_C@_01POHCFINO@Z@        0000000180018fc4     FileDescriptor_md.obj
 0002:00000fc8       ??_C@_06PCICMFGG@append@   0000000180018fc8     FileDescriptor_md.obj
 0002:00000fd0       ??_C@_0M@IALGLCNJ@sync?5failed@ 0000000180018fd0     FileDescriptor_md.obj
 0002:00000fe0       ??_C@_0BM@MBMINGIL@java?1io?1SyncFailedException@ 0000000180018fe0     FileDescriptor_md.obj
 0002:00001000       ??_C@_0N@NOKLILHD@close?5failed@ 0000000180019000     FileDescriptor_md.obj
 0002:00001010       ??_C@_0BJ@BDFOFHPL@Ljava?1io?1FileDescriptor?$DL@ 0000000180019010     FileInputStream.obj
 0002:00001030       ??_C@_0O@KLFONINF@Stream?5Closed@ 0000000180019030     FileInputStream.obj
 0002:00001040       ??_C@_0L@FCLNKJKA@Seek?5error@ 0000000180019040     FileInputStream.obj
 0002:0000104c       ??_C@_11LOCGONAA@@         000000018001904c     HostLocaleProviderAdapter_md.obj
 0002:00001050       ??_C@_13BMLCKOLB@?$PP?$KE@ 0000000180019050     HostLocaleProviderAdapter_md.obj
 0002:00001054       ??_C@_15GMICKCJK@?$PP?$KE?$AA?5@ 0000000180019054     HostLocaleProviderAdapter_md.obj
 0002:0000105c       ??_C@_13EJFHHPOP@?$AA?$CF@ 000000018001905c     HostLocaleProviderAdapter_md.obj
 0002:00001060       ??_C@_15LJGOGFOH@?$AA?$CF?$AA?5@ 0000000180019060     HostLocaleProviderAdapter_md.obj
 0002:00001068       ??_C@_13LLDNKHDC@?$AA?$CI@ 0000000180019068     HostLocaleProviderAdapter_md.obj
 0002:0000106c       ??_C@_13IMODFHAA@?$AA?9@   000000018001906c     HostLocaleProviderAdapter_md.obj
 0002:00001070       ??_C@_15FFDNOHIK@?$AA?9?$AA?5@ 0000000180019070     HostLocaleProviderAdapter_md.obj
 0002:00001078       ??_C@_15GHMLFHFF@?$AA?$CI?$PP?$KE@ 0000000180019078     HostLocaleProviderAdapter_md.obj
 0002:00001080       ??_C@_15DHAGMGOG@?$AA?9?$PP?$KE@ 0000000180019080     HostLocaleProviderAdapter_md.obj
 0002:00001088       ??_C@_15JOOIHKEH@?$PP?$KE?$AA?9@ 0000000180019088     HostLocaleProviderAdapter_md.obj
 0002:00001090       ??_C@_17NKBBKLNH@?$AA?9?$PP?$KE?$AA?5@ 0000000180019090     HostLocaleProviderAdapter_md.obj
 0002:00001098       ??_C@_17OBCOLLDF@?$PP?$KE?$AA?5?$AA?9@ 0000000180019098     HostLocaleProviderAdapter_md.obj
 0002:000010a0       ??_C@_17JCPBKFLD@?$AA?$CI?$PP?$KE?$AA?5@ 00000001800190a0     HostLocaleProviderAdapter_md.obj
 0002:000010a8       ??_C@_15GCODBHLI@?$AA?9?$AA?$CF@ 00000001800190a8     HostLocaleProviderAdapter_md.obj
 0002:000010b0       ??_C@_15ELAELNDK@?$AA?$CF?$AA?9@ 00000001800190b0     HostLocaleProviderAdapter_md.obj
 0002:000010b8       ??_C@_17PPNGMKK@?$AA?9?$AA?$CF?$AA?5@ 00000001800190b8     HostLocaleProviderAdapter_md.obj
 0002:000010c0       ??_C@_17HOLPDOHB@?$AA?$CF?$AA?5?$AA?9@ 00000001800190c0     HostLocaleProviderAdapter_md.obj
 0002:000010c8       ??_C@_15ILJINFDI@?$AA?5?$PP?$KE@ 00000001800190c8     HostLocaleProviderAdapter_md.obj
 0002:000010d0       ??_C@_15NOHNAEGG@?$AA?5?$AA?$CF@ 00000001800190d0     HostLocaleProviderAdapter_md.obj
 0002:000010d8       ??_C@_13DIBMAFH@?$AA?$CJ@  00000001800190d8     HostLocaleProviderAdapter_md.obj
 0002:000010dc       ??_C@_13HOIJIPNN@?$AA?5@   00000001800190dc     HostLocaleProviderAdapter_md.obj
 0002:000010e0       ??_C@_15BLMJCMIJ@?$AA?5?$AA?9@ 00000001800190e0     HostLocaleProviderAdapter_md.obj
 0002:000010e8       ??_C@_15BBIKONBA@?$PP?$KE?$AA?$CJ@ 00000001800190e8     HostLocaleProviderAdapter_md.obj
 0002:000010f0       ??_C@_17LDHOGGNL@?$AA?5?$PP?$KE?$AA?9@ 00000001800190f0     HostLocaleProviderAdapter_md.obj
 0002:000010f8       ??_C@_17DNALNMHF@?$AA?9?$AA?5?$PP?$KE@ 00000001800190f8     HostLocaleProviderAdapter_md.obj
 0002:00001100       ??_C@_17DMBMPBIM@?$AA?5?$PP?$KE?$AA?$CJ@ 0000000180019100     HostLocaleProviderAdapter_md.obj
 0002:00001108       ??_C@_17GGJCKBKG@?$AA?5?$AA?$CF?$AA?9@ 0000000180019108     HostLocaleProviderAdapter_md.obj
 0002:00001110       ??_C@_17GIOOANCL@?$AA?9?$AA?5?$AA?$CF@ 0000000180019110     HostLocaleProviderAdapter_md.obj
 0002:00001118       ??_C@_0BA@ONOKGCMP@GetLocaleInfoEx@ 0000000180019118     HostLocaleProviderAdapter_md.obj
 0002:00001128       ??_C@_0N@MDJJJHMB@kernel32?4dll@ 0000000180019128     HostLocaleProviderAdapter_md.obj
 0002:00001138       ??_C@_0BC@NJJJJEJP@GetCalendarInfoEx@ 0000000180019138     HostLocaleProviderAdapter_md.obj
 0002:00001150       ??_C@_0BF@IALNPCBG@EnumCalendarInfoExEx@ 0000000180019150     HostLocaleProviderAdapter_md.obj
 0002:00001168       ??_C@_0BI@FKAGBMCL@memory?5allocation?5error@ 0000000180019168     HostLocaleProviderAdapter_md.obj
 0002:00001180       ??_C@_0BB@FLFAIHG@java?1lang?1String@ 0000000180019180     HostLocaleProviderAdapter_md.obj
 0002:00001198       ??_C@_17PINHLBBM@?$AAu?$AAn?$AAd@ 0000000180019198     HostLocaleProviderAdapter_md.obj
 0002:000011a0       ??_C@_15MNPNEAIF@?$AAe?$AAn@ 00000001800191a0     HostLocaleProviderAdapter_md.obj
 0002:000011a8       ??_C@_13PJJBFPED@?$AA?$DL@ 00000001800191a8     HostLocaleProviderAdapter_md.obj
 0002:000011ac       ??_C@_13DEFPDAGF@?$AA?0@   00000001800191ac     HostLocaleProviderAdapter_md.obj
 0002:000011b0       ??_C@_0BA@LGKIEDIB@package?5is?5null@ 00000001800191b0     Module.obj
 0002:000011c0       ??_C@_08PAGJBGJL@hashCode@ 00000001800191c0     Object.obj
 0002:000011cc       ??_C@_04PNOAOIAG@wait@     00000001800191cc     Object.obj
 0002:000011d4       ??_C@_04OHLIFDMD@?$CIJ?$CJV@ 00000001800191d4     Object.obj
 0002:000011dc       ??_C@_06LIGDCBBN@notify@   00000001800191dc     Object.obj
 0002:000011e4       ??_C@_03GAEACAIP@?$CI?$CJV@ 00000001800191e4     Object.obj
 0002:000011e8       ??_C@_09OHPHDMCN@notifyAll@ 00000001800191e8     Object.obj
 0002:000011f4       ??_C@_05KFBJCHHJ@clone@    00000001800191f4     Object.obj
 0002:00001200       ??_C@_0BF@LHBAMMHC@?$CI?$CJLjava?1lang?1Object?$DL@ 0000000180019200     Object.obj
 0002:00001218       ??_C@_0BM@LKJNLDJK@java?1lang?1NoSuchMethodError@ 0000000180019218     ObjectStreamClass.obj
 0002:00001238       ??_C@_08JOGLKNJI@?$DMclinit?$DO@ 0000000180019238     ObjectStreamClass.obj
 0002:00001244       ??_C@_05GBDANG@?$CI?$FLB?$CJV@ 0000000180019244     ProcessEnvironment_md.obj
 0002:0000124c       ??_C@_06FALKBLGB@?$DMinit?$DO@ 000000018001924c     ProcessEnvironment_md.obj
 0002:00001258       ??_C@_0BN@PKAKOFME@GetEnvironmentStrings?5failed@ 0000000180019258     ProcessEnvironment_md.obj
 0002:00001278       ??_C@_0BD@JFADHEFE@Ljava?1lang?1String?$DL@ 0000000180019278     ProcessHandleImpl_win.obj
 0002:00001290       ??_C@_07KMMNMMFF@command@  0000000180019290     ProcessHandleImpl_win.obj
 0002:00001298       ??_C@_0M@EELMKCHN@commandLine@ 0000000180019298     ProcessHandleImpl_win.obj
 0002:000012a8       ??_C@_0BE@KHJCLGPN@?$FLLjava?1lang?1String?$DL@ 00000001800192a8     ProcessHandleImpl_win.obj
 0002:000012c0       ??_C@_09PBNAMLIK@arguments@ 00000001800192c0     ProcessHandleImpl_win.obj
 0002:000012d0       ??_C@_09MJNIPNBH@totalTime@ 00000001800192d0     ProcessHandleImpl_win.obj
 0002:000012e0       ??_C@_09IIHJADCI@startTime@ 00000001800192e0     ProcessHandleImpl_win.obj
 0002:000012ec       ??_C@_04CCHAHKJA@user@     00000001800192ec     ProcessHandleImpl_win.obj
 0002:000012f8       ??_C@_0BD@OOONFEIA@GetExitCodeProcess@ 00000001800192f8     ProcessHandleImpl_win.obj
 0002:00001310       ??_C@_0BL@IONOAEOO@java?1lang?1RuntimeException@ 0000000180019310     ProcessHandleImpl_win.obj
 0002:00001330       ??_C@_0BH@LBENJJIP@WaitForMultipleObjects@ 0000000180019330     ProcessHandleImpl_win.obj
 0002:00001348       ??_C@_0BH@DJKIHHBP@snapshot?5not?5available@ 0000000180019348     ProcessHandleImpl_win.obj
 0002:00001360       ??_C@_0BG@LPMGLOAP@array?5sizes?5not?5equal@ 0000000180019360     ProcessHandleImpl_win.obj
 0002:00001378       ??_C@_0BE@JIDLIKOL@GetTokenInformation@ 0000000180019378     ProcessHandleImpl_win.obj
 0002:0000138c       ??_C@_13FPGAJAPJ@?$AA?2@   000000018001938c     ProcessHandleImpl_win.obj
 0002:00001390       ??_C@_1CA@BNEMBNGE@?$AA?$CF?$AAs?$AA?5?$AAe?$AAr?$AAr?$AAo?$AAr?$AA?$DN?$AA?$CF?$AAd?$AA?0?$AA?5?$AA?$CF?$AAs@ 0000000180019390     ProcessImpl_md.obj
 0002:000013b0       ??_C@_1CI@OBOFAJOJ@?$AA?$CF?$AAs?$AA?5?$AAf?$AAa?$AAi?$AAl?$AAe?$AAd?$AA?0?$AA?5?$AAe?$AAr?$AAr?$AAo@ 00000001800193b0     ProcessImpl_md.obj
 0002:000013d8       ??_C@_0CM@EAKDBECK@Secondary?5error?5while?5OS?5messag@ 00000001800193d8     ProcessImpl_md.obj
 0002:00001408       ??_C@_1BG@HKMEIOD@?$AAC?$AAr?$AAe?$AAa?$AAt?$AAe?$AAP?$AAi?$AAp?$AAe@ 0000000180019408     ProcessImpl_md.obj
 0002:00001420       ??_C@_1BM@MMIOBBBF@?$AAC?$AAr?$AAe?$AAa?$AAt?$AAe?$AAP?$AAr?$AAo?$AAc?$AAe?$AAs?$AAs@ 0000000180019420     ProcessImpl_md.obj
 0002:00001440       ??_C@_1CG@LCLEBLIK@?$AAG?$AAe?$AAt?$AAE?$AAx?$AAi?$AAt?$AAC?$AAo?$AAd?$AAe?$AAP?$AAr?$AAo?$AAc@ 0000000180019440     ProcessImpl_md.obj
 0002:00001468       ??_C@_1CO@PLEHGDKC@?$AAW?$AAa?$AAi?$AAt?$AAF?$AAo?$AAr?$AAM?$AAu?$AAl?$AAt?$AAi?$AAp?$AAl?$AAe@ 0000000180019468     ProcessImpl_md.obj
 0002:00001498       ??_C@_0M@GPOOGHPH@CreateFileW@ 0000000180019498     ProcessImpl_md.obj
 0002:000014b0       __xmm@ffffffffffffffffffffffffffffffff 00000001800194b0     ProcessImpl_md.obj
 0002:000014c0       ??_C@_0M@HPFDGGMC@Seek?5failed@ 00000001800194c0     RandomAccessFile.obj
 0002:000014d0       ??_C@_0BB@CEBOPAFI@GetLength?5failed@ 00000001800194d0     RandomAccessFile.obj
 0002:000014e8       ??_C@_0BF@HDGNMJHD@Negative?5seek?5offset@ 00000001800194e8     RandomAccessFile.obj
 0002:00001500       ??_C@_0BB@GOOEHMBA@setLength?5failed@ 0000000180019500     RandomAccessFile.obj
 0002:00001518       ??_C@_0BK@FOJCHAGK@java?1lang?1SecurityManager@ 0000000180019518     SecurityManager.obj
 0002:00001538       ??_C@_0M@PBLAKOBI@initialized@ 0000000180019538     SecurityManager.obj
 0002:00001548       ??_C@_0BM@MPFHLPCE@java?1lang?1SecurityException@ 0000000180019548     SecurityManager.obj
 0002:00001568       ??_C@_0CC@HPKFBHGI@security?5manager?5not?5initialize@ 0000000180019568     SecurityManager.obj
 0002:0000158c       ??_C@_04MEMAJGDJ@name@     000000018001958c     Signal.obj
 0002:00001594       ??_C@_02DKCKIIND@?$CFs@    0000000180019594     StringCoding.obj
 0002:00001598       ??_C@_0BC@JMDLHMGP@currentTimeMillis@ 0000000180019598     System.obj
 0002:000015ac       ??_C@_03IGDHHNNC@?$CI?$CJJ@ 00000001800195ac     System.obj
 0002:000015b0       ??_C@_08GAAFINGG@nanoTime@ 00000001800195b0     System.obj
 0002:000015c0       ??_C@_09EEHNOAG@arraycopy@ 00000001800195c0     System.obj
 0002:000015d0       ??_C@_0CL@DPOGMIND@?$CILjava?1lang?1Object?$DLILjava?1lang?1@ 00000001800195d0     System.obj
 0002:00001600       ??_C@_0L@MMANBJOI@?$CFs?4display@ 0000000180019600     System.obj
 0002:00001610       ??_C@_09MJAPJFKN@?$CFs?4format@ 0000000180019610     System.obj
 0002:00001620       ??_C@_0DJ@FLFJBGBN@?$CILjava?1lang?1Object?$DLLjava?1lang?1O@ 0000000180019620     System.obj
 0002:0000165c       ??_C@_03KMONJGDG@put@      000000018001965c     System.obj
 0002:00001660       ??_C@_0CH@JHKCBJOB@?$CILjava?1lang?1Object?$DL?$CJLjava?1lang?1@ 0000000180019660     System.obj
 0002:00001688       ??_C@_06LEMKAMD@remove@    0000000180019688     System.obj
 0002:00001690       ??_C@_0CH@NCPCFFHJ@?$CILjava?1lang?1String?$DL?$CJLjava?1lang?1@ 0000000180019690     System.obj
 0002:000016b8       ??_C@_0M@NBNLNHMA@getProperty@ 00000001800196b8     System.obj
 0002:000016c8       ??_C@_0BL@KBDBBBPF@java?4specification?4version@ 00000001800196c8     System.obj
 0002:000016e4       ??_C@_02ODEKKOPI@11@       00000001800196e4     System.obj
 0002:000016e8       ??_C@_0CH@LBKCLBBN@java?4specification?4maintenance?4@ 00000001800196e8     System.obj
 0002:00001710       ??_C@_01EKENIIDA@3@        0000000180019710     System.obj
 0002:00001718       ??_C@_0BI@OKHEICGJ@java?4specification?4name@ 0000000180019718     System.obj
 0002:00001730       ??_C@_0CA@KOJBOKHO@Java?5Platform?5API?5Specification@ 0000000180019730     System.obj
 0002:00001750       ??_C@_0BK@NJLHMCPF@java?4specification?4vendor@ 0000000180019750     System.obj
 0002:00001770       ??_C@_0BD@HKAOFKOF@Oracle?5Corporation@ 0000000180019770     System.obj
 0002:00001784       ??_C@_05KBEOJPB@?$CFd?4?$CFd@ 0000000180019784     System.obj
 0002:00001790       ??_C@_0BD@FIJFIPLK@java?4class?4version@ 0000000180019790     System.obj
 0002:000017a8       ??_C@_0M@EFKDJKKO@awt?4toolkit@ 00000001800197a8     System.obj
 0002:000017b8       ??_C@_07IOCNKCKK@os?4name@ 00000001800197b8     System.obj
 0002:000017c0       ??_C@_0L@LFOLPEHK@os?4version@ 00000001800197c0     System.obj
 0002:000017d0       ??_C@_07PBOBJOEN@os?4arch@ 00000001800197d0     System.obj
 0002:000017d8       ??_C@_0P@EIENLPCI@file?4separator@ 00000001800197d8     System.obj
 0002:000017e8       ??_C@_0P@GNCHJOPK@path?4separator@ 00000001800197e8     System.obj
 0002:000017f8       ??_C@_0P@EPBOHHHF@line?4separator@ 00000001800197f8     System.obj
 0002:00001808       ??_C@_0BE@PAJOPCOJ@sun?4stdout?4encoding@ 0000000180019808     System.obj
 0002:00001820       ??_C@_0BE@FGOMLHAD@sun?4stderr?4encoding@ 0000000180019820     System.obj
 0002:00001838       ??_C@_0BI@KFHOHPJL@sun?4io?4unicode?4encoding@ 0000000180019838     System.obj
 0002:00001850       ??_C@_0BA@PDNGFEIL@sun?4cpu?4isalist@ 0000000180019850     System.obj
 0002:00001860       ??_C@_0P@EOOEEPOA@sun?4cpu?4endian@ 0000000180019860     System.obj
 0002:00001870       ??_C@_0BE@HFHNEHBI@java?4awt?4printerjob@ 0000000180019870     System.obj
 0002:00001884       ??_C@_02JLHCEMDI@64@       0000000180019884     System.obj
 0002:00001888       ??_C@_0BE@EHGHNJFA@sun?4arch?4data?4model@ 0000000180019888     System.obj
 0002:000018a0       ??_C@_0BD@ELJFNNDH@sun?4os?4patch?4level@ 00000001800198a0     System.obj
 0002:000018b8       ??_C@_0BF@EKEAJFNI@java?4awt?4graphicsenv@ 00000001800198b8     System.obj
 0002:000018d0       ??_C@_0BE@BAAMABKP@sun?4java2d?4fontpath@ 00000001800198d0     System.obj
 0002:000018e8       ??_C@_0P@JIMDBPAK@java?4io?4tmpdir@ 00000001800198e8     System.obj
 0002:000018f8       ??_C@_09OGHMLDAF@user?4name@ 00000001800198f8     System.obj
 0002:00001908       ??_C@_09IJODDBJG@user?4home@ 0000000180019908     System.obj
 0002:00001918       ??_C@_0O@FKMKHEGF@user?4timezone@ 0000000180019918     System.obj
 0002:00001928       ??_C@_08IOMDCONK@user?4dir@ 0000000180019928     System.obj
 0002:00001938       ??_C@_0M@LLAEMPMH@sun?4desktop@ 0000000180019938     System.obj
 0002:00001948       ??_C@_0O@IPEJOPEC@user?4language@ 0000000180019948     System.obj
 0002:00001958       ??_C@_0M@NDBKMHED@user?4script@ 0000000180019958     System.obj
 0002:00001968       ??_C@_0N@IOCKJEEA@user?4country@ 0000000180019968     System.obj
 0002:00001978       ??_C@_0N@ICDOLPAO@user?4variant@ 0000000180019978     System.obj
 0002:00001988       ??_C@_0O@FMHCFFFK@file?4encoding@ 0000000180019988     System.obj
 0002:00001998       ??_C@_0BB@PEJNKEBD@sun?4jnu?4encoding@ 0000000180019998     System.obj
 0002:000019b0       ??_C@_0BG@GPDHLGHH@Ljava?1io?1InputStream?$DL@ 00000001800199b0     System.obj
 0002:000019c8       ??_C@_02LMMGJAGL@in@       00000001800199c8     System.obj
 0002:000019d0       ??_C@_0BG@FPECDKGJ@Ljava?1io?1PrintStream?$DL@ 00000001800199d0     System.obj
 0002:000019e8       ??_C@_03KEJHNBPP@out@      00000001800199e8     System.obj
 0002:000019ec       ??_C@_03JIDPIAJI@err@      00000001800199ec     System.obj
 0002:000019f0       ??_C@_0O@OLOAHEKB@name?5too?5long@ 00000001800199f0     System.obj
 0002:00001a00       ??_C@_06MGHKGFHF@start0@   0000000180019a00     Thread.obj
 0002:00001a08       ??_C@_05CHCLNOMK@stop0@    0000000180019a08     Thread.obj
 0002:00001a10       ??_C@_0BG@JLFLBLJI@?$CILjava?1lang?1Object?$DL?$CJV@ 0000000180019a10     Thread.obj
 0002:00001a28       ??_C@_07BOOHCBLM@isAlive@  0000000180019a28     Thread.obj
 0002:00001a30       ??_C@_08PIHJGBMA@suspend0@ 0000000180019a30     Thread.obj
 0002:00001a40       ??_C@_07EJLENFAP@resume0@  0000000180019a40     Thread.obj
 0002:00001a48       ??_C@_0N@GOFHJCMI@setPriority0@ 0000000180019a48     Thread.obj
 0002:00001a58       ??_C@_04PFANPMCN@?$CII?$CJV@ 0000000180019a58     Thread.obj
 0002:00001a60       ??_C@_05LKJGIMLP@yield@    0000000180019a60     Thread.obj
 0002:00001a68       ??_C@_05PCJCMMHD@sleep@    0000000180019a68     Thread.obj
 0002:00001a70       ??_C@_0O@GIDKOGNF@currentThread@ 0000000180019a70     Thread.obj
 0002:00001a80       ??_C@_0BF@GLBLFFEM@?$CI?$CJLjava?1lang?1Thread?$DL@ 0000000180019a80     Thread.obj
 0002:00001a98       ??_C@_0BB@DMGBDJPC@countStackFrames@ 0000000180019a98     Thread.obj
 0002:00001ab0       ??_C@_0L@KOCFLKPP@interrupt0@ 0000000180019ab0     Thread.obj
 0002:00001ac0       ??_C@_0O@NBKAIMLM@isInterrupted@ 0000000180019ac0     Thread.obj
 0002:00001ad0       ??_C@_04BLBEELFA@?$CIZ?$CJZ@ 0000000180019ad0     Thread.obj
 0002:00001ad8       ??_C@_09BKEKKKBN@holdsLock@ 0000000180019ad8     Thread.obj
 0002:00001ae8       ??_C@_0BG@DHOOFEJE@?$CILjava?1lang?1Object?$DL?$CJZ@ 0000000180019ae8     Thread.obj
 0002:00001b00       ??_C@_0L@MBENOCKD@getThreads@ 0000000180019b00     Thread.obj
 0002:00001b10       ??_C@_0BG@CJDMDLMO@?$CI?$CJ?$FLLjava?1lang?1Thread?$DL@ 0000000180019b10     Thread.obj
 0002:00001b28       ??_C@_0M@ECOKKOKF@dumpThreads@ 0000000180019b28     Thread.obj
 0002:00001b38       ??_C@_0DF@ELFIABCA@?$CI?$FLLjava?1lang?1Thread?$DL?$CJ?$FL?$FLLjava?1la@ 0000000180019b38     Thread.obj
 0002:00001b70       ??_C@_0O@LPHHHNKJ@setNativeName@ 0000000180019b70     Thread.obj
 0002:00001b80       ??_C@_0BG@IKDDPPGD@?$CILjava?1lang?1String?$DL?$CJV@ 0000000180019b80     Thread.obj
 0002:00001b98       ??_C@_1BK@BOBBLECB@?$AAS?$AAt?$AAa?$AAn?$AAd?$AAa?$AAr?$AAd?$AAN?$AAa?$AAm?$AAe@ 0000000180019b98     TimeZone_md.obj
 0002:00001bb8       ??_C@_0N@PEHDGIGO@StandardName@ 0000000180019bb8     TimeZone_md.obj
 0002:00001bc8       ??_C@_17GFIDPLDA@?$AAS?$AAt?$AAd@ 0000000180019bc8     TimeZone_md.obj
 0002:00001bd0       ??_C@_03FFGKOOIA@Std@      0000000180019bd0     TimeZone_md.obj
 0002:00001bd8       ??_C@_0P@EKMDNJBA@GMT?$CFc?$CF02d?3?$CF02d@ 0000000180019bd8     TimeZone_md.obj
 0002:00001be8       ??_C@_03HOONMGKE@GMT@      0000000180019be8     TimeZone_md.obj
 0002:00001bf0       ??_C@_0DF@OCPBGDJE@System?2CurrentControlSet?2Contro@ 0000000180019bf0     TimeZone_md.obj
 0002:00001c28       ??_C@_0BM@HEGPJGEC@DynamicDaylightTimeDisabled@ 0000000180019c28     TimeZone_md.obj
 0002:00001c48       ??_C@_0BA@GCKJIEGO@TimeZoneKeyName@ 0000000180019c48     TimeZone_md.obj
 0002:00001c58       ??_C@_0DI@LLEGOPFO@SOFTWARE?2Microsoft?2Windows?5NT?2C@ 0000000180019c58     TimeZone_md.obj
 0002:00001c90       ??_C@_0DF@JEJGGGGH@SOFTWARE?2Microsoft?2Windows?2Curr@ 0000000180019c90     TimeZone_md.obj
 0002:00001cc8       ??_C@_03NKEEOHDM@TZI@      0000000180019cc8     TimeZone_md.obj
 0002:00001cd0       ??_C@_0BA@PBEHAGHA@?2lib?2tzmappings@ 0000000180019cd0     TimeZone_md.obj
 0002:00001ce0       ??_C@_01KDCPPGHE@r@        0000000180019ce0     TimeZone_md.obj
 0002:00001ce8       ??_C@_0BA@PMGFJNJD@can?8t?5open?5?$CFs?4?6@ 0000000180019ce8     TimeZone_md.obj
 0002:00001cf8       ??_C@_0BG@MJJAMJBB@premature?5end?5of?5line@ 0000000180019cf8     TimeZone_md.obj
 0002:00001d10       ??_C@_0BN@NFCIANLB@illegal?5null?5character?5found@ 0000000180019d10     TimeZone_md.obj
 0002:00001d30       ??_C@_0CE@OJDILIEN@illegal?5non?9newline?5character?5f@ 0000000180019d30     TimeZone_md.obj
 0002:00001d54       ??_C@_03MMKGDKGA@001@      0000000180019d54     TimeZone_md.obj
 0002:00001d58       ??_C@_0DO@EINJANBE@Illegal?5format?5in?5tzmappings?5fi@ 0000000180019d58     TimeZone_md.obj
 0002:00001d98       ??_C@_0P@DOCHMBNE@ActiveTimeBias@ 0000000180019d98     TimeZone_md.obj
 0002:00001da8       ??_C@_0BG@FPHJJCID@getNanoTimeAdjustment@ 0000000180019da8     VM.obj
 0002:00001dc0       ??_C@_04BMPAOJO@?$CIJ?$CJJ@ 0000000180019dc0     VM.obj
 0002:00001dc8       ??_C@_0CL@NBAOCADG@Handle?5for?5JVM?5not?5found?5for?5sy@ 0000000180019dc8     VM.obj
 0002:00001df4       ??_C@_04JCEIFDIJ@J2SE@     0000000180019df4     WinCAPISeedGenerator.obj
 0002:00001e00       ??_C@_0N@IOFABHFH@java?1io?1File@ 0000000180019e00     WinNTFileSystem_md.obj
 0002:00001e10       ??_C@_04LNEJFJGI@path@     0000000180019e10     WinNTFileSystem_md.obj
 0002:00001e18       ??_C@_0BK@PDKDDAF@GetFinalPathNameByHandleW@ 0000000180019e18     WinNTFileSystem_md.obj
 0002:00001e38       ??_C@_0CA@NIIGFDJD@native?5memory?5allocation?5failed@ 0000000180019e38     WinNTFileSystem_md.obj
 0002:00001e58       ??_C@_0N@NMICNPLE@Bad?5pathname@ 0000000180019e58     WinNTFileSystem_md.obj
 0002:00001e68       ??_C@_17LIAKHCCP@?$AAC?$AAO?$AAN@ 0000000180019e68     WinNTFileSystem_md.obj
 0002:00001e70       ??_C@_17PFHGFFKC@?$AAP?$AAR?$AAN@ 0000000180019e70     WinNTFileSystem_md.obj
 0002:00001e78       ??_C@_17CNBAFMOM@?$AAA?$AAU?$AAX@ 0000000180019e78     WinNTFileSystem_md.obj
 0002:00001e80       ??_C@_17CLELIOII@?$AAN?$AAU?$AAL@ 0000000180019e80     WinNTFileSystem_md.obj
 0002:00001e88       ??_C@_17KKLPNNMB@?$AAC?$AAO?$AAM@ 0000000180019e88     WinNTFileSystem_md.obj
 0002:00001e90       ??_C@_17KMAOGHDG@?$AAL?$AAP?$AAT@ 0000000180019e90     WinNTFileSystem_md.obj
 0002:00001e98       ??_C@_0BE@LONNMHBH@Could?5not?5open?5file@ 0000000180019e98     WinNTFileSystem_md.obj
 0002:00001eac       ??_C@_13BBDEGPLJ@?$AA?$CK@ 0000000180019eac     WinNTFileSystem_md.obj
 0002:00001eb0       ??_C@_15PKPONJIK@?$AA?2?$AA?$CK@ 0000000180019eb0     WinNTFileSystem_md.obj
 0002:00001eb8       ??_C@_13JOFGPIOO@?$AA?4@   0000000180019eb8     WinNTFileSystem_md.obj
 0002:00001ebc       ??_C@_15DDHGOCBH@?$AA?4?$AA?4@ 0000000180019ebc     WinNTFileSystem_md.obj
 0002:00001ec8       ??_C@_0CH@PNOGCBMH@Could?5not?5get?5maximum?5component@ 0000000180019ec8     WinNTFileSystem_md.obj
 0002:00001ef0       ??_C@_19BKJMDJK@?$AA?2?$AA?2?$AA?4?$AA?2@ 0000000180019ef0     canonicalize_md.obj
 0002:00001f00       ??_C@_1BC@FBJNHMLC@?$AA?2?$AA?2?$AA?$DP?$AA?2?$AAU?$AAN?$AAC?$AA?$AA@ 0000000180019f00     canonicalize_md.obj
 0002:00001f18       ??_C@_1M@DJNCMBIG@?$AA?2?$AA?2?$AA?$DP?$AA?2?$AA?$AA@ 0000000180019f18     canonicalize_md.obj
 0002:00001f28       ??_C@_0DG@ONCIMJCB@JVM?5interface?5version?5mismatch?3@ 0000000180019f28     check_version.obj
 0002:00001f60       ??_C@_0L@BHPPDFMA@Read?5error@ 0000000180019f60     io_util.obj
 0002:00001f70       ??_C@_0CE@JOEPHHFN@java?1lang?1IndexOutOfBoundsExcep@ 0000000180019f70     io_util.obj
 0002:00001f98       ??_C@_0M@PJBDJJDJ@Write?5error@ 0000000180019f98     io_util.obj
 0002:00001fa8       ??_C@_0CI@HEGLGDKJ@?$CILjava?1lang?1String?$DLLjava?1lang?1S@ 0000000180019fa8     io_util.obj
 0002:00001fd0       ??_C@_0BO@FDOOLAPO@java?1io?1FileNotFoundException@ 0000000180019fd0     io_util.obj
 0002:00001ff0       ??_C@_05EGJIMALK@UTF?98@   0000000180019ff0     java_props_md.obj
 0002:00001ff8       ??_C@_03LIOLIPAH@GBK@      0000000180019ff8     java_props_md.obj
 0002:00002000       ??_C@_07DNCGDNOG@GB18030@  000000018001a000     java_props_md.obj
 0002:00002008       ??_C@_05PCINFEFG@MS950@    000000018001a008     java_props_md.obj
 0002:00002010       ??_C@_0P@JHCFFHNK@MS950_HKSCS_XP@ 000000018001a010     java_props_md.obj
 0002:00002020       ??_C@_0BH@NKFNLGAB@?2FONTS?2SimSun18030?4ttc@ 000000018001a020     java_props_md.obj
 0002:00002038       ??_C@_01JOAMLHOP@?9@       000000018001a038     java_props_md.obj
 0002:0000203c       ??_C@_04LFKJOHGN@ia64@     000000018001a03c     java_props_md.obj
 0002:00002044       ??_C@_05MDLPDLNO@amd64@    000000018001a044     java_props_md.obj
 0002:00002050       ??_C@_0DO@DIFICBBG@pentium_pro?$CLmmx?5pentium_pro?5pen@ 000000018001a050     java_props_md.obj
 0002:00002090       ??_C@_0CC@BIODACBF@pentium_pro?5pentium?5i486?5i386?5i@ 000000018001a090     java_props_md.obj
 0002:000020b8       ??_C@_0CC@PPFBHJAM@pentium?$CLmmx?5pentium?5i486?5i386?5i@ 000000018001a0b8     java_props_md.obj
 0002:000020e0       ??_C@_0BG@CMPGKFGL@pentium?5i486?5i386?5i86@ 000000018001a0e0     java_props_md.obj
 0002:000020f8       ??_C@_0O@MAAOGNKJ@i486?5i386?5i86@ 000000018001a0f8     java_props_md.obj
 0002:00002108       ??_C@_08IPFADFGF@i386?5i86@ 000000018001a108     java_props_md.obj
 0002:00002118       ??_C@_0BH@NIHCMEPJ@?$CF?$CK?$FLa?9z?2?9?$FN?$CF1?$FLA?9Z?$FN?$CF?$FLa?9z?$FN@ 000000018001a118     java_props_md.obj
 0002:00002130       ??_C@_02LFNMGJAP@en@       000000018001a130     java_props_md.obj
 0002:00002134       ??_C@_02PLFPMECB@US@       000000018001a134     java_props_md.obj
 0002:00002138       ??_C@_02BFDMMJOC@nb@       000000018001a138     java_props_md.obj
 0002:0000213c       ??_C@_02KAJCLHKP@no@       000000018001a13c     java_props_md.obj
 0002:00002140       ??_C@_02NFLNFON@NO@        000000018001a140     java_props_md.obj
 0002:00002144       ??_C@_02LJIJIGOO@nn@       000000018001a144     java_props_md.obj
 0002:00002148       ??_C@_02BBMDGADK@NY@       000000018001a148     java_props_md.obj
 0002:00002150       ??_C@_0BJ@LLNEBFHD@sun?4awt?4windows?4WToolkit@ 000000018001a150     java_props_md.obj
 0002:00002170       ??_C@_0BM@DKPHMFNL@sun?4awt?4windows?4WPrinterJob@ 000000018001a170     java_props_md.obj
 0002:00002190       ??_C@_0CB@BDHJBLNP@sun?4awt?4Win32GraphicsEnvironmen@ 000000018001a190     java_props_md.obj
 0002:000021b8       ??_C@_1CA@GPNFACCO@?$AAJ?$AAA?$AAV?$AAA?$AA2?$AAD?$AA_?$AAF?$AAO?$AAN?$AAT?$AAP?$AAA?$AAT?$AAH@ 000000018001a1b8     java_props_md.obj
 0002:000021d8       ??_C@_0O@BAKIPCDE@?2kernel32?4dll@ 000000018001a1d8     java_props_md.obj
 0002:000021e8       ??_C@_1BM@JEABEHHA@?$AA?2?$AAk?$AAe?$AAr?$AAn?$AAe?$AAl?$AA3?$AA2?$AA?4?$AAd?$AAl?$AAl@ 000000018001a1e8     java_props_md.obj
 0002:00002208       ??_C@_0L@NEBNHFIE@Windows?595@ 000000018001a208     java_props_md.obj
 0002:00002218       ??_C@_0L@GBLDALMJ@Windows?598@ 000000018001a218     java_props_md.obj
 0002:00002228       ??_C@_0L@DNFOOIFM@Windows?5Me@ 000000018001a228     java_props_md.obj
 0002:00002238       ??_C@_0BF@KOJMMOAG@Windows?59X?5?$CIunknown?$CJ@ 000000018001a238     java_props_md.obj
 0002:00002250       ??_C@_0L@PJEFFBLH@Windows?5NT@ 000000018001a250     java_props_md.obj
 0002:00002260       ??_C@_0N@MEKDBOKB@Windows?52000@ 000000018001a260     java_props_md.obj
 0002:00002270       ??_C@_0L@IFICELHB@Windows?5XP@ 000000018001a270     java_props_md.obj
 0002:00002280       ??_C@_0N@OPIOENGC@Windows?52003@ 000000018001a280     java_props_md.obj
 0002:00002290       ??_C@_0BF@GMBBPJFL@Windows?5NT?5?$CIunknown?$CJ@ 000000018001a290     java_props_md.obj
 0002:000022a8       ??_C@_0O@IFKHFILP@Windows?5Vista@ 000000018001a2a8     java_props_md.obj
 0002:000022b8       ??_C@_09GOHFIPMO@Windows?57@ 000000018001a2b8     java_props_md.obj
 0002:000022c8       ??_C@_09OJONJDAB@Windows?58@ 000000018001a2c8     java_props_md.obj
 0002:000022d8       ??_C@_0M@IEJDHGAK@Windows?58?41@ 000000018001a2d8     java_props_md.obj
 0002:000022e8       ??_C@_0BE@GHBPPLPA@Windows?5Server?52008@ 000000018001a2e8     java_props_md.obj
 0002:00002300       ??_C@_0BH@ONPOEHKF@Windows?5Server?52008?5R2@ 000000018001a300     java_props_md.obj
 0002:00002318       ??_C@_0BE@JMDCHJEN@Windows?5Server?52012@ 000000018001a318     java_props_md.obj
 0002:00002330       ??_C@_0BH@GMBCIMKB@Windows?5Server?52012?5R2@ 000000018001a330     java_props_md.obj
 0002:00002348       ??_C@_0L@LOGCOBDI@Windows?511@ 000000018001a348     java_props_md.obj
 0002:00002358       ??_C@_0L@KHHJNAHJ@Windows?510@ 000000018001a358     java_props_md.obj
 0002:00002368       ??_C@_0BE@NBDFFBND@Windows?5Server?52025@ 000000018001a368     java_props_md.obj
 0002:00002380       ??_C@_0BE@JOHEMHBE@Windows?5Server?52022@ 000000018001a380     java_props_md.obj
 0002:00002398       ??_C@_0BE@HPMGKAIG@Windows?5Server?52019@ 000000018001a398     java_props_md.obj
 0002:000023b0       ??_C@_0BE@PIFOLMEJ@Windows?5Server?52016@ 000000018001a3b0     java_props_md.obj
 0002:000023c8       ??_C@_0BC@JFKFADHL@Windows?5?$CIunknown?$CJ@ 000000018001a3c8     java_props_md.obj
 0002:000023e0       ??_C@_07EKMDLNDL@windows@  000000018001a3e0     java_props_md.obj
 0002:000023e8       ??_C@_06LADGIEOA@little@   000000018001a3e8     java_props_md.obj
 0002:000023f0       ??_C@_1BC@GGLDBIGJ@?$AAU?$AAS?$AAE?$AAR?$AAN?$AAA?$AAM?$AAE@ 000000018001a3f0     java_props_md.obj
 0002:00002408       ??_C@_1BA@KDMGPDJH@?$AAu?$AAn?$AAk?$AAn?$AAo?$AAw?$AAn@ 000000018001a408     java_props_md.obj
 0002:00002418       ??_C@_17BJPFHBEJ@?$AAC?$AA?3?$AA?2@ 000000018001a418     java_props_md.obj
 0002:00002420       ??_C@_0M@JNHAKOPM@MS950_HKSCS@ 000000018001a420     java_props_md.obj
 0002:00002430       ??_C@_0O@KBEEOPPB@UnicodeLittle@ 000000018001a430     java_props_md.obj
 0002:00002440       ??_C@_01KICIPPFI@?2@       000000018001a440     java_props_md.obj
 0002:00002444       ??_C@_01ICJEACDI@?$DL@     000000018001a444     java_props_md.obj
 0002:00002448       ??_C@_02PCIJFNDE@?$AN?6@   000000018001a448     java_props_md.obj
 0002:00002450       ??_C@_07KCBEICKO@jvm?4dll@ 000000018001a450     jdk_util_md.obj
 0002:00002458       ??_C@_0BP@GJLHLAKJ@java?1lang?1NullPointerException@ 000000018001a458     jni_util.obj
 0002:00002478       ??_C@_0CJ@ODBKFPOB@java?1lang?1ArrayIndexOutOfBounds@ 000000018001a478     jni_util.obj
 0002:000024a8       ??_C@_0BL@ENCPOIKC@java?1lang?1OutOfMemoryError@ 000000018001a4a8     jni_util.obj
 0002:000024c8       ??_C@_0CD@MOHADDFA@java?1lang?1IllegalArgumentExcept@ 000000018001a4c8     jni_util.obj
 0002:000024f0       ??_C@_0BN@BNEPGEKD@java?1lang?1IllegalAccessError@ 000000018001a4f0     jni_util.obj
 0002:00002510       ??_C@_0CB@DKOJJLNI@java?1lang?1IllegalAccessExceptio@ 000000018001a510     jni_util.obj
 0002:00002538       ??_C@_0BI@NBLNIHIB@java?1lang?1InternalError@ 000000018001a538     jni_util.obj
 0002:00002550       ??_C@_0BP@OCPHDAGE@java?1lang?1NoSuchFieldException@ 000000018001a550     jni_util.obj
 0002:00002570       ??_C@_0CA@MELAJOJA@java?1lang?1NoSuchMethodException@ 000000018001a570     jni_util.obj
 0002:00002590       ??_C@_0CB@KCPANAMN@java?1lang?1ClassNotFoundExceptio@ 000000018001a590     jni_util.obj
 0002:000025b8       ??_C@_0CA@EACDMHAF@java?1lang?1NumberFormatException@ 000000018001a5b8     jni_util.obj
 0002:000025d8       ??_C@_0BE@EBAPEBGJ@java?1io?1IOException@ 000000018001a5d8     jni_util.obj
 0002:000025f0       ??_C@_0BL@MDAGAKCG@java?1lang?1NoSuchFieldError@ 000000018001a5f0     jni_util.obj
 0002:00002610       ??_C@_0CK@GIGMFKA@java?1lang?1StringIndexOutOfBound@ 000000018001a610     jni_util.obj
 0002:00002640       ??_C@_0CB@DFBEHFCE@java?1lang?1InstantiationExceptio@ 000000018001a640     jni_util.obj
 0002:00002664       ??_C@_05DNDNCJEB@?5?$CI?$CFs?$CJ@ 000000018001a664     jni_util.obj
 0002:0000266c       ??_C@_06CMLIEHFC@concat@   000000018001a66c     jni_util.obj
 0002:00002678       ??_C@_0BH@GDIHDDN@no?5further?5information@ 000000018001a678     jni_util.obj
 0002:00002690       ??_C@_0CO@NPADHBGE@JNU_CallStaticMethodByName?3?5ill@ 000000018001a690     jni_util.obj
 0002:000026c0       ??_C@_0CJ@MELNKLJP@JNU_CallMethodByNameV?3?5illegal?5@ 000000018001a6c0     jni_util.obj
 0002:000026f0       ??_C@_0BG@CGIGLAGP@?$CILjava?1lang?1String?$DL?$CJZ@ 000000018001a6f0     jni_util.obj
 0002:00002708       ??_C@_0M@CPFODPBC@isSupported@ 000000018001a708     jni_util.obj
 0002:00002718       ??_C@_0BJ@ECKJLLIP@java?1nio?1charset?1Charset@ 000000018001a718     jni_util.obj
 0002:00002734       ??_C@_06FEGJKAJG@8859_1@   000000018001a734     jni_util.obj
 0002:00002740       ??_C@_09KEDHCKDI@ISO8859?91@ 000000018001a740     jni_util.obj
 0002:00002750       ??_C@_09PDECJGAG@ISO8859_1@ 000000018001a750     jni_util.obj
 0002:00002760       ??_C@_0L@GJIJNDEK@ISO?98859?91@ 000000018001a760     jni_util.obj
 0002:00002770       ??_C@_09BGDIBLML@ISO646?9US@ 000000018001a770     jni_util.obj
 0002:0000277c       ??_C@_06BFOBJALC@Cp1252@   000000018001a77c     jni_util.obj
 0002:00002788       ??_C@_08MIMKAGHL@utf?916le@ 000000018001a788     jni_util.obj
 0002:00002798       ??_C@_0BM@KEODIIBN@platform?5encoding?5undefined@ 000000018001a798     jni_util.obj
 0002:000027b8       ??_C@_0BH@BOKGLNMJ@?$CILjava?1lang?1String?$DL?$CJ?$FLB@ 000000018001a7b8     jni_util.obj
 0002:000027d0       ??_C@_08LJNJGADH@getBytes@ 000000018001a7d0     jni_util.obj
 0002:000027e0       ??_C@_0BI@KCGPNIE@?$CI?$FLBLjava?1lang?1String?$DL?$CJV@ 000000018001a7e0     jni_util.obj
 0002:000027f8       ??_C@_01HMGJMAIH@B@        000000018001a7f8     jni_util.obj
 0002:000027fc       ??_C@_05DMGOLBNP@coder@    000000018001a7fc     jni_util.obj
 0002:00002804       ??_C@_02KCBIMKDL@?$FLB@    000000018001a804     jni_util.obj
 0002:00002808       ??_C@_05MFEJDJP@value@     000000018001a808     jni_util.obj
 0002:00002810       ??_C@_0CC@PDGFIJNH@platform?5encoding?5not?5initializ@ 000000018001a810     jni_util.obj
 0002:00002838       ??_C@_0CG@BPPCDHBK@requested?5array?5size?5exceeds?5VM@ 000000018001a838     jni_util.obj
 0002:00002860       ??_C@_0BA@JJLOPNCP@java?1lang?1Class@ 000000018001a860     jni_util.obj
 0002:00002870       ??_C@_0BB@DDFKOHA@java?1lang?1Object@ 000000018001a870     jni_util.obj
 0002:00002888       ??_C@_0BE@ILKHHCBH@java?1lang?1Throwable@ 000000018001a888     jni_util.obj
 0002:0000289c       ??_C@_06IMBEHKAP@equals@   000000018001a89c     jni_util.obj
 0002:000028a8       ??_C@_0BJ@GFFKIMMI@JNU_MonitorWait?5argument@ 000000018001a8a8     jni_util.obj
 0002:000028c8       ??_C@_0BE@MJCNDKI@JNU_Notify?5argument@ 000000018001a8c8     jni_util.obj
 0002:000028e0       ??_C@_0BH@GMHIOCNA@JNU_NotifyAll?5argument@ 000000018001a8e0     jni_util.obj
 0002:000028f8       ??_C@_0N@CDIMKML@?$CFs?3?5is?5NULL?6@ 000000018001a8f8     jni_util.obj
 0002:00002908       ??_C@_07KJFPOMFC@?$CFs?3?5?$CFs?6@ 000000018001a908     jni_util.obj
 0002:00002910       ??_C@_0BE@JBOGKGNB@?$CFs?3?5object?5is?5NULL?6@ 000000018001a910     jni_util.obj
 0002:00002924       ??_C@_04HIBGFPH@NULL@      000000018001a924     jni_util.obj
 0002:00002930       ??_C@_08JCDFGHAO@toString@ 000000018001a930     jni_util.obj
 0002:00002940       ??_C@_0CG@ENHAICHD@JNU_GetFieldByName?3?5illegal?5sig@ 000000018001a940     jni_util.obj
 0002:00002968       ??_C@_0CG@PKMPNPAI@JNU_SetFieldByName?3?5illegal?5sig@ 000000018001a968     jni_util.obj
 0002:00002990       ??_C@_0CM@FFECHOAH@JNU_GetStaticFieldByName?3?5illeg@ 000000018001a990     jni_util.obj
 0002:000029c0       ??_C@_0CM@HBCEDOCG@JNU_SetStaticFieldByName?3?5illeg@ 000000018001a9c0     jni_util.obj
 0002:000029ec       ??_C@_01IDAFKMJL@_@        000000018001a9ec     jni_util_md.obj
 0002:000029f0       __real@3ff8000000000000    000000018001a9f0     fdlibm:s_atan.obj
 0002:000029f8       __real@4000000000000000    000000018001a9f8     fdlibm:s_atan.obj
 0002:00002a00       __real@bff0000000000000    000000018001aa00     fdlibm:s_atan.obj
 0002:00002a10       __xmm@80000000000000008000000000000000 000000018001aa10     fdlibm:s_atan.obj
 0002:00002a20       __real@3fe0000000000000    000000018001aa20     fdlibm:s_expm1.obj
 0002:00002a28       __real@4008000000000000    000000018001aa28     fdlibm:s_expm1.obj
 0002:00002a30       __real@4018000000000000    000000018001aa30     fdlibm:s_expm1.obj
 0002:00002a38       __real@bfd0000000000000    000000018001aa38     fdlibm:s_expm1.obj
 0002:00002a40       __real@bfe0000000000000    000000018001aa40     fdlibm:s_expm1.obj
 0002:00002a48       __real@c000000000000000    000000018001aa48     fdlibm:s_expm1.obj
 0002:00002a50       __real@3fe5555555555555    000000018001aa50     fdlibm:s_log1p.obj
 0002:00002a58       __real@3ff0000000000000    000000018001aa58     fdlibm:s_log1p.obj
 0002:00002a60       __real@c008000000000000    000000018001aa60     fdlibm:e_atan2.obj
 0002:00002a68       __real@3fd2000000000000    000000018001aa68     fdlibm:k_cos.obj
 0002:00002a70       __real@3fd5555555555555    000000018001aa70     fdlibm:e_log.obj
 0002:00002a78       __real@0000000000000000    000000018001aa78     fdlibm:k_rem_pio2.obj
 0002:00002a80       __real@3fc0000000000000    000000018001aa80     fdlibm:k_rem_pio2.obj
 0002:00002a88       __real@4020000000000000    000000018001aa88     fdlibm:k_rem_pio2.obj
 0002:00002a90       __sz_SHELL32_dll           000000018001aa90     shell32:SHELL32.dll
 0002:00002aa0       FOLDERID_Profile           000000018001aaa0     shell32:shguid.obj
 0002:00002ab0       ??_C@_1BK@DBDEIDLH@?$AAK?$AAE?$AAR?$AAN?$AAE?$AAL?$AA3?$AA2?$AA?4?$AAD?$AAL?$AAL@ 000000018001aab0     delayimp:delayhlp.obj
 0002:00002ad0       ??_C@_0BI@OMNLIJDB@AcquireSRWLockExclusive@ 000000018001aad0     delayimp:delayhlp.obj
 0002:00002ae8       ??_C@_0BI@HMIEPCNJ@ReleaseSRWLockExclusive@ 000000018001aae8     delayimp:delayhlp.obj
 0002:00002b00       __pfnDliNotifyHook2        000000018001ab00     delayimp:delayhk2.obj
 0002:00002b08       __pfnDliFailureHook2       000000018001ab08     delayimp:delayhk1.obj
 0002:00002b20       _pDefaultRawDllMain        000000018001ab20     MSVCRT:dll_dllmain.obj
 0002:00002b20       _pRawDllMain               000000018001ab20     MSVCRT:dll_dllmain.obj
 0002:00002b30       _load_config_used          000000018001ab30     MSVCRT:loadcfg.obj
 0002:00002d00       __volatile_metadata        000000018001ad00     <linker-defined>
 0002:000030e8       __rtc_iaa                  000000018001b0e8     MSVCRT:initsect.obj
 0002:000030f0       __rtc_izz                  000000018001b0f0     MSVCRT:initsect.obj
 0002:000030f8       __rtc_taa                  000000018001b0f8     MSVCRT:initsect.obj
 0002:00003100       __rtc_tzz                  000000018001b100     MSVCRT:initsect.obj
 0002:00003dec       __DELAY_IMPORT_DESCRIPTOR_shell32_dll 000000018001bdec     shell32:SHELL32.dll
 0002:00003e0c       __NULL_DELAY_IMPORT_DESCRIPTOR 000000018001be0c     shell32:SHELL32.dll
 0002:00003e40       \177SHELL32_NULL_THUNK_DATA_DLN 000000018001be40     shell32:SHELL32.dll
 0002:00003e80       \177SHELL32_NULL_THUNK_DATA_DLB 000000018001be80     shell32:SHELL32.dll
 0002:00007d48       __IMPORT_DESCRIPTOR_jvm    000000018001fd48     jvm:jvm.dll
 0002:00007d5c       __IMPORT_DESCRIPTOR_verify 000000018001fd5c     verify:verify.dll
 0002:00007d70       __IMPORT_DESCRIPTOR_ADVAPI32 000000018001fd70     advapi32:ADVAPI32.dll
 0002:00007d84       __IMPORT_DESCRIPTOR_VERSION 000000018001fd84     version:VERSION.dll
 0002:00007d98       __IMPORT_DESCRIPTOR_KERNEL32 000000018001fd98     kernel32:KERNEL32.dll
 0002:00007dac       __IMPORT_DESCRIPTOR_VCRUNTIME140 000000018001fdac     vcruntime:VCRUNTIME140.dll
 0002:00007dc0       __IMPORT_DESCRIPTOR_api-ms-win-crt-heap-l1-1-0 000000018001fdc0     ucrt:api-ms-win-crt-heap-l1-1-0.dll
 0002:00007dd4       __IMPORT_DESCRIPTOR_api-ms-win-crt-string-l1-1-0 000000018001fdd4     ucrt:api-ms-win-crt-string-l1-1-0.dll
 0002:00007de8       __IMPORT_DESCRIPTOR_api-ms-win-crt-stdio-l1-1-0 000000018001fde8     ucrt:api-ms-win-crt-stdio-l1-1-0.dll
 0002:00007dfc       __IMPORT_DESCRIPTOR_api-ms-win-crt-math-l1-1-0 000000018001fdfc     ucrt:api-ms-win-crt-math-l1-1-0.dll
 0002:00007e10       __IMPORT_DESCRIPTOR_api-ms-win-crt-convert-l1-1-0 000000018001fe10     ucrt:api-ms-win-crt-convert-l1-1-0.dll
 0002:00007e24       __IMPORT_DESCRIPTOR_api-ms-win-crt-runtime-l1-1-0 000000018001fe24     ucrt:api-ms-win-crt-runtime-l1-1-0.dll
 0002:00007e38       __IMPORT_DESCRIPTOR_api-ms-win-crt-filesystem-l1-1-0 000000018001fe38     ucrt:api-ms-win-crt-filesystem-l1-1-0.dll
 0002:00007e4c       __IMPORT_DESCRIPTOR_api-ms-win-crt-environment-l1-1-0 000000018001fe4c     ucrt:api-ms-win-crt-environment-l1-1-0.dll
 0002:00007e60       __NULL_IMPORT_DESCRIPTOR   000000018001fe60     jvm:jvm.dll
 0003:00000270       monthsType                 0000000180023270     HostLocaleProviderAdapter_md.obj
 0003:000002a8       sMonthsType                00000001800232a8     HostLocaleProviderAdapter_md.obj
 0003:000002e0       wDaysType                  00000001800232e0     HostLocaleProviderAdapter_md.obj
 0003:00000300       sWDaysType                 0000000180023300     HostLocaleProviderAdapter_md.obj
 0003:00000320       fixes                      0000000180023320     HostLocaleProviderAdapter_md.obj
 0003:00001350       _fltused                   0000000180024350     MSVCRT:fltused.obj
 0003:00001360       __security_cookie_complement 0000000180024360     MSVCRT:gs_cookie.obj
 0003:00001368       __security_cookie          0000000180024368     MSVCRT:gs_cookie.obj
 0003:00001370       __scrt_native_dllmain_reason 0000000180024370     MSVCRT:utility.obj
 0003:00001380       __isa_available            0000000180024380     MSVCRT:cpu_disp.obj
 0003:00001384       __isa_enabled              0000000180024384     MSVCRT:cpu_disp.obj
 0003:00001388       __memset_fast_string_threshold 0000000180024388     MSVCRT:cpu_disp.obj
 0003:00001390       __memset_nt_threshold      0000000180024390     MSVCRT:cpu_disp.obj
 0003:00001398       __scrt_ucrt_dll_is_in_use  0000000180024398     MSVCRT:ucrt_stubs.obj
 0003:000013a0       __imp_SHGetKnownFolderPath 00000001800243a0     shell32:SHELL32.dll
 0003:000013a8       __imp_SHGetFolderPathW     00000001800243a8     shell32:SHELL32.dll
 0003:000013b0       \177SHELL32_NULL_THUNK_DATA_DLA 00000001800243b0     shell32:SHELL32.dll
 0003:000013d8       initialized                00000001800243d8     HostLocaleProviderAdapter_md.obj
 0003:00001618       __hmod__SHELL32_dll        0000000180024618     shell32:SHELL32.dll
 0003:00001620       ?DloadKernel32@@3PEAUHINSTANCE__@@EA 0000000180024620     delayimp:delayhlp.obj
 0003:00001628       ?DloadAcquireSRWLockExclusive@@3P6AXPEA_K@ZEA 0000000180024628     delayimp:delayhlp.obj
 0003:00001630       ?DloadReleaseSRWLockExclusive@@3P6AXPEA_K@ZEA 0000000180024630     delayimp:delayhlp.obj
 0003:00001638       ?DloadSrwLock@@3_KA        0000000180024638     delayimp:delayhlp.obj
 0003:00001640       ?DloadSectionLockCount@@3KA 0000000180024640     delayimp:delayhlp.obj
 0003:00001644       ?DloadSectionOldProtection@@3KA 0000000180024644     delayimp:delayhlp.obj
 0003:00001648       ?DloadSectionCommitPermanent@@3KA 0000000180024648     delayimp:delayhlp.obj
 0003:00001bd0       ?__type_info_root_node@@3U__type_info_node@@A 0000000180024bd0     MSVCRT:tncleanup.obj
 0003:00001be0       __scrt_current_native_startup_state 0000000180024be0     MSVCRT:utility.obj
 0003:00001be8       __scrt_native_startup_lock 0000000180024be8     MSVCRT:utility.obj
 0003:00001c28       __scrt_debugger_hook_flag  0000000180024c28     MSVCRT:utility_desktop.obj
 0003:00001c2c       __favor                    0000000180024c2c     MSVCRT:cpu_disp.obj
 0003:00001c30       ?_OptionsStorage@?1??__local_stdio_scanf_options@@9@9 0000000180024c30     <common>
 0003:00001c38       raf_fd                     0000000180024c38     <common>
 0003:00001c40       pEnumCalendarInfoExEx      0000000180024c40     <common>
 0003:00001c48       pGetCalendarInfoEx         0000000180024c48     <common>
 0003:00001c50       pGetLocaleInfoEx           0000000180024c50     <common>
 0003:00001c58       fos_fd                     0000000180024c58     <common>
 0003:00001c60       fis_fd                     0000000180024c60     <common>
 0003:00001c68       IO_append_fdID             0000000180024c68     <common>
 0003:00001c70       IO_handle_fdID             0000000180024c70     <common>
 0003:00001c78       IO_fd_fdID                 0000000180024c78     <common>
 0003:00001c80       ?_OptionsStorage@?1??__local_stdio_printf_options@@9@9 0000000180024c80     <common>
 0003:00001c88       __dyn_tls_init_callback    0000000180024c88     <common>

 entry point at        0001:00015eb8

 Static symbols

 0000:fffd8000       .debug$S                   0000000180000000     java.exp
 0000:fffd8000       .debug$S                   0000000180000000     vcruntime:VCRUNTIME140.dll
 0000:fffd8000       .debug$S                   0000000180000000     vcruntime:VCRUNTIME140.dll
 0000:fffd8000       .debug$S                   0000000180000000     vcruntime:VCRUNTIME140.dll
 0000:fffd8000       .debug$S                   0000000180000000     vcruntime:VCRUNTIME140.dll
 0000:fffd8000       .debug$S                   0000000180000000     vcruntime:VCRUNTIME140.dll
 0000:fffd8000       .debug$S                   0000000180000000     vcruntime:VCRUNTIME140.dll
 0000:fffd8000       .debug$S                   0000000180000000     vcruntime:VCRUNTIME140.dll
 0000:fffd8000       .debug$S                   0000000180000000     vcruntime:VCRUNTIME140.dll
 0000:fffd8000       .debug$S                   0000000180000000     vcruntime:VCRUNTIME140.dll
 0000:fffd8000       .debug$S                   0000000180000000     vcruntime:VCRUNTIME140.dll
 0000:fffd8000       .debug$S                   0000000180000000     vcruntime:VCRUNTIME140.dll
 0000:fffd8000       .debug$S                   0000000180000000     ucrt:api-ms-win-crt-convert-l1-1-0.dll
 0000:fffd8000       .debug$S                   0000000180000000     ucrt:api-ms-win-crt-convert-l1-1-0.dll
 0000:fffd8000       .debug$S                   0000000180000000     ucrt:api-ms-win-crt-convert-l1-1-0.dll
 0000:fffd8000       .debug$S                   0000000180000000     ucrt:api-ms-win-crt-convert-l1-1-0.dll
 0000:fffd8000       .debug$S                   0000000180000000     ucrt:api-ms-win-crt-convert-l1-1-0.dll
 0000:fffd8000       .debug$S                   0000000180000000     ucrt:api-ms-win-crt-environment-l1-1-0.dll
 0000:fffd8000       .debug$S                   0000000180000000     ucrt:api-ms-win-crt-environment-l1-1-0.dll
 0000:fffd8000       .debug$S                   0000000180000000     ucrt:api-ms-win-crt-environment-l1-1-0.dll
 0000:fffd8000       .debug$S                   0000000180000000     ucrt:api-ms-win-crt-filesystem-l1-1-0.dll
 0000:fffd8000       .debug$S                   0000000180000000     ucrt:api-ms-win-crt-filesystem-l1-1-0.dll
 0000:fffd8000       .debug$S                   0000000180000000     ucrt:api-ms-win-crt-filesystem-l1-1-0.dll
 0000:fffd8000       .debug$S                   0000000180000000     ucrt:api-ms-win-crt-filesystem-l1-1-0.dll
 0000:fffd8000       .debug$S                   0000000180000000     ucrt:api-ms-win-crt-heap-l1-1-0.dll
 0000:fffd8000       .debug$S                   0000000180000000     ucrt:api-ms-win-crt-heap-l1-1-0.dll
 0000:fffd8000       .debug$S                   0000000180000000     ucrt:api-ms-win-crt-heap-l1-1-0.dll
 0000:fffd8000       .debug$S                   0000000180000000     ucrt:api-ms-win-crt-heap-l1-1-0.dll
 0000:fffd8000       .debug$S                   0000000180000000     ucrt:api-ms-win-crt-math-l1-1-0.dll
 0000:fffd8000       .debug$S                   0000000180000000     ucrt:api-ms-win-crt-runtime-l1-1-0.dll
 0000:fffd8000       .debug$S                   0000000180000000     ucrt:api-ms-win-crt-runtime-l1-1-0.dll
 0000:fffd8000       .debug$S                   0000000180000000     ucrt:api-ms-win-crt-runtime-l1-1-0.dll
 0000:fffd8000       .debug$S                   0000000180000000     ucrt:api-ms-win-crt-runtime-l1-1-0.dll
 0000:fffd8000       .debug$S                   0000000180000000     ucrt:api-ms-win-crt-runtime-l1-1-0.dll
 0000:fffd8000       .debug$S                   0000000180000000     ucrt:api-ms-win-crt-runtime-l1-1-0.dll
 0000:fffd8000       .debug$S                   0000000180000000     ucrt:api-ms-win-crt-runtime-l1-1-0.dll
 0000:fffd8000       .debug$S                   0000000180000000     ucrt:api-ms-win-crt-runtime-l1-1-0.dll
 0000:fffd8000       .debug$S                   0000000180000000     ucrt:api-ms-win-crt-runtime-l1-1-0.dll
 0000:fffd8000       .debug$S                   0000000180000000     ucrt:api-ms-win-crt-runtime-l1-1-0.dll
 0000:fffd8000       .debug$S                   0000000180000000     ucrt:api-ms-win-crt-runtime-l1-1-0.dll
 0000:fffd8000       .debug$S                   0000000180000000     ucrt:api-ms-win-crt-runtime-l1-1-0.dll
 0000:fffd8000       .debug$S                   0000000180000000     ucrt:api-ms-win-crt-runtime-l1-1-0.dll
 0000:fffd8000       .debug$S                   0000000180000000     ucrt:api-ms-win-crt-runtime-l1-1-0.dll
 0000:fffd8000       .debug$S                   0000000180000000     ucrt:api-ms-win-crt-stdio-l1-1-0.dll
 0000:fffd8000       .debug$S                   0000000180000000     ucrt:api-ms-win-crt-stdio-l1-1-0.dll
 0000:fffd8000       .debug$S                   0000000180000000     ucrt:api-ms-win-crt-stdio-l1-1-0.dll
 0000:fffd8000       .debug$S                   0000000180000000     ucrt:api-ms-win-crt-stdio-l1-1-0.dll
 0000:fffd8000       .debug$S                   0000000180000000     ucrt:api-ms-win-crt-stdio-l1-1-0.dll
 0000:fffd8000       .debug$S                   0000000180000000     ucrt:api-ms-win-crt-stdio-l1-1-0.dll
 0000:fffd8000       .debug$S                   0000000180000000     ucrt:api-ms-win-crt-stdio-l1-1-0.dll
 0000:fffd8000       .debug$S                   0000000180000000     ucrt:api-ms-win-crt-stdio-l1-1-0.dll
 0000:fffd8000       .debug$S                   0000000180000000     ucrt:api-ms-win-crt-string-l1-1-0.dll
 0000:fffd8000       .debug$S                   0000000180000000     ucrt:api-ms-win-crt-string-l1-1-0.dll
 0000:fffd8000       .debug$S                   0000000180000000     ucrt:api-ms-win-crt-string-l1-1-0.dll
 0000:fffd8000       .debug$S                   0000000180000000     ucrt:api-ms-win-crt-string-l1-1-0.dll
 0000:fffd8000       .debug$S                   0000000180000000     ucrt:api-ms-win-crt-string-l1-1-0.dll
 0000:fffd8000       .debug$S                   0000000180000000     ucrt:api-ms-win-crt-string-l1-1-0.dll
 0000:fffd8000       .debug$S                   0000000180000000     ucrt:api-ms-win-crt-string-l1-1-0.dll
 0000:fffd8000       .debug$S                   0000000180000000     ucrt:api-ms-win-crt-string-l1-1-0.dll
 0000:fffd8000       .debug$S                   0000000180000000     ucrt:api-ms-win-crt-string-l1-1-0.dll
 0000:fffd8000       .debug$S                   0000000180000000     ucrt:api-ms-win-crt-string-l1-1-0.dll
 0000:fffd8000       .debug$S                   0000000180000000     ucrt:api-ms-win-crt-string-l1-1-0.dll
 0000:fffd8000       .debug$S                   0000000180000000     ucrt:api-ms-win-crt-string-l1-1-0.dll
 0000:fffd8000       .debug$S                   0000000180000000     ucrt:api-ms-win-crt-string-l1-1-0.dll
 0000:fffd8000       .debug$S                   0000000180000000     ucrt:api-ms-win-crt-string-l1-1-0.dll
 0000:fffd8000       .debug$S                   0000000180000000     ucrt:api-ms-win-crt-string-l1-1-0.dll
 0000:fffd8000       .debug$S                   0000000180000000     ucrt:api-ms-win-crt-string-l1-1-0.dll
 0000:fffd8000       .debug$S                   0000000180000000     ucrt:api-ms-win-crt-string-l1-1-0.dll
 0000:fffd8000       .debug$S                   0000000180000000     ucrt:api-ms-win-crt-string-l1-1-0.dll
 0000:fffd8000       .debug$S                   0000000180000000     ucrt:api-ms-win-crt-string-l1-1-0.dll
 0000:fffd8000       .debug$S                   0000000180000000     advapi32:ADVAPI32.dll
 0000:fffd8000       .debug$S                   0000000180000000     advapi32:ADVAPI32.dll
 0000:fffd8000       .debug$S                   0000000180000000     advapi32:ADVAPI32.dll
 0000:fffd8000       .debug$S                   0000000180000000     advapi32:ADVAPI32.dll
 0000:fffd8000       .debug$S                   0000000180000000     advapi32:ADVAPI32.dll
 0000:fffd8000       .debug$S                   0000000180000000     advapi32:ADVAPI32.dll
 0000:fffd8000       .debug$S                   0000000180000000     advapi32:ADVAPI32.dll
 0000:fffd8000       .debug$S                   0000000180000000     advapi32:ADVAPI32.dll
 0000:fffd8000       .debug$S                   0000000180000000     advapi32:ADVAPI32.dll
 0000:fffd8000       .debug$S                   0000000180000000     advapi32:ADVAPI32.dll
 0000:fffd8000       .debug$S                   0000000180000000     advapi32:ADVAPI32.dll
 0000:fffd8000       .debug$S                   0000000180000000     advapi32:ADVAPI32.dll
 0000:fffd8000       .debug$S                   0000000180000000     advapi32:ADVAPI32.dll
 0000:fffd8000       .debug$S                   0000000180000000     advapi32:ADVAPI32.dll
 0000:fffd8000       .debug$S                   0000000180000000     advapi32:ADVAPI32.dll
 0000:fffd8000       .debug$S                   0000000180000000     kernel32:KERNEL32.dll
 0000:fffd8000       .debug$S                   0000000180000000     kernel32:KERNEL32.dll
 0000:fffd8000       .debug$S                   0000000180000000     kernel32:KERNEL32.dll
 0000:fffd8000       .debug$S                   0000000180000000     kernel32:KERNEL32.dll
 0000:fffd8000       .debug$S                   0000000180000000     kernel32:KERNEL32.dll
 0000:fffd8000       .debug$S                   0000000180000000     kernel32:KERNEL32.dll
 0000:fffd8000       .debug$S                   0000000180000000     kernel32:KERNEL32.dll
 0000:fffd8000       .debug$S                   0000000180000000     kernel32:KERNEL32.dll
 0000:fffd8000       .debug$S                   0000000180000000     kernel32:KERNEL32.dll
 0000:fffd8000       .debug$S                   0000000180000000     kernel32:KERNEL32.dll
 0000:fffd8000       .debug$S                   0000000180000000     kernel32:KERNEL32.dll
 0000:fffd8000       .debug$S                   0000000180000000     kernel32:KERNEL32.dll
 0000:fffd8000       .debug$S                   0000000180000000     kernel32:KERNEL32.dll
 0000:fffd8000       .debug$S                   0000000180000000     kernel32:KERNEL32.dll
 0000:fffd8000       .debug$S                   0000000180000000     kernel32:KERNEL32.dll
 0000:fffd8000       .debug$S                   0000000180000000     kernel32:KERNEL32.dll
 0000:fffd8000       .debug$S                   0000000180000000     kernel32:KERNEL32.dll
 0000:fffd8000       .debug$S                   0000000180000000     kernel32:KERNEL32.dll
 0000:fffd8000       .debug$S                   0000000180000000     kernel32:KERNEL32.dll
 0000:fffd8000       .debug$S                   0000000180000000     kernel32:KERNEL32.dll
 0000:fffd8000       .debug$S                   0000000180000000     kernel32:KERNEL32.dll
 0000:fffd8000       .debug$S                   0000000180000000     kernel32:KERNEL32.dll
 0000:fffd8000       .debug$S                   0000000180000000     kernel32:KERNEL32.dll
 0000:fffd8000       .debug$S                   0000000180000000     kernel32:KERNEL32.dll
 0000:fffd8000       .debug$S                   0000000180000000     kernel32:KERNEL32.dll
 0000:fffd8000       .debug$S                   0000000180000000     kernel32:KERNEL32.dll
 0000:fffd8000       .debug$S                   0000000180000000     kernel32:KERNEL32.dll
 0000:fffd8000       .debug$S                   0000000180000000     kernel32:KERNEL32.dll
 0000:fffd8000       .debug$S                   0000000180000000     kernel32:KERNEL32.dll
 0000:fffd8000       .debug$S                   0000000180000000     kernel32:KERNEL32.dll
 0000:fffd8000       .debug$S                   0000000180000000     kernel32:KERNEL32.dll
 0000:fffd8000       .debug$S                   0000000180000000     kernel32:KERNEL32.dll
 0000:fffd8000       .debug$S                   0000000180000000     kernel32:KERNEL32.dll
 0000:fffd8000       .debug$S                   0000000180000000     kernel32:KERNEL32.dll
 0000:fffd8000       .debug$S                   0000000180000000     kernel32:KERNEL32.dll
 0000:fffd8000       .debug$S                   0000000180000000     kernel32:KERNEL32.dll
 0000:fffd8000       .debug$S                   0000000180000000     kernel32:KERNEL32.dll
 0000:fffd8000       .debug$S                   0000000180000000     kernel32:KERNEL32.dll
 0000:fffd8000       .debug$S                   0000000180000000     kernel32:KERNEL32.dll
 0000:fffd8000       .debug$S                   0000000180000000     kernel32:KERNEL32.dll
 0000:fffd8000       .debug$S                   0000000180000000     kernel32:KERNEL32.dll
 0000:fffd8000       .debug$S                   0000000180000000     kernel32:KERNEL32.dll
 0000:fffd8000       .debug$S                   0000000180000000     kernel32:KERNEL32.dll
 0000:fffd8000       .debug$S                   0000000180000000     kernel32:KERNEL32.dll
 0000:fffd8000       .debug$S                   0000000180000000     kernel32:KERNEL32.dll
 0000:fffd8000       .debug$S                   0000000180000000     kernel32:KERNEL32.dll
 0000:fffd8000       .debug$S                   0000000180000000     kernel32:KERNEL32.dll
 0000:fffd8000       .debug$S                   0000000180000000     kernel32:KERNEL32.dll
 0000:fffd8000       .debug$S                   0000000180000000     kernel32:KERNEL32.dll
 0000:fffd8000       .debug$S                   0000000180000000     kernel32:KERNEL32.dll
 0000:fffd8000       .debug$S                   0000000180000000     kernel32:KERNEL32.dll
 0000:fffd8000       .debug$S                   0000000180000000     kernel32:KERNEL32.dll
 0000:fffd8000       .debug$S                   0000000180000000     kernel32:KERNEL32.dll
 0000:fffd8000       .debug$S                   0000000180000000     kernel32:KERNEL32.dll
 0000:fffd8000       .debug$S                   0000000180000000     kernel32:KERNEL32.dll
 0000:fffd8000       .debug$S                   0000000180000000     kernel32:KERNEL32.dll
 0000:fffd8000       .debug$S                   0000000180000000     kernel32:KERNEL32.dll
 0000:fffd8000       .debug$S                   0000000180000000     kernel32:KERNEL32.dll
 0000:fffd8000       .debug$S                   0000000180000000     kernel32:KERNEL32.dll
 0000:fffd8000       .debug$S                   0000000180000000     kernel32:KERNEL32.dll
 0000:fffd8000       .debug$S                   0000000180000000     kernel32:KERNEL32.dll
 0000:fffd8000       .debug$S                   0000000180000000     kernel32:KERNEL32.dll
 0000:fffd8000       .debug$S                   0000000180000000     kernel32:KERNEL32.dll
 0000:fffd8000       .debug$S                   0000000180000000     kernel32:KERNEL32.dll
 0000:fffd8000       .debug$S                   0000000180000000     kernel32:KERNEL32.dll
 0000:fffd8000       .debug$S                   0000000180000000     kernel32:KERNEL32.dll
 0000:fffd8000       .debug$S                   0000000180000000     kernel32:KERNEL32.dll
 0000:fffd8000       .debug$S                   0000000180000000     kernel32:KERNEL32.dll
 0000:fffd8000       .debug$S                   0000000180000000     kernel32:KERNEL32.dll
 0000:fffd8000       .debug$S                   0000000180000000     kernel32:KERNEL32.dll
 0000:fffd8000       .debug$S                   0000000180000000     kernel32:KERNEL32.dll
 0000:fffd8000       .debug$S                   0000000180000000     kernel32:KERNEL32.dll
 0000:fffd8000       .debug$S                   0000000180000000     kernel32:KERNEL32.dll
 0000:fffd8000       .debug$S                   0000000180000000     kernel32:KERNEL32.dll
 0000:fffd8000       .debug$S                   0000000180000000     kernel32:KERNEL32.dll
 0000:fffd8000       .debug$S                   0000000180000000     kernel32:KERNEL32.dll
 0000:fffd8000       .debug$S                   0000000180000000     kernel32:KERNEL32.dll
 0000:fffd8000       .debug$S                   0000000180000000     kernel32:KERNEL32.dll
 0000:fffd8000       .debug$S                   0000000180000000     kernel32:KERNEL32.dll
 0000:fffd8000       .debug$S                   0000000180000000     kernel32:KERNEL32.dll
 0000:fffd8000       .debug$S                   0000000180000000     kernel32:KERNEL32.dll
 0000:fffd8000       .debug$S                   0000000180000000     kernel32:KERNEL32.dll
 0000:fffd8000       .debug$S                   0000000180000000     kernel32:KERNEL32.dll
 0000:fffd8000       .debug$S                   0000000180000000     kernel32:KERNEL32.dll
 0000:fffd8000       .debug$S                   0000000180000000     kernel32:KERNEL32.dll
 0000:fffd8000       .debug$S                   0000000180000000     kernel32:KERNEL32.dll
 0000:fffd8000       .debug$S                   0000000180000000     kernel32:KERNEL32.dll
 0000:fffd8000       .debug$S                   0000000180000000     kernel32:KERNEL32.dll
 0000:fffd8000       .debug$S                   0000000180000000     kernel32:KERNEL32.dll
 0000:fffd8000       .debug$S                   0000000180000000     kernel32:KERNEL32.dll
 0000:fffd8000       .debug$S                   0000000180000000     kernel32:KERNEL32.dll
 0000:fffd8000       .debug$S                   0000000180000000     kernel32:KERNEL32.dll
 0000:fffd8000       .debug$S                   0000000180000000     kernel32:KERNEL32.dll
 0000:fffd8000       .debug$S                   0000000180000000     kernel32:KERNEL32.dll
 0000:fffd8000       .debug$S                   0000000180000000     kernel32:KERNEL32.dll
 0000:fffd8000       .debug$S                   0000000180000000     kernel32:KERNEL32.dll
 0000:fffd8000       .debug$S                   0000000180000000     kernel32:KERNEL32.dll
 0000:fffd8000       .debug$S                   0000000180000000     kernel32:KERNEL32.dll
 0000:fffd8000       .debug$S                   0000000180000000     kernel32:KERNEL32.dll
 0000:fffd8000       .debug$S                   0000000180000000     kernel32:KERNEL32.dll
 0000:fffd8000       .debug$S                   0000000180000000     kernel32:KERNEL32.dll
 0000:fffd8000       .debug$S                   0000000180000000     kernel32:KERNEL32.dll
 0000:fffd8000       .debug$S                   0000000180000000     kernel32:KERNEL32.dll
 0000:fffd8000       .debug$S                   0000000180000000     kernel32:KERNEL32.dll
 0000:fffd8000       .debug$S                   0000000180000000     kernel32:KERNEL32.dll
 0000:fffd8000       .debug$S                   0000000180000000     kernel32:KERNEL32.dll
 0000:fffd8000       .debug$S                   0000000180000000     kernel32:KERNEL32.dll
 0000:fffd8000       .debug$S                   0000000180000000     kernel32:KERNEL32.dll
 0000:fffd8000       .debug$S                   0000000180000000     shell32:SHELL32.dll
 0000:fffd8000       .debug$S                   0000000180000000     shell32:SHELL32.dll
 0000:fffd8000       .debug$S                   0000000180000000     version:VERSION.dll
 0000:fffd8000       .debug$S                   0000000180000000     version:VERSION.dll
 0000:fffd8000       .debug$S                   0000000180000000     version:VERSION.dll
 0000:fffd8000       .debug$S                   0000000180000000     jvm:jvm.dll
 0000:fffd8000       .debug$S                   0000000180000000     jvm:jvm.dll
 0000:fffd8000       .debug$S                   0000000180000000     jvm:jvm.dll
 0000:fffd8000       .debug$S                   0000000180000000     jvm:jvm.dll
 0000:fffd8000       .debug$S                   0000000180000000     jvm:jvm.dll
 0000:fffd8000       .debug$S                   0000000180000000     jvm:jvm.dll
 0000:fffd8000       .debug$S                   0000000180000000     jvm:jvm.dll
 0000:fffd8000       .debug$S                   0000000180000000     jvm:jvm.dll
 0000:fffd8000       .debug$S                   0000000180000000     jvm:jvm.dll
 0000:fffd8000       .debug$S                   0000000180000000     jvm:jvm.dll
 0000:fffd8000       .debug$S                   0000000180000000     jvm:jvm.dll
 0000:fffd8000       .debug$S                   0000000180000000     jvm:jvm.dll
 0000:fffd8000       .debug$S                   0000000180000000     jvm:jvm.dll
 0000:fffd8000       .debug$S                   0000000180000000     jvm:jvm.dll
 0000:fffd8000       .debug$S                   0000000180000000     jvm:jvm.dll
 0000:fffd8000       .debug$S                   0000000180000000     jvm:jvm.dll
 0000:fffd8000       .debug$S                   0000000180000000     jvm:jvm.dll
 0000:fffd8000       .debug$S                   0000000180000000     jvm:jvm.dll
 0000:fffd8000       .debug$S                   0000000180000000     jvm:jvm.dll
 0000:fffd8000       .debug$S                   0000000180000000     jvm:jvm.dll
 0000:fffd8000       .debug$S                   0000000180000000     jvm:jvm.dll
 0000:fffd8000       .debug$S                   0000000180000000     jvm:jvm.dll
 0000:fffd8000       .debug$S                   0000000180000000     jvm:jvm.dll
 0000:fffd8000       .debug$S                   0000000180000000     jvm:jvm.dll
 0000:fffd8000       .debug$S                   0000000180000000     jvm:jvm.dll
 0000:fffd8000       .debug$S                   0000000180000000     jvm:jvm.dll
 0000:fffd8000       .debug$S                   0000000180000000     jvm:jvm.dll
 0000:fffd8000       .debug$S                   0000000180000000     jvm:jvm.dll
 0000:fffd8000       .debug$S                   0000000180000000     jvm:jvm.dll
 0000:fffd8000       .debug$S                   0000000180000000     jvm:jvm.dll
 0000:fffd8000       .debug$S                   0000000180000000     jvm:jvm.dll
 0000:fffd8000       .debug$S                   0000000180000000     jvm:jvm.dll
 0000:fffd8000       .debug$S                   0000000180000000     jvm:jvm.dll
 0000:fffd8000       .debug$S                   0000000180000000     jvm:jvm.dll
 0000:fffd8000       .debug$S                   0000000180000000     jvm:jvm.dll
 0000:fffd8000       .debug$S                   0000000180000000     jvm:jvm.dll
 0000:fffd8000       .debug$S                   0000000180000000     jvm:jvm.dll
 0000:fffd8000       .debug$S                   0000000180000000     jvm:jvm.dll
 0000:fffd8000       .debug$S                   0000000180000000     jvm:jvm.dll
 0000:fffd8000       .debug$S                   0000000180000000     jvm:jvm.dll
 0000:fffd8000       .debug$S                   0000000180000000     jvm:jvm.dll
 0000:fffd8000       .debug$S                   0000000180000000     jvm:jvm.dll
 0000:fffd8000       .debug$S                   0000000180000000     jvm:jvm.dll
 0000:fffd8000       .debug$S                   0000000180000000     jvm:jvm.dll
 0000:fffd8000       .debug$S                   0000000180000000     jvm:jvm.dll
 0000:fffd8000       .debug$S                   0000000180000000     jvm:jvm.dll
 0000:fffd8000       .debug$S                   0000000180000000     jvm:jvm.dll
 0000:fffd8000       .debug$S                   0000000180000000     jvm:jvm.dll
 0000:fffd8000       .debug$S                   0000000180000000     jvm:jvm.dll
 0000:fffd8000       .debug$S                   0000000180000000     jvm:jvm.dll
 0000:fffd8000       .debug$S                   0000000180000000     jvm:jvm.dll
 0000:fffd8000       .debug$S                   0000000180000000     jvm:jvm.dll
 0000:fffd8000       .debug$S                   0000000180000000     jvm:jvm.dll
 0000:fffd8000       .debug$S                   0000000180000000     jvm:jvm.dll
 0000:fffd8000       .debug$S                   0000000180000000     jvm:jvm.dll
 0000:fffd8000       .debug$S                   0000000180000000     jvm:jvm.dll
 0000:fffd8000       .debug$S                   0000000180000000     jvm:jvm.dll
 0000:fffd8000       .debug$S                   0000000180000000     jvm:jvm.dll
 0000:fffd8000       .debug$S                   0000000180000000     jvm:jvm.dll
 0000:fffd8000       .debug$S                   0000000180000000     jvm:jvm.dll
 0000:fffd8000       .debug$S                   0000000180000000     jvm:jvm.dll
 0000:fffd8000       .debug$S                   0000000180000000     jvm:jvm.dll
 0000:fffd8000       .debug$S                   0000000180000000     jvm:jvm.dll
 0000:fffd8000       .debug$S                   0000000180000000     jvm:jvm.dll
 0000:fffd8000       .debug$S                   0000000180000000     jvm:jvm.dll
 0000:fffd8000       .debug$S                   0000000180000000     jvm:jvm.dll
 0000:fffd8000       .debug$S                   0000000180000000     jvm:jvm.dll
 0000:fffd8000       .debug$S                   0000000180000000     jvm:jvm.dll
 0000:fffd8000       .debug$S                   0000000180000000     jvm:jvm.dll
 0000:fffd8000       .debug$S                   0000000180000000     jvm:jvm.dll
 0000:fffd8000       .debug$S                   0000000180000000     jvm:jvm.dll
 0000:fffd8000       .debug$S                   0000000180000000     jvm:jvm.dll
 0000:fffd8000       .debug$S                   0000000180000000     jvm:jvm.dll
 0000:fffd8000       .debug$S                   0000000180000000     jvm:jvm.dll
 0000:fffd8000       .debug$S                   0000000180000000     jvm:jvm.dll
 0000:fffd8000       .debug$S                   0000000180000000     jvm:jvm.dll
 0000:fffd8000       .debug$S                   0000000180000000     jvm:jvm.dll
 0000:fffd8000       .debug$S                   0000000180000000     jvm:jvm.dll
 0000:fffd8000       .debug$S                   0000000180000000     jvm:jvm.dll
 0000:fffd8000       .debug$S                   0000000180000000     jvm:jvm.dll
 0000:fffd8000       .debug$S                   0000000180000000     jvm:jvm.dll
 0000:fffd8000       .debug$S                   0000000180000000     jvm:jvm.dll
 0000:fffd8000       .debug$S                   0000000180000000     jvm:jvm.dll
 0000:fffd8000       .debug$S                   0000000180000000     jvm:jvm.dll
 0000:fffd8000       .debug$S                   0000000180000000     jvm:jvm.dll
 0000:fffd8000       .debug$S                   0000000180000000     jvm:jvm.dll
 0000:fffd8000       .debug$S                   0000000180000000     jvm:jvm.dll
 0000:fffd8000       .debug$S                   0000000180000000     jvm:jvm.dll
 0000:fffd8000       .debug$S                   0000000180000000     jvm:jvm.dll
 0000:fffd8000       .debug$S                   0000000180000000     jvm:jvm.dll
 0000:fffd8000       .debug$S                   0000000180000000     jvm:jvm.dll
 0000:fffd8000       .debug$S                   0000000180000000     jvm:jvm.dll
 0000:fffd8000       .debug$S                   0000000180000000     jvm:jvm.dll
 0000:fffd8000       .debug$S                   0000000180000000     jvm:jvm.dll
 0000:fffd8000       .debug$S                   0000000180000000     jvm:jvm.dll
 0000:fffd8000       .debug$S                   0000000180000000     jvm:jvm.dll
 0000:fffd8000       .debug$S                   0000000180000000     jvm:jvm.dll
 0000:fffd8000       .debug$S                   0000000180000000     jvm:jvm.dll
 0000:fffd8000       .debug$S                   0000000180000000     jvm:jvm.dll
 0000:fffd8000       .debug$S                   0000000180000000     jvm:jvm.dll
 0000:fffd8000       .debug$S                   0000000180000000     jvm:jvm.dll
 0000:fffd8000       .debug$S                   0000000180000000     jvm:jvm.dll
 0000:fffd8000       .debug$S                   0000000180000000     jvm:jvm.dll
 0000:fffd8000       .debug$S                   0000000180000000     jvm:jvm.dll
 0000:fffd8000       .debug$S                   0000000180000000     jvm:jvm.dll
 0000:fffd8000       .debug$S                   0000000180000000     jvm:jvm.dll
 0000:fffd8000       .debug$S                   0000000180000000     jvm:jvm.dll
 0000:fffd8000       .debug$S                   0000000180000000     jvm:jvm.dll
 0000:fffd8000       .debug$S                   0000000180000000     jvm:jvm.dll
 0000:fffd8000       .debug$S                   0000000180000000     jvm:jvm.dll
 0000:fffd8000       .debug$S                   0000000180000000     jvm:jvm.dll
 0000:fffd8000       .debug$S                   0000000180000000     jvm:jvm.dll
 0000:fffd8000       .debug$S                   0000000180000000     jvm:jvm.dll
 0000:fffd8000       .debug$S                   0000000180000000     jvm:jvm.dll
 0000:fffd8000       .debug$S                   0000000180000000     jvm:jvm.dll
 0000:fffd8000       .debug$S                   0000000180000000     jvm:jvm.dll
 0000:fffd8000       .debug$S                   0000000180000000     jvm:jvm.dll
 0000:fffd8000       .debug$S                   0000000180000000     jvm:jvm.dll
 0000:fffd8000       .debug$S                   0000000180000000     jvm:jvm.dll
 0000:fffd8000       .debug$S                   0000000180000000     jvm:jvm.dll
 0000:fffd8000       .debug$S                   0000000180000000     jvm:jvm.dll
 0000:fffd8000       .debug$S                   0000000180000000     jvm:jvm.dll
 0000:fffd8000       .debug$S                   0000000180000000     jvm:jvm.dll
 0000:fffd8000       .debug$S                   0000000180000000     jvm:jvm.dll
 0000:fffd8000       .debug$S                   0000000180000000     jvm:jvm.dll
 0000:fffd8000       .debug$S                   0000000180000000     jvm:jvm.dll
 0000:fffd8000       .debug$S                   0000000180000000     jvm:jvm.dll
 0000:fffd8000       .debug$S                   0000000180000000     jvm:jvm.dll
 0000:fffd8000       .debug$S                   0000000180000000     jvm:jvm.dll
 0000:fffd8000       .debug$S                   0000000180000000     jvm:jvm.dll
 0000:fffd8000       .debug$S                   0000000180000000     jvm:jvm.dll
 0000:fffd8000       .debug$S                   0000000180000000     jvm:jvm.dll
 0000:fffd8000       .debug$S                   0000000180000000     jvm:jvm.dll
 0000:fffd8000       .debug$S                   0000000180000000     verify:verify.dll
 0000:fffd8000       .debug$S                   0000000180000000     verify:verify.dll
 0000:fffd8000       .debug$S                   0000000180000000     verify:verify.dll
 0000:fffd8000       .debug$S                   0000000180000000     verify:verify.dll
 0001:00000df0       findJniFunction            0000000180001df0 f   ClassLoader.obj
 0001:00000ef4       getUTF                     0000000180001ef4 f   ClassLoader.obj
 0001:00000f98       initIDs                    0000000180001f98 f   ClassLoader.obj
 0001:00003130       GetInternalPackageName     0000000180004130 f   Module.obj
 0001:00003cc0       environmentBlock9x         0000000180004cc0 f   ProcessEnvironment_md.obj
 0001:000044a0       getCmdlineInfo             00000001800054a0 f   ProcessHandleImpl_win.obj
 0001:000045b0       getStartTime               00000001800055b0 f   ProcessHandleImpl_win.obj
 0001:00004618       getStatInfo                0000000180005618 f   ProcessHandleImpl_win.obj
 0001:00004730       procToUser                 0000000180005730 f   ProcessHandleImpl_win.obj
 0001:00004c28       initHolder                 0000000180005c28 f   ProcessImpl_md.obj
 0001:00004d48       processCreate              0000000180005d48 f   ProcessImpl_md.obj
 0001:00005048       releaseHolder              0000000180006048 f   ProcessImpl_md.obj
 0001:000050ec       win32Error                 00000001800060ec f   ProcessImpl_md.obj
 0001:00007694       customZoneName             0000000180008694 f   TimeZone_md.obj
 0001:00007884       getValueInRegistry         0000000180008884 f   TimeZone_md.obj
 0001:0000797c       getWinTimeZone             000000018000897c f   TimeZone_md.obj
 0001:00007e5c       matchJavaTZ                0000000180008e5c f   TimeZone_md.obj
 0001:000092e8       getFileInformation         000000018000a2e8 f   WinNTFileSystem_md.obj
 0001:00009464       getFinalPath               000000018000a464 f   WinNTFileSystem_md.obj
 0001:00009660       isReservedDeviceNameW      000000018000a660 f   WinNTFileSystem_md.obj
 0001:00009ba8       cp                         000000018000aba8 f   canonicalize_md.obj
 0001:00009ce0       nextsep                    000000018000ace0 f   canonicalize_md.obj
 0001:0000a194       wcp                        000000018000b194 f   canonicalize_md.obj
 0001:0000ace0       handleStdinAvailable       000000018000bce0 f   io_util_md.obj
 0001:0000b89c       SetupI18nProps             000000018000c89c f   java_props_md.obj
 0001:0000baa8       cpu_isalist                000000018000caa8 f   java_props_md.obj
 0001:0000bb58       getConsoleEncoding         000000018000cb58 f   java_props_md.obj
 0001:0000bbc8       getEncodingInternal        000000018000cbc8 f   java_props_md.obj
 0001:0000dbec       getString646_USChars       000000018000ebec f   jni_util.obj
 0001:0000dcdc       getString8859_1Chars       000000018000ecdc f   jni_util.obj
 0001:0000ddd4       getStringBytes             000000018000edd4 f   jni_util.obj
 0001:0000df30       getStringCp1252Chars       000000018000ef30 f   jni_util.obj
 0001:0000e1b8       getStringUTF8              000000018000f1b8 f   jni_util.obj
 0001:0000e358       jnuEncodingSupported       000000018000f358 f   jni_util.obj
 0001:0000e3a4       newSizedString8859_1       000000018000f3a4 f   jni_util.obj
 0001:0000e48c       newSizedStringJava         000000018000f48c f   jni_util.obj
 0001:0000e5a4       newString646_US            000000018000f5a4 f   jni_util.obj
 0001:0000e69c       newStringCp1252            000000018000f69c f   jni_util.obj
 0001:000157e0       $$000000                   00000001800167e0     MSVCRT:amdsecgs.obj
 0001:000159c8       capture_current_context    00000001800169c8 f   MSVCRT:gs_report.obj
 0001:00015a38       capture_previous_context   0000000180016a38 f   MSVCRT:gs_report.obj
 0001:00015ab0       $$000000                   0000000180016ab0     MSVCRT:chkstk.obj
 0001:00015b98       ?dllmain_crt_dispatch@@YAHQEAUHINSTANCE__@@KQEAX@Z 0000000180016b98 f   MSVCRT:dll_dllmain.obj
 0001:00015be8       ?dllmain_crt_process_attach@@YAHQEAUHINSTANCE__@@QEAX@Z 0000000180016be8 f   MSVCRT:dll_dllmain.obj
 0001:00015d00       ?dllmain_crt_process_detach@@YAH_N@Z 0000000180016d00 f   MSVCRT:dll_dllmain.obj
 0001:00015d84       ?dllmain_dispatch@@YAHQEAUHINSTANCE__@@KQEAX@Z 0000000180016d84 f   MSVCRT:dll_dllmain.obj
 0001:00016760       $$000000                   0000000180017760     MSVCRT:guard_dispatch.obj
 0001:00016780       $$000000                   0000000180017780     MSVCRT:guard_xfg_dispatch.obj
 0001:00016796       ?fin$0@?0??dllmain_crt_process_attach@@YAHQEAUHINSTANCE__@@QEAX@Z@4HA 0000000180017796 f   MSVCRT:dll_dllmain.obj
 0001:000167ad       ?fin$0@?0??dllmain_crt_process_detach@@YAH_N@Z@4HA 00000001800177ad f   MSVCRT:dll_dllmain.obj
 0001:000167c6       ?fin$1@?0??dllmain_crt_process_detach@@YAH_N@Z@4HA 00000001800177c6 f   MSVCRT:dll_dllmain.obj
 0001:000167da       ?filt$0@?0??dllmain_dispatch@@YAHQEAUHINSTANCE__@@KQEAX@Z@4HA 00000001800177da f   MSVCRT:dll_dllmain.obj
 0001:00016810       __scrt_is_nonwritable_in_current_image$filt$0 0000000180017810 f   MSVCRT:utility.obj
 0002:00002b10       GS_ExceptionPointers       000000018001ab10     MSVCRT:gs_report.obj
 0002:00003108       $unwind$Java_java_security_AccessController_doPrivileged__Ljava_security_PrivilegedAction_2 000000018001b108     AccessController.obj
 0002:00003108       $unwind$Java_java_security_AccessController_doPrivileged__Ljava_security_PrivilegedAction_2Ljava_security_AccessControlContext_2 000000018001b108     AccessController.obj
 0002:00003108       $unwind$Java_java_security_AccessController_doPrivileged__Ljava_security_PrivilegedExceptionAction_2 000000018001b108     AccessController.obj
 0002:00003108       $unwind$Java_java_security_AccessController_doPrivileged__Ljava_security_PrivilegedExceptionAction_2Ljava_security_AccessControlContext_2 000000018001b108     AccessController.obj
 0002:00003108       $unwind$Java_java_lang_reflect_Array_getDouble 000000018001b108     Array.obj
 0002:00003108       $unwind$Java_java_lang_reflect_Array_getFloat 000000018001b108     Array.obj
 0002:00003108       $unwind$Java_java_lang_reflect_Array_setLong 000000018001b108     Array.obj
 0002:00003108       $unwind$Java_java_io_FileInputStream_open0 000000018001b108     FileInputStream.obj
 0002:00003108       $unwind$Java_java_io_FileInputStream_readBytes 000000018001b108     FileInputStream.obj
 0002:00003108       $unwind$Java_java_io_FileOutputStream_open0 000000018001b108     FileOutputStream_md.obj
 0002:00003108       $unwind$Java_java_io_FileOutputStream_write 000000018001b108     FileOutputStream_md.obj
 0002:00003108       $unwind$Java_sun_util_locale_provider_HostLocaleProviderAdapterImpl_getEras 000000018001b108     HostLocaleProviderAdapter_md.obj
 0002:00003108       $unwind$Java_java_io_RandomAccessFile_open0 000000018001b108     RandomAccessFile.obj
 0002:00003108       $unwind$Java_java_io_RandomAccessFile_readBytes 000000018001b108     RandomAccessFile.obj
 0002:00003108       $unwind$Java_java_io_RandomAccessFile_write0 000000018001b108     RandomAccessFile.obj
 0002:00003108       $unwind$customZoneName     000000018001b108     TimeZone_md.obj
 0002:00003108       $unwind$handleRead         000000018001b108     io_util_md.obj
 0002:00003108       $unwind$JNU_ToString       000000018001b108     jni_util.obj
 0002:00003108       $unwind$jnuEncodingSupported 000000018001b108     jni_util.obj
 0002:00003110       $unwind$Java_java_lang_reflect_Array_setBoolean 000000018001b110     Array.obj
 0002:00003110       $unwind$Java_java_lang_reflect_Array_setByte 000000018001b110     Array.obj
 0002:00003110       $unwind$Java_java_lang_reflect_Array_setChar 000000018001b110     Array.obj
 0002:00003110       $unwind$Java_java_lang_reflect_Array_setFloat 000000018001b110     Array.obj
 0002:00003110       $unwind$Java_java_lang_reflect_Array_setInt 000000018001b110     Array.obj
 0002:00003110       $unwind$Java_java_lang_reflect_Array_setShort 000000018001b110     Array.obj
 0002:00003110       $unwind$Java_java_io_FileOutputStream_writeBytes 000000018001b110     FileOutputStream_md.obj
 0002:00003110       $unwind$Java_java_io_RandomAccessFile_writeBytes 000000018001b110     RandomAccessFile.obj
 0002:00003118       $unwind$Java_java_lang_Class_forName0 000000018001b118     Class.obj
 0002:0000313c       $unwind$Java_java_lang_Class_isAssignableFrom 000000018001b13c     Class.obj
 0002:0000313c       $unwind$Java_java_io_Console_istty 000000018001b13c     Console_md.obj
 0002:0000313c       $unwind$Java_java_io_FileInputStream_initIDs 000000018001b13c     FileInputStream.obj
 0002:0000313c       $unwind$Java_java_io_FileOutputStream_initIDs 000000018001b13c     FileOutputStream_md.obj
 0002:0000313c       $unwind$getCalendarID      000000018001b13c     HostLocaleProviderAdapter_md.obj
 0002:0000313c       $unwind$Java_java_lang_Object_getClass 000000018001b13c     Object.obj
 0002:0000313c       $unwind$Java_java_lang_ProcessHandleImpl_getCurrentPid0 000000018001b13c     ProcessHandleImpl_win.obj
 0002:0000313c       $unwind$Java_java_lang_ProcessImpl_isProcessAlive 000000018001b13c     ProcessImpl_md.obj
 0002:0000313c       $unwind$Java_java_io_RandomAccessFile_initIDs 000000018001b13c     RandomAccessFile.obj
 0002:0000313c       $unwind$Java_sun_io_Win32ErrorMode_setErrorMode 000000018001b13c     Win32ErrorMode.obj
 0002:0000313c       $unwind$cp                 000000018001b13c     canonicalize_md.obj
 0002:0000313c       $unwind$lastErrorReportable 000000018001b13c     canonicalize_md.obj
 0002:0000313c       $unwind$wcp                000000018001b13c     canonicalize_md.obj
 0002:0000313c       $unwind$handleGetLength    000000018001b13c     io_util_md.obj
 0002:0000313c       $unwind$handleLseek        000000018001b13c     io_util_md.obj
 0002:0000313c       $unwind$handleSync         000000018001b13c     io_util_md.obj
 0002:0000313c       $unwind$JDK_InitJvmHandle  000000018001b13c     jdk_util_md.obj
 0002:0000313c       $unwind$JNU_GetEnv         000000018001b13c     jni_util.obj
 0002:0000313c       $unwind$JNU_GetStringPlatformChars 000000018001b13c     jni_util.obj
 0002:0000313c       $unwind$__scrt_initialize_default_local_stdio_options 000000018001b13c     MSVCRT:default_local_stdio_options.obj
 0002:0000313c       $unwind$?dllmain_crt_dispatch@@YAHQEAUHINSTANCE__@@KQEAX@Z 000000018001b13c     MSVCRT:dll_dllmain.obj
 0002:0000313c       $unwind$DllMain            000000018001b13c     MSVCRT:dll_dllmain_stub.obj
 0002:0000313c       $unwind$__report_rangecheckfailure 000000018001b13c     MSVCRT:gs_report.obj
 0002:0000313c       $unwind$__GSHandlerCheck   000000018001b13c     MSVCRT:gshandler.obj
 0002:0000313c       $unwind$__scrt_acquire_startup_lock 000000018001b13c     MSVCRT:utility.obj
 0002:0000313c       $unwind$__scrt_dllmain_after_initialize_c 000000018001b13c     MSVCRT:utility.obj
 0002:0000313c       $unwind$__scrt_dllmain_before_initialize_c 000000018001b13c     MSVCRT:utility.obj
 0002:0000313c       $unwind$__scrt_dllmain_crt_thread_attach 000000018001b13c     MSVCRT:utility.obj
 0002:0000313c       $unwind$__scrt_dllmain_crt_thread_detach 000000018001b13c     MSVCRT:utility.obj
 0002:0000313c       $unwind$__scrt_dllmain_uninitialize_c 000000018001b13c     MSVCRT:utility.obj
 0002:0000313c       $unwind$__scrt_dllmain_uninitialize_critical 000000018001b13c     MSVCRT:utility.obj
 0002:0000313c       $unwind$?DloadReleaseSectionWriteAccess@@YAXXZ 000000018001b13c     delayimp:delayhlp.obj
 0002:00003144       $unwind$Java_java_lang_Class_getPrimitiveClass 000000018001b144     Class.obj
 0002:00003144       $unwind$Java_java_lang_ClassLoader_00024NativeLibrary_findEntry 000000018001b144     ClassLoader.obj
 0002:00003144       $unwind$Java_sun_util_locale_provider_HostLocaleProviderAdapterImpl_getCalendarID 000000018001b144     HostLocaleProviderAdapter_md.obj
 0002:00003144       $unwind$getLocaleInfoWrapper 000000018001b144     HostLocaleProviderAdapter_md.obj
 0002:00003144       $unwind$Java_java_io_RandomAccessFile_seek0 000000018001b144     RandomAccessFile.obj
 0002:00003144       $unwind$Java_java_io_RandomAccessFile_setLength 000000018001b144     RandomAccessFile.obj
 0002:00003144       $unwind$Java_jdk_internal_misc_Signal_findSignal0 000000018001b144     Signal.obj
 0002:00003144       $unwind$Java_java_io_WinNTFileSystem_getDriveDirectory 000000018001b144     WinNTFileSystem_md.obj
 0002:00003144       $unwind$Java_java_io_WinNTFileSystem_rename0 000000018001b144     WinNTFileSystem_md.obj
 0002:00003144       $unwind$JNU_IsInstanceOfByName 000000018001b144     jni_util.obj
 0002:00003144       $unwind$__scrt_dllmain_exception_filter 000000018001b144     MSVCRT:utility.obj
 0002:00003158       $unwind$Java_java_lang_ClassLoader_defineClass1 000000018001b158     ClassLoader.obj
 0002:00003158       $unwind$Java_java_lang_ClassLoader_defineClass2 000000018001b158     ClassLoader.obj
 0002:0000317c       $unwind$Java_java_lang_ClassLoader_findBootstrapClass 000000018001b17c     ClassLoader.obj
 0002:00003198       $unwind$Java_java_lang_ClassLoader_findBuiltinLib 000000018001b198     ClassLoader.obj
 0002:00003198       $unwind$pathToNTPath       000000018001b198     io_util_md.obj
 0002:00003198       $unwind$JNU_CallMethodByNameV 000000018001b198     jni_util.obj
 0002:000031b4       $unwind$Java_java_lang_ClassLoader_00024NativeLibrary_load0 000000018001b1b4     ClassLoader.obj
 0002:000031d4       $unwind$Java_java_lang_ClassLoader_00024NativeLibrary_unload 000000018001b1d4     ClassLoader.obj
 0002:000031d4       $unwind$getStringBytes     000000018001b1d4     jni_util.obj
 0002:000031ec       $unwind$getUTF             000000018001b1ec     ClassLoader.obj
 0002:000031ec       $unwind$GetInternalPackageName 000000018001b1ec     Module.obj
 0002:000031ec       $unwind$environmentBlock9x 000000018001b1ec     ProcessEnvironment_md.obj
 0002:000031ec       $unwind$newSizedStringJava 000000018001b1ec     jni_util.obj
 0002:00003204       $unwind$initIDs            000000018001b204     ClassLoader.obj
 0002:00003204       $unwind$Java_java_io_FileDescriptor_initIDs 000000018001b204     FileDescriptor_md.obj
 0002:00003204       $unwind$Java_java_lang_ProcessEnvironment_environmentBlock 000000018001b204     ProcessEnvironment_md.obj
 0002:00003204       $unwind$Java_java_lang_ProcessHandleImpl_00024Info_initIDs 000000018001b204     ProcessHandleImpl_win.obj
 0002:00003204       $unwind$Java_java_lang_ProcessHandleImpl_isAlive0 000000018001b204     ProcessHandleImpl_win.obj
 0002:00003204       $unwind$releaseHolder      000000018001b204     ProcessImpl_md.obj
 0002:00003204       $unwind$Java_java_lang_SecurityManager_getClassContext 000000018001b204     SecurityManager.obj
 0002:00003204       $unwind$Java_jdk_internal_misc_VM_initialize 000000018001b204     VM.obj
 0002:00003204       $unwind$Java_java_io_WinNTFileSystem_createDirectory 000000018001b204     WinNTFileSystem_md.obj
 0002:00003204       $unwind$Java_java_io_WinNTFileSystem_delete0 000000018001b204     WinNTFileSystem_md.obj
 0002:00003204       $unwind$Java_java_io_WinNTFileSystem_getBooleanAttributes 000000018001b204     WinNTFileSystem_md.obj
 0002:00003204       $unwind$currentDirLength   000000018001b204     io_util_md.obj
 0002:00003204       $unwind$JNU_ClassClass     000000018001b204     jni_util.obj
 0002:00003204       $unwind$JNU_ClassObject    000000018001b204     jni_util.obj
 0002:00003204       $unwind$JNU_ClassString    000000018001b204     jni_util.obj
 0002:00003204       $unwind$JNU_ClassThrowable 000000018001b204     jni_util.obj
 0002:00003204       $unwind$JNU_NewStringPlatform 000000018001b204     jni_util.obj
 0002:00003204       $unwind$JNU_Notify         000000018001b204     jni_util.obj
 0002:00003204       $unwind$JNU_NotifyAll      000000018001b204     jni_util.obj
 0002:00003204       $unwind$JNU_PrintString    000000018001b204     jni_util.obj
 0002:00003204       $unwind$JNU_ThrowByName    000000018001b204     jni_util.obj
 0002:00003204       $unwind$_RTC_Initialize    000000018001b204     MSVCRT:initsect.obj
 0002:00003204       $unwind$_RTC_Terminate     000000018001b204     MSVCRT:initsect.obj
 0002:00003204       $unwind$?DloadGetSRWLockFunctionPointers@@YAEXZ 000000018001b204     delayimp:delayhlp.obj
 0002:00003210       $unwind$findJniFunction    000000018001b210     ClassLoader.obj
 0002:00003210       $unwind$getFinalPath       000000018001b210     WinNTFileSystem_md.obj
 0002:0000322c       $unwind$sprintf            000000018001b22c     Console_md.obj
 0002:0000322c       $unwind$sscanf             000000018001b22c     java_props_md.obj
 0002:0000322c       $unwind$fprintf            000000018001b22c     jni_util.obj
 0002:00003238       $unwind$Java_java_io_Console_encoding 000000018001b238     Console_md.obj
 0002:00003248       $unwind$Java_java_io_Console_echo 000000018001b248     Console_md.obj
 0002:00003248       $unwind$Java_sun_util_locale_provider_HostLocaleProviderAdapterImpl_getDefaultLocale 000000018001b248     HostLocaleProviderAdapter_md.obj
 0002:00003248       $unwind$Java_java_io_ObjectStreamClass_hasStaticInitializer 000000018001b248     ObjectStreamClass.obj
 0002:00003248       $unwind$Java_java_lang_ProcessHandleImpl_00024Info_info0 000000018001b248     ProcessHandleImpl_win.obj
 0002:00003248       $unwind$Java_java_lang_ProcessHandleImpl_destroy0 000000018001b248     ProcessHandleImpl_win.obj
 0002:00003248       $unwind$Java_java_io_RandomAccessFile_getFilePointer 000000018001b248     RandomAccessFile.obj
 0002:00003248       $unwind$Java_java_io_RandomAccessFile_length 000000018001b248     RandomAccessFile.obj
 0002:00003248       $unwind$Java_java_lang_System_setErr0 000000018001b248     System.obj
 0002:00003248       $unwind$Java_java_lang_System_setIn0 000000018001b248     System.obj
 0002:00003248       $unwind$Java_java_lang_System_setOut0 000000018001b248     System.obj
 0002:00003248       $unwind$Java_java_util_TimeZone_getSystemGMTOffsetID 000000018001b248     TimeZone.obj
 0002:00003248       $unwind$Java_java_io_WinNTFileSystem_checkAccess 000000018001b248     WinNTFileSystem_md.obj
 0002:00003248       $unwind$Java_java_io_WinNTFileSystem_setReadOnly 000000018001b248     WinNTFileSystem_md.obj
 0002:00003248       $unwind$getPrefixed        000000018001b248     canonicalize_md.obj
 0002:00003248       $unwind$fileDescriptorClose 000000018001b248     io_util_md.obj
 0002:00003248       $unwind$GetStringPlatform  000000018001b248     java_props_md.obj
 0002:00003248       $unwind$InitializeEncoding 000000018001b248     jni_util.obj
 0002:00003248       $unwind$JNU_Equals         000000018001b248     jni_util.obj
 0002:00003248       $unwind$JNU_MonitorWait    000000018001b248     jni_util.obj
 0002:00003248       $unwind$_DllMainCRTStartup 000000018001b248     MSVCRT:dll_dllmain.obj
 0002:00003258       $unwind$Java_java_io_FileDescriptor_sync 000000018001b258     FileDescriptor_md.obj
 0002:00003258       $unwind$EnumCalendarInfoProc 000000018001b258     HostLocaleProviderAdapter_md.obj
 0002:00003258       $unwind$Java_sun_util_locale_provider_HostLocaleProviderAdapterImpl_initialize 000000018001b258     HostLocaleProviderAdapter_md.obj
 0002:00003258       $unwind$Java_java_io_ObjectStreamClass_initNative 000000018001b258     ObjectStreamClass.obj
 0002:00003258       $unwind$Java_java_lang_ProcessImpl_getExitCodeProcess 000000018001b258     ProcessImpl_md.obj
 0002:00003258       $unwind$Java_java_lang_Throwable_fillInStackTrace 000000018001b258     Throwable.obj
 0002:00003258       $unwind$Java_java_io_WinNTFileSystem_initIDs 000000018001b258     WinNTFileSystem_md.obj
 0002:00003258       $unwind$nextsep            000000018001b258     canonicalize_md.obj
 0002:00003258       $unwind$fileToNTPath       000000018001b258     io_util_md.obj
 0002:00003258       $unwind$handleSetLength    000000018001b258     io_util_md.obj
 0002:00003258       $unwind$getConsoleEncoding 000000018001b258     java_props_md.obj
 0002:00003258       $unwind$JDK_GetVersionInfo0 000000018001b258     jdk_util.obj
 0002:00003258       $unwind$__raise_securityfailure 000000018001b258     MSVCRT:gs_report.obj
 0002:00003258       $unwind$__scrt_initialize_crt 000000018001b258     MSVCRT:utility.obj
 0002:00003258       $unwind$__scrt_initialize_onexit_tables 000000018001b258     MSVCRT:utility.obj
 0002:00003258       $unwind$__scrt_release_startup_lock 000000018001b258     MSVCRT:utility.obj
 0002:00003258       $unwind$__scrt_uninitialize_crt 000000018001b258     MSVCRT:utility.obj
 0002:00003258       $unwind$?DloadAcquireSectionWriteAccess@@YAXXZ 000000018001b258     delayimp:delayhlp.obj
 0002:00003260       $unwind$Java_java_io_FileCleanable_cleanupClose0 000000018001b260     FileDescriptor_md.obj
 0002:00003268       $unwind$Java_java_io_FileInputStream_skip0 000000018001b268     FileInputStream.obj
 0002:00003268       $unwind$Java_sun_util_locale_provider_HostLocaleProviderAdapterImpl_getNumberPattern 000000018001b268     HostLocaleProviderAdapter_md.obj
 0002:00003268       $unwind$Java_java_util_TimeZone_getSystemTimeZoneID 000000018001b268     TimeZone.obj
 0002:00003268       $unwind$getString646_USChars 000000018001b268     jni_util.obj
 0002:00003268       $unwind$getString8859_1Chars 000000018001b268     jni_util.obj
 0002:00003268       $unwind$buildJniFunctionName 000000018001b268     jni_util_md.obj
 0002:00003268       $unwind$__GSHandlerCheck_SEH 000000018001b268     MSVCRT:gshandlerseh.obj
 0002:00003280       $unwind$Java_java_io_FileInputStream_available0 000000018001b280     FileInputStream.obj
 0002:00003290       $unwind$Java_sun_util_locale_provider_HostLocaleProviderAdapterImpl_getDateTimePattern 000000018001b290     HostLocaleProviderAdapter_md.obj
 0002:000032b0       $unwind$Java_sun_util_locale_provider_HostLocaleProviderAdapterImpl_getAmPmStrings 000000018001b2b0     HostLocaleProviderAdapter_md.obj
 0002:000032cc       $unwind$Java_sun_util_locale_provider_HostLocaleProviderAdapterImpl_getMonths 000000018001b2cc     HostLocaleProviderAdapter_md.obj
 0002:000032cc       $unwind$Java_sun_util_locale_provider_HostLocaleProviderAdapterImpl_getShortMonths 000000018001b2cc     HostLocaleProviderAdapter_md.obj
 0002:000032cc       $unwind$Java_sun_util_locale_provider_HostLocaleProviderAdapterImpl_getShortWeekdays 000000018001b2cc     HostLocaleProviderAdapter_md.obj
 0002:000032cc       $unwind$Java_sun_util_locale_provider_HostLocaleProviderAdapterImpl_getWeekdays 000000018001b2cc     HostLocaleProviderAdapter_md.obj
 0002:000032d4       $unwind$Java_sun_util_locale_provider_HostLocaleProviderAdapterImpl_getCalendarDataValue 000000018001b2d4     HostLocaleProviderAdapter_md.obj
 0002:000032d4       $unwind$Java_sun_util_locale_provider_HostLocaleProviderAdapterImpl_isNativeDigit 000000018001b2d4     HostLocaleProviderAdapter_md.obj
 0002:000032d4       $unwind$JNU_GetStaticFieldByName 000000018001b2d4     jni_util.obj
 0002:000032e8       $unwind$Java_sun_util_locale_provider_HostLocaleProviderAdapterImpl_getCurrencySymbol 000000018001b2e8     HostLocaleProviderAdapter_md.obj
 0002:000032e8       $unwind$Java_sun_util_locale_provider_HostLocaleProviderAdapterImpl_getDecimalSeparator 000000018001b2e8     HostLocaleProviderAdapter_md.obj
 0002:000032e8       $unwind$Java_sun_util_locale_provider_HostLocaleProviderAdapterImpl_getGroupingSeparator 000000018001b2e8     HostLocaleProviderAdapter_md.obj
 0002:000032e8       $unwind$Java_sun_util_locale_provider_HostLocaleProviderAdapterImpl_getInfinity 000000018001b2e8     HostLocaleProviderAdapter_md.obj
 0002:000032e8       $unwind$Java_sun_util_locale_provider_HostLocaleProviderAdapterImpl_getInternationalCurrencySymbol 000000018001b2e8     HostLocaleProviderAdapter_md.obj
 0002:000032e8       $unwind$Java_sun_util_locale_provider_HostLocaleProviderAdapterImpl_getMinusSign 000000018001b2e8     HostLocaleProviderAdapter_md.obj
 0002:000032e8       $unwind$Java_sun_util_locale_provider_HostLocaleProviderAdapterImpl_getMonetaryDecimalSeparator 000000018001b2e8     HostLocaleProviderAdapter_md.obj
 0002:000032e8       $unwind$Java_sun_util_locale_provider_HostLocaleProviderAdapterImpl_getNaN 000000018001b2e8     HostLocaleProviderAdapter_md.obj
 0002:000032e8       $unwind$Java_sun_util_locale_provider_HostLocaleProviderAdapterImpl_getPerMill 000000018001b2e8     HostLocaleProviderAdapter_md.obj
 0002:000032e8       $unwind$Java_sun_util_locale_provider_HostLocaleProviderAdapterImpl_getPercent 000000018001b2e8     HostLocaleProviderAdapter_md.obj
 0002:000032e8       $unwind$Java_sun_util_locale_provider_HostLocaleProviderAdapterImpl_getZeroDigit 000000018001b2e8     HostLocaleProviderAdapter_md.obj
 0002:00003308       $unwind$Java_sun_util_locale_provider_HostLocaleProviderAdapterImpl_getCalendarDisplayStrings 000000018001b308     HostLocaleProviderAdapter_md.obj
 0002:00003308       $unwind$getCalendarInfoWrapper 000000018001b308     HostLocaleProviderAdapter_md.obj
 0002:00003308       $unwind$winFileHandleOpen  000000018001b308     io_util_md.obj
 0002:0000331c       $unwind$Java_sun_util_locale_provider_HostLocaleProviderAdapterImpl_getDisplayString 000000018001b31c     HostLocaleProviderAdapter_md.obj
 0002:00003338       $unwind$replaceCalendarArrayElems 000000018001b338     HostLocaleProviderAdapter_md.obj
 0002:00003358       $unwind$getNumberPattern   000000018001b358     HostLocaleProviderAdapter_md.obj
 0002:00003374       $unwind$getNumberPart      000000018001b374     HostLocaleProviderAdapter_md.obj
 0002:00003394       $unwind$getFixPart         000000018001b394     HostLocaleProviderAdapter_md.obj
 0002:000033a8       $unwind$enumCalendarInfoWrapper 000000018001b3a8     HostLocaleProviderAdapter_md.obj
 0002:000033a8       $unwind$JNU_PrintClass     000000018001b3a8     jni_util.obj
 0002:000033bc       $unwind$getErasImpl        000000018001b3bc     HostLocaleProviderAdapter_md.obj
 0002:000033e0       $unwind$Java_java_lang_Module_defineModule0 000000018001b3e0     Module.obj
 0002:000033fc       $unwind$Java_java_lang_Module_addExports0 000000018001b3fc     Module.obj
 0002:00003418       $unwind$Java_java_lang_Module_addExportsToAll0 000000018001b418     Module.obj
 0002:00003418       $unwind$Java_java_lang_Module_addExportsToAllUnnamed0 000000018001b418     Module.obj
 0002:00003430       $unwind$Java_java_io_ObjectInputStream_bytesToDoubles 000000018001b430     ObjectInputStream.obj
 0002:00003430       $unwind$Java_java_io_ObjectInputStream_bytesToFloats 000000018001b430     ObjectInputStream.obj
 0002:00003448       $unwind$Java_java_io_ObjectOutputStream_doublesToBytes 000000018001b448     ObjectOutputStream.obj
 0002:00003448       $unwind$Java_java_io_ObjectOutputStream_floatsToBytes 000000018001b448     ObjectOutputStream.obj
 0002:00003468       $unwind$Java_java_lang_ProcessHandleImpl_waitForProcessExit0 000000018001b468     ProcessHandleImpl_win.obj
 0002:00003468       $unwind$Java_java_lang_ProcessImpl_waitForTimeoutInterruptibly 000000018001b468     ProcessImpl_md.obj
 0002:00003474       $unwind$Java_java_lang_ProcessHandleImpl_parent0 000000018001b474     ProcessHandleImpl_win.obj
 0002:00003494       $unwind$Java_java_lang_ProcessHandleImpl_getProcessPids0 000000018001b494     ProcessHandleImpl_win.obj
 0002:000034b8       $unwind$getStatInfo        000000018001b4b8     ProcessHandleImpl_win.obj
 0002:000034cc       $unwind$getCmdlineInfo     000000018001b4cc     ProcessHandleImpl_win.obj
 0002:000034e8       $unwind$procToUser         000000018001b4e8     ProcessHandleImpl_win.obj
 0002:00003504       $unwind$getStartTime       000000018001b504     ProcessHandleImpl_win.obj
 0002:0000350c       $unwind$swprintf           000000018001b50c     ProcessImpl_md.obj
 0002:0000351c       $unwind$Java_java_lang_ProcessImpl_waitForInterruptibly 000000018001b51c     ProcessImpl_md.obj
 0002:0000351c       $unwind$handleWrite        000000018001b51c     io_util_md.obj
 0002:00003524       $unwind$Java_java_lang_ProcessImpl_create 000000018001b524     ProcessImpl_md.obj
 0002:0000353c       $unwind$Java_java_lang_ProcessImpl_openForAtomicAppend 000000018001b53c     ProcessImpl_md.obj
 0002:0000353c       $unwind$Java_java_io_WinNTFileSystem_createFileExclusively 000000018001b53c     WinNTFileSystem_md.obj
 0002:0000353c       $unwind$Java_java_io_WinNTFileSystem_getLastModifiedTime 000000018001b53c     WinNTFileSystem_md.obj
 0002:0000354c       $unwind$os_error_message   000000018001b54c     ProcessImpl_md.obj
 0002:00003558       $unwind$win32Error         000000018001b558     ProcessImpl_md.obj
 0002:00003574       $unwind$initHolder         000000018001b574     ProcessImpl_md.obj
 0002:00003574       $unwind$Java_java_io_WinNTFileSystem_setPermission 000000018001b574     WinNTFileSystem_md.obj
 0002:00003588       $unwind$processCreate      000000018001b588     ProcessImpl_md.obj
 0002:000035a8       $unwind$Java_java_lang_StringCoding_err 000000018001b5a8     StringCoding.obj
 0002:000035a8       $unwind$fileOpen           000000018001b5a8     io_util_md.obj
 0002:000035a8       $unwind$prefixAbpath       000000018001b5a8     io_util_md.obj
 0002:000035a8       $unwind$JNU_CopyObjectArray 000000018001b5a8     jni_util.obj
 0002:000035a8       $unwind$getStringUTF8      000000018001b5a8     jni_util.obj
 0002:000035c0       $unwind$Java_java_lang_System_initProperties 000000018001b5c0     System.obj
 0002:000035e4       $unwind$Java_java_lang_System_mapLibraryName 000000018001b5e4     System.obj
 0002:00003608       $unwind$fillI18nProps      000000018001b608     System.obj
 0002:00003628       $unwind$findJavaTZ_md      000000018001b628     TimeZone_md.obj
 0002:00003640       $unwind$getGMTOffsetID     000000018001b640     TimeZone_md.obj
 0002:0000365c       $unwind$getValueInRegistry 000000018001b65c     TimeZone_md.obj
 0002:0000367c       $unwind$getWinTimeZone     000000018001b67c     TimeZone_md.obj
 0002:000036a0       $unwind$matchJavaTZ        000000018001b6a0     TimeZone_md.obj
 0002:000036c0       $unwind$Java_sun_security_provider_NativeSeedGenerator_nativeGenerateSeed 000000018001b6c0     WinCAPISeedGenerator.obj
 0002:000036d4       $unwind$getFileInformation 000000018001b6d4     WinNTFileSystem_md.obj
 0002:000036e4       $unwind$getFinalAttributesIfReparsePoint 000000018001b6e4     WinNTFileSystem_md.obj
 0002:000036f4       $unwind$getFinalAttributes 000000018001b6f4     WinNTFileSystem_md.obj
 0002:00003710       $unwind$Java_java_io_WinNTFileSystem_canonicalize0 000000018001b710     WinNTFileSystem_md.obj
 0002:00003730       $unwind$Java_java_io_WinNTFileSystem_canonicalizeWithPrefix0 000000018001b730     WinNTFileSystem_md.obj
 0002:00003754       $unwind$isReservedDeviceNameW 000000018001b754     WinNTFileSystem_md.obj
 0002:00003764       $unwind$Java_java_io_WinNTFileSystem_getLength 000000018001b764     WinNTFileSystem_md.obj
 0002:00003784       $unwind$Java_java_io_WinNTFileSystem_list 000000018001b784     WinNTFileSystem_md.obj
 0002:000037a8       $unwind$Java_java_io_WinNTFileSystem_setLastModifiedTime 000000018001b7a8     WinNTFileSystem_md.obj
 0002:000037bc       $unwind$Java_java_io_WinNTFileSystem_getSpace0 000000018001b7bc     WinNTFileSystem_md.obj
 0002:000037d8       $unwind$Java_java_io_WinNTFileSystem_getNameMax0 000000018001b7d8     WinNTFileSystem_md.obj
 0002:000037ec       $unwind$wcanonicalize      000000018001b7ec     canonicalize_md.obj
 0002:00003810       $unwind$canonicalize       000000018001b810     canonicalize_md.obj
 0002:00003834       $unwind$wcanonicalizeWithPrefix 000000018001b834     canonicalize_md.obj
 0002:00003850       $unwind$JNI_OnLoad         000000018001b850     check_version.obj
 0002:00003864       $unwind$readSingle         000000018001b864     io_util.obj
 0002:00003878       $unwind$readBytes          000000018001b878     io_util.obj
 0002:00003898       $unwind$writeSingle        000000018001b898     io_util.obj
 0002:000038ac       $unwind$writeBytes         000000018001b8ac     io_util.obj
 0002:000038cc       $unwind$throwFileNotFoundException 000000018001b8cc     io_util.obj
 0002:000038e8       $unwind$currentDir         000000018001b8e8     io_util_md.obj
 0002:000038f8       $unwind$handleAvailable    000000018001b8f8     io_util_md.obj
 0002:00003908       $unwind$handleAppend       000000018001b908     io_util_md.obj
 0002:00003910       $unwind$handleStdinAvailable 000000018001b910     io_util_md.obj
 0002:00003924       $unwind$getJavaIDFromLangID 000000018001b924     java_props_md.obj
 0002:00003940       $unwind$GetJavaProperties  000000018001b940     java_props_md.obj
 0002:00003968       $unwind$SetupI18nProps     000000018001b968     java_props_md.obj
 0002:00003988       $unwind$getEncodingInternal 000000018001b988     java_props_md.obj
 0002:000039a4       $unwind$getHomeFromShell32 000000018001b9a4     java_props_md.obj
 0002:000039cc       $unwind$cpu_isalist        000000018001b9cc     java_props_md.obj
 0002:000039d4       $unwind$JDK_LoadSystemLibrary 000000018001b9d4     jdk_util_md.obj
 0002:000039ec       $unwind$jio_snprintf       000000018001b9ec     jio.obj
 0002:000039f4       $unwind$jio_fprintf        000000018001b9f4     jio.obj
 0002:000039fc       $unwind$JNU_ThrowByNameWithLastError 000000018001b9fc     jni_util.obj
 0002:00003a14       $unwind$JNU_ThrowByNameWithMessageAndLastError 000000018001ba14     jni_util.obj
 0002:00003a34       $unwind$JNU_CallStaticMethodByName 000000018001ba34     jni_util.obj
 0002:00003a44       $unwind$JNU_CallMethodByName 000000018001ba44     jni_util.obj
 0002:00003a4c       $unwind$JNU_NewObjectByName 000000018001ba4c     jni_util.obj
 0002:00003a5c       $unwind$JNU_GetFieldByName 000000018001ba5c     jni_util.obj
 0002:00003a74       $unwind$JNU_SetFieldByName 000000018001ba74     jni_util.obj
 0002:00003a84       $unwind$JNU_SetStaticFieldByName 000000018001ba84     jni_util.obj
 0002:00003a94       $unwind$newSizedString8859_1 000000018001ba94     jni_util.obj
 0002:00003ab4       $unwind$newString646_US    000000018001bab4     jni_util.obj
 0002:00003ab4       $unwind$newStringCp1252    000000018001bab4     jni_util.obj
 0002:00003ad4       $unwind$getStringCp1252Chars 000000018001bad4     jni_util.obj
 0002:00003af0       $unwind$getLastErrorString 000000018001baf0     jni_util_md.obj
 0002:00003afc       $unwind$jacos              000000018001bafc     fdlibm:w_acos.obj
 0002:00003b04       $unwind$jasin              000000018001bb04     fdlibm:w_asin.obj
 0002:00003b0c       $unwind$jatan              000000018001bb0c     fdlibm:s_atan.obj
 0002:00003b1c       $unwind$jatan2             000000018001bb1c     fdlibm:w_atan2.obj
 0002:00003b24       $unwind$jcos               000000018001bb24     fdlibm:s_cos.obj
 0002:00003b2c       $unwind$jsin               000000018001bb2c     fdlibm:s_sin.obj
 0002:00003b34       $unwind$jtan               000000018001bb34     fdlibm:s_tan.obj
 0002:00003b3c       $unwind$jcosh              000000018001bb3c     fdlibm:w_cosh.obj
 0002:00003b44       $unwind$jsinh              000000018001bb44     fdlibm:w_sinh.obj
 0002:00003b4c       $unwind$jtanh              000000018001bb4c     fdlibm:s_tanh.obj
 0002:00003b54       $unwind$jlog               000000018001bb54     fdlibm:w_log.obj
 0002:00003b5c       $unwind$jlog10             000000018001bb5c     fdlibm:w_log10.obj
 0002:00003b64       $unwind$jsqrt              000000018001bb64     fdlibm:w_sqrt.obj
 0002:00003b6c       $unwind$jremainder         000000018001bb6c     fdlibm:w_remainder.obj
 0002:00003b74       $unwind$jexpm1             000000018001bb74     fdlibm:s_expm1.obj
 0002:00003b7c       $unwind$jlog1p             000000018001bb7c     fdlibm:s_log1p.obj
 0002:00003b84       $unwind$__ieee754_acos     000000018001bb84     fdlibm:e_acos.obj
 0002:00003b8c       $unwind$__ieee754_asin     000000018001bb8c     fdlibm:e_asin.obj
 0002:00003b94       $unwind$__ieee754_atan2    000000018001bb94     fdlibm:e_atan2.obj
 0002:00003b9c       $unwind$__ieee754_rem_pio2 000000018001bb9c     fdlibm:e_rem_pio2.obj
 0002:00003bac       $unwind$__kernel_sin       000000018001bbac     fdlibm:k_sin.obj
 0002:00003bb4       $unwind$__kernel_cos       000000018001bbb4     fdlibm:k_cos.obj
 0002:00003bbc       $unwind$__kernel_tan       000000018001bbbc     fdlibm:k_tan.obj
 0002:00003bcc       $unwind$__ieee754_cosh     000000018001bbcc     fdlibm:e_cosh.obj
 0002:00003bd4       $unwind$__ieee754_sinh     000000018001bbd4     fdlibm:e_sinh.obj
 0002:00003bdc       $unwind$__ieee754_log      000000018001bbdc     fdlibm:e_log.obj
 0002:00003be4       $unwind$__ieee754_log10    000000018001bbe4     fdlibm:e_log10.obj
 0002:00003bec       $unwind$__ieee754_sqrt     000000018001bbec     fdlibm:e_sqrt.obj
 0002:00003bf4       $unwind$__ieee754_remainder 000000018001bbf4     fdlibm:e_remainder.obj
 0002:00003bfc       $unwind$__kernel_rem_pio2  000000018001bbfc     fdlibm:k_rem_pio2.obj
 0002:00003c0c       $unwind$__ieee754_exp      000000018001bc0c     fdlibm:e_exp.obj
 0002:00003c14       $unwind$__ieee754_fmod     000000018001bc14     fdlibm:e_fmod.obj
 0002:00003c1c       $unwind$jfloor             000000018001bc1c     fdlibm:s_floor.obj
 0002:00003c24       $unwind$scalbn             000000018001bc24     fdlibm:s_scalbn.obj
 0002:00003c2c       xdata                      000000018001bc2c     shell32:SHELL32.dll
 0002:00003c34       $unwind$?DloadObtainSection@@YAPEAXPEAK0@Z 000000018001bc34     delayimp:delayhlp.obj
 0002:00003c44       $unwind$?DloadMakePermanentImageCommit@@YAXPEAX_K@Z 000000018001bc44     delayimp:delayhlp.obj
 0002:00003c50       $unwind$?DloadProtectSection@@YAXKPEAK@Z 000000018001bc50     delayimp:delayhlp.obj
 0002:00003c60       $unwind$__delayLoadHelper2 000000018001bc60     delayimp:delayhlp.obj
 0002:00003c7c       $unwind$__GSHandlerCheckCommon 000000018001bc7c     MSVCRT:gshandler.obj
 0002:00003c88       $xdatasym                  000000018001bc88     MSVCRT:amdsecgs.obj
 0002:00003c8c       $unwind$__report_securityfailure 000000018001bc8c     MSVCRT:gs_report.obj
 0002:00003c94       $unwind$__report_gsfailure 000000018001bc94     MSVCRT:gs_report.obj
 0002:00003c9c       $unwind$capture_current_context 000000018001bc9c     MSVCRT:gs_report.obj
 0002:00003ca8       $unwind$capture_previous_context 000000018001bca8     MSVCRT:gs_report.obj
 0002:00003cb8       $xdatasym                  000000018001bcb8     MSVCRT:chkstk.obj
 0002:00003cc0       $unwind$?dllmain_crt_process_attach@@YAHQEAUHINSTANCE__@@QEAX@Z 000000018001bcc0     MSVCRT:dll_dllmain.obj
 0002:00003cfc       $unwind$?fin$0@?0??dllmain_crt_process_attach@@YAHQEAUHINSTANCE__@@QEAX@Z@4HA 000000018001bcfc     MSVCRT:dll_dllmain.obj
 0002:00003cfc       $unwind$?fin$0@?0??dllmain_crt_process_detach@@YAH_N@Z@4HA 000000018001bcfc     MSVCRT:dll_dllmain.obj
 0002:00003cfc       $unwind$?fin$1@?0??dllmain_crt_process_detach@@YAH_N@Z@4HA 000000018001bcfc     MSVCRT:dll_dllmain.obj
 0002:00003d04       $unwind$?dllmain_crt_process_detach@@YAH_N@Z 000000018001bd04     MSVCRT:dll_dllmain.obj
 0002:00003d58       $unwind$?dllmain_dispatch@@YAHQEAUHINSTANCE__@@KQEAX@Z 000000018001bd58     MSVCRT:dll_dllmain.obj
 0002:00003d80       $unwind$?filt$0@?0??dllmain_dispatch@@YAHQEAUHINSTANCE__@@KQEAX@Z@4HA 000000018001bd80     MSVCRT:dll_dllmain.obj
 0002:00003d88       $unwind$__security_init_cookie 000000018001bd88     MSVCRT:gs_support.obj
 0002:00003d94       $unwind$__scrt_is_nonwritable_in_current_image 000000018001bd94     MSVCRT:utility.obj
 0002:00003db4       $unwind$__scrt_is_nonwritable_in_current_image$filt$0 000000018001bdb4     MSVCRT:utility.obj
 0002:00003dbc       $unwind$__scrt_fastfail    000000018001bdbc     MSVCRT:utility_desktop.obj
 0002:00003dd0       $xdatasym                  000000018001bdd0     MSVCRT:guard_dispatch.obj
 0002:00003dd8       $xdatasym                  000000018001bdd8     MSVCRT:guard_xfg_dispatch.obj
 0002:00003ddc       $unwind$__isa_available_init 000000018001bddc     MSVCRT:cpu_disp.obj
 0002:00003e90       .edata                     000000018001be90     java.exp
 0002:00003eb8       rgpv                       000000018001beb8     java.exp
 0002:00004388       rgszName                   000000018001c388     java.exp
 0002:00004858       rgwOrd                     000000018001c858     java.exp
 0002:00004ac0       szName                     000000018001cac0     java.exp
 0002:00004ac9       $N00001                    000000018001cac9     java.exp
 0002:00004ad6       $N00002                    000000018001cad6     java.exp
 0002:00004aed       $N00003                    000000018001caed     java.exp
 0002:00004b00       $N00004                    000000018001cb00     java.exp
 0002:00004b14       $N00005                    000000018001cb14     java.exp
 0002:00004b2a       $N00006                    000000018001cb2a     java.exp
 0002:00004b35       $N00007                    000000018001cb35     java.exp
 0002:00004b4a       $N00008                    000000018001cb4a     java.exp
 0002:00004b60       $N00009                    000000018001cb60     java.exp
 0002:00004b7b       $N00010                    000000018001cb7b     java.exp
 0002:00004b8a       $N00011                    000000018001cb8a     java.exp
 0002:00004b9a       $N00012                    000000018001cb9a     java.exp
 0002:00004baa       $N00013                    000000018001cbaa     java.exp
 0002:00004bbd       $N00014                    000000018001cbbd     java.exp
 0002:00004bd1       $N00015                    000000018001cbd1     java.exp
 0002:00004bdc       $N00016                    000000018001cbdc     java.exp
 0002:00004be7       $N00017                    000000018001cbe7     java.exp
 0002:00004bfa       $N00018                    000000018001cbfa     java.exp
 0002:00004c13       $N00019                    000000018001cc13     java.exp
 0002:00004c2e       $N00020                    000000018001cc2e     java.exp
 0002:00004c45       $N00021                    000000018001cc45     java.exp
 0002:00004c55       $N00022                    000000018001cc55     java.exp
 0002:00004c69       $N00023                    000000018001cc69     java.exp
 0002:00004c7f       $N00024                    000000018001cc7f     java.exp
 0002:00004c8a       $N00025                    000000018001cc8a     java.exp
 0002:00004c98       $N00026                    000000018001cc98     java.exp
 0002:00004ca7       $N00027                    000000018001cca7     java.exp
 0002:00004cb7       $N00028                    000000018001ccb7     java.exp
 0002:00004cd6       $N00029                    000000018001ccd6     java.exp
 0002:00004ce9       $N00030                    000000018001cce9     java.exp
 0002:00004d02       $N00031                    000000018001cd02     java.exp
 0002:00004d2a       $N00032                    000000018001cd2a     java.exp
 0002:00004d3a       $N00033                    000000018001cd3a     java.exp
 0002:00004d57       $N00034                    000000018001cd57     java.exp
 0002:00004d7e       $N00035                    000000018001cd7e     java.exp
 0002:00004d9e       $N00036                    000000018001cd9e     java.exp
 0002:00004db3       $N00037                    000000018001cdb3     java.exp
 0002:00004dd5       $N00038                    000000018001cdd5     java.exp
 0002:00004df1       $N00039                    000000018001cdf1     java.exp
 0002:00004e11       $N00040                    000000018001ce11     java.exp
 0002:00004e33       $N00041                    000000018001ce33     java.exp
 0002:00004e53       $N00042                    000000018001ce53     java.exp
 0002:00004e6a       $N00043                    000000018001ce6a     java.exp
 0002:00004e84       $N00044                    000000018001ce84     java.exp
 0002:00004ea2       $N00045                    000000018001cea2     java.exp
 0002:00004ebd       $N00046                    000000018001cebd     java.exp
 0002:00004edc       $N00047                    000000018001cedc     java.exp
 0002:00004efa       $N00048                    000000018001cefa     java.exp
 0002:00004f19       $N00049                    000000018001cf19     java.exp
 0002:00004f33       $N00050                    000000018001cf33     java.exp
 0002:00004f5c       $N00051                    000000018001cf5c     java.exp
 0002:00004f69       $N00052                    000000018001cf69     java.exp
 0002:00004f83       $N00053                    000000018001cf83     java.exp
 0002:00004fa1       $N00054                    000000018001cfa1     java.exp
 0002:00004fbc       $N00055                    000000018001cfbc     java.exp
 0002:00004fe5       $N00056                    000000018001cfe5     java.exp
 0002:00005008       $N00057                    000000018001d008     java.exp
 0002:0000502e       $N00058                    000000018001d02e     java.exp
 0002:00005054       $N00059                    000000018001d054     java.exp
 0002:00005078       $N00060                    000000018001d078     java.exp
 0002:00005099       $N00061                    000000018001d099     java.exp
 0002:000050c1       $N00062                    000000018001d0c1     java.exp
 0002:000050e6       $N00063                    000000018001d0e6     java.exp
 0002:00005109       $N00064                    000000018001d109     java.exp
 0002:0000512c       $N00065                    000000018001d12c     java.exp
 0002:00005153       $N00066                    000000018001d153     java.exp
 0002:00005176       $N00067                    000000018001d176     java.exp
 0002:0000519c       $N00068                    000000018001d19c     java.exp
 0002:000051c0       $N00069                    000000018001d1c0     java.exp
 0002:000051e4       $N00070                    000000018001d1e4     java.exp
 0002:0000520d       $N00071                    000000018001d20d     java.exp
 0002:0000523b       $N00072                    000000018001d23b     java.exp
 0002:00005268       $N00073                    000000018001d268     java.exp
 0002:00005297       $N00074                    000000018001d297     java.exp
 0002:000052c5       $N00075                    000000018001d2c5     java.exp
 0002:000052f9       $N00076                    000000018001d2f9     java.exp
 0002:00005323       $N00077                    000000018001d323     java.exp
 0002:00005350       $N00078                    000000018001d350     java.exp
 0002:00005376       $N00079                    000000018001d376     java.exp
 0002:0000539b       $N00080                    000000018001d39b     java.exp
 0002:000053bf       $N00081                    000000018001d3bf     java.exp
 0002:000053e3       $N00082                    000000018001d3e3     java.exp
 0002:0000540b       $N00083                    000000018001d40b     java.exp
 0002:0000542f       $N00084                    000000018001d42f     java.exp
 0002:00005457       $N00085                    000000018001d457     java.exp
 0002:0000547c       $N00086                    000000018001d47c     java.exp
 0002:000054a5       $N00087                    000000018001d4a5     java.exp
 0002:000054d0       $N00088                    000000018001d4d0     java.exp
 0002:00005505       $N00089                    000000018001d505     java.exp
 0002:0000552e       $N00090                    000000018001d52e     java.exp
 0002:0000555b       $N00091                    000000018001d55b     java.exp
 0002:0000558e       $N00092                    000000018001d58e     java.exp
 0002:000055b3       $N00093                    000000018001d5b3     java.exp
 0002:000055e5       $N00094                    000000018001d5e5     java.exp
 0002:00005614       $N00095                    000000018001d614     java.exp
 0002:00005645       $N00096                    000000018001d645     java.exp
 0002:0000566c       $N00097                    000000018001d66c     java.exp
 0002:00005695       $N00098                    000000018001d695     java.exp
 0002:000056bc       $N00099                    000000018001d6bc     java.exp
 0002:000056e1       $N00100                    000000018001d6e1     java.exp
 0002:00005703       $N00101                    000000018001d703     java.exp
 0002:0000572b       $N00102                    000000018001d72b     java.exp
 0002:00005750       $N00103                    000000018001d750     java.exp
 0002:00005781       $N00104                    000000018001d781     java.exp
 0002:000057ac       $N00105                    000000018001d7ac     java.exp
 0002:000057d5       $N00106                    000000018001d7d5     java.exp
 0002:0000580d       $N00107                    000000018001d80d     java.exp
 0002:00005841       $N00108                    000000018001d841     java.exp
 0002:00005876       $N00109                    000000018001d876     java.exp
 0002:0000589e       $N00110                    000000018001d89e     java.exp
 0002:000058c6       $N00111                    000000018001d8c6     java.exp
 0002:000058f4       $N00112                    000000018001d8f4     java.exp
 0002:0000591e       $N00113                    000000018001d91e     java.exp
 0002:0000594a       $N00114                    000000018001d94a     java.exp
 0002:00005975       $N00115                    000000018001d975     java.exp
 0002:00005993       $N00116                    000000018001d993     java.exp
 0002:000059ba       $N00117                    000000018001d9ba     java.exp
 0002:000059e0       $N00118                    000000018001d9e0     java.exp
 0002:00005a00       $N00119                    000000018001da00     java.exp
 0002:00005a25       $N00120                    000000018001da25     java.exp
 0002:00005a4f       $N00121                    000000018001da4f     java.exp
 0002:00005a76       $N00122                    000000018001da76     java.exp
 0002:00005a9d       $N00123                    000000018001da9d     java.exp
 0002:00005ac1       $N00124                    000000018001dac1     java.exp
 0002:00005ae3       $N00125                    000000018001dae3     java.exp
 0002:00005b0a       $N00126                    000000018001db0a     java.exp
 0002:00005b38       $N00127                    000000018001db38     java.exp
 0002:00005b58       $N00128                    000000018001db58     java.exp
 0002:00005b7c       $N00129                    000000018001db7c     java.exp
 0002:00005b9b       $N00130                    000000018001db9b     java.exp
 0002:00005bc1       $N00131                    000000018001dbc1     java.exp
 0002:00005bf4       $N00132                    000000018001dbf4     java.exp
 0002:00005c25       $N00133                    000000018001dc25     java.exp
 0002:00005c58       $N00134                    000000018001dc58     java.exp
 0002:00005c82       $N00135                    000000018001dc82     java.exp
 0002:00005cb2       $N00136                    000000018001dcb2     java.exp
 0002:00005ce3       $N00137                    000000018001dce3     java.exp
 0002:00005d0f       $N00138                    000000018001dd0f     java.exp
 0002:00005d39       $N00139                    000000018001dd39     java.exp
 0002:00005d62       $N00140                    000000018001dd62     java.exp
 0002:00005d97       $N00141                    000000018001dd97     java.exp
 0002:00005dbe       $N00142                    000000018001ddbe     java.exp
 0002:00005de0       $N00143                    000000018001dde0     java.exp
 0002:00005e0e       $N00144                    000000018001de0e     java.exp
 0002:00005e37       $N00145                    000000018001de37     java.exp
 0002:00005e61       $N00146                    000000018001de61     java.exp
 0002:00005e8b       $N00147                    000000018001de8b     java.exp
 0002:00005eba       $N00148                    000000018001deba     java.exp
 0002:00005ee6       $N00149                    000000018001dee6     java.exp
 0002:00005f16       $N00150                    000000018001df16     java.exp
 0002:00005f4d       $N00151                    000000018001df4d     java.exp
 0002:00005f78       $N00152                    000000018001df78     java.exp
 0002:00005f9a       $N00153                    000000018001df9a     java.exp
 0002:00005fb4       $N00154                    000000018001dfb4     java.exp
 0002:00005fd5       $N00155                    000000018001dfd5     java.exp
 0002:00005ff8       $N00156                    000000018001dff8     java.exp
 0002:00006027       $N00157                    000000018001e027     java.exp
 0002:0000604a       $N00158                    000000018001e04a     java.exp
 0002:00006068       $N00159                    000000018001e068     java.exp
 0002:000060b1       $N00160                    000000018001e0b1     java.exp
 0002:000060fd       $N00161                    000000018001e0fd     java.exp
 0002:00006133       $N00162                    000000018001e133     java.exp
 0002:0000616a       $N00163                    000000018001e16a     java.exp
 0002:000061a2       $N00164                    000000018001e1a2     java.exp
 0002:000061ca       $N00165                    000000018001e1ca     java.exp
 0002:000061e9       $N00166                    000000018001e1e9     java.exp
 0002:00006208       $N00167                    000000018001e208     java.exp
 0002:00006227       $N00168                    000000018001e227     java.exp
 0002:00006247       $N00169                    000000018001e247     java.exp
 0002:00006265       $N00170                    000000018001e265     java.exp
 0002:00006284       $N00171                    000000018001e284     java.exp
 0002:000062a4       $N00172                    000000018001e2a4     java.exp
 0002:000062c2       $N00173                    000000018001e2c2     java.exp
 0002:000062e2       $N00174                    000000018001e2e2     java.exp
 0002:00006302       $N00175                    000000018001e302     java.exp
 0002:00006320       $N00176                    000000018001e320     java.exp
 0002:0000633f       $N00177                    000000018001e33f     java.exp
 0002:0000635e       $N00178                    000000018001e35e     java.exp
 0002:0000637c       $N00179                    000000018001e37c     java.exp
 0002:0000639b       $N00180                    000000018001e39b     java.exp
 0002:000063bb       $N00181                    000000018001e3bb     java.exp
 0002:000063e2       $N00182                    000000018001e3e2     java.exp
 0002:000063ff       $N00183                    000000018001e3ff     java.exp
 0002:00006426       $N00184                    000000018001e426     java.exp
 0002:0000644b       $N00185                    000000018001e44b     java.exp
 0002:00006470       $N00186                    000000018001e470     java.exp
 0002:00006496       $N00187                    000000018001e496     java.exp
 0002:000064b4       $N00188                    000000018001e4b4     java.exp
 0002:000064d1       $N00189                    000000018001e4d1     java.exp
 0002:000064ef       $N00190                    000000018001e4ef     java.exp
 0002:00006515       $N00191                    000000018001e515     java.exp
 0002:0000653f       $N00192                    000000018001e53f     java.exp
 0002:0000657c       $N00193                    000000018001e57c     java.exp
 0002:000065b1       $N00194                    000000018001e5b1     java.exp
 0002:000065ea       $N00195                    000000018001e5ea     java.exp
 0002:0000660b       $N00196                    000000018001e60b     java.exp
 0002:00006633       $N00197                    000000018001e633     java.exp
 0002:00006658       $N00198                    000000018001e658     java.exp
 0002:0000667d       $N00199                    000000018001e67d     java.exp
 0002:000066a4       $N00200                    000000018001e6a4     java.exp
 0002:000066ca       $N00201                    000000018001e6ca     java.exp
 0002:000066ee       $N00202                    000000018001e6ee     java.exp
 0002:00006715       $N00203                    000000018001e715     java.exp
 0002:0000673a       $N00204                    000000018001e73a     java.exp
 0002:00006760       $N00205                    000000018001e760     java.exp
 0002:0000678b       $N00206                    000000018001e78b     java.exp
 0002:000067b1       $N00207                    000000018001e7b1     java.exp
 0002:000067d2       $N00208                    000000018001e7d2     java.exp
 0002:000067fa       $N00209                    000000018001e7fa     java.exp
 0002:0000681f       $N00210                    000000018001e81f     java.exp
 0002:00006844       $N00211                    000000018001e844     java.exp
 0002:0000686b       $N00212                    000000018001e86b     java.exp
 0002:00006891       $N00213                    000000018001e891     java.exp
 0002:000068b5       $N00214                    000000018001e8b5     java.exp
 0002:000068da       $N00215                    000000018001e8da     java.exp
 0002:00006900       $N00216                    000000018001e900     java.exp
 0002:00006931       $N00217                    000000018001e931     java.exp
 0002:0000696b       $N00218                    000000018001e96b     java.exp
 0002:000069a0       $N00219                    000000018001e9a0     java.exp
 0002:000069f4       $N00220                    000000018001e9f4     java.exp
 0002:00006a6d       $N00221                    000000018001ea6d     java.exp
 0002:00006aca       $N00222                    000000018001eaca     java.exp
 0002:00006b4c       $N00223                    000000018001eb4c     java.exp
 0002:00006b91       $N00224                    000000018001eb91     java.exp
 0002:00006bd2       $N00225                    000000018001ebd2     java.exp
 0002:00006bff       $N00226                    000000018001ebff     java.exp
 0002:00006c2b       $N00227                    000000018001ec2b     java.exp
 0002:00006c65       $N00228                    000000018001ec65     java.exp
 0002:00006ca2       $N00229                    000000018001eca2     java.exp
 0002:00006cdc       $N00230                    000000018001ecdc     java.exp
 0002:00006d1c       $N00231                    000000018001ed1c     java.exp
 0002:00006d46       $N00232                    000000018001ed46     java.exp
 0002:00006d6c       $N00233                    000000018001ed6c     java.exp
 0002:00006d91       $N00234                    000000018001ed91     java.exp
 0002:00006dbf       $N00235                    000000018001edbf     java.exp
 0002:00006de1       $N00236                    000000018001ede1     java.exp
 0002:00006e03       $N00237                    000000018001ee03     java.exp
 0002:00006e24       $N00238                    000000018001ee24     java.exp
 0002:00006e45       $N00239                    000000018001ee45     java.exp
 0002:00006e6a       $N00240                    000000018001ee6a     java.exp
 0002:00006e9a       $N00241                    000000018001ee9a     java.exp
 0002:00006ecd       $N00242                    000000018001eecd     java.exp
 0002:00006f00       $N00243                    000000018001ef00     java.exp
 0002:00006f3b       $N00244                    000000018001ef3b     java.exp
 0002:00006f76       $N00245                    000000018001ef76     java.exp
 0002:00006faa       $N00246                    000000018001efaa     java.exp
 0002:00006fdd       $N00247                    000000018001efdd     java.exp
 0002:00007018       $N00248                    000000018001f018     java.exp
 0002:0000704b       $N00249                    000000018001f04b     java.exp
 0002:0000707c       $N00250                    000000018001f07c     java.exp
 0002:000070ae       $N00251                    000000018001f0ae     java.exp
 0002:000070e9       $N00252                    000000018001f0e9     java.exp
 0002:0000711d       $N00253                    000000018001f11d     java.exp
 0002:00007159       $N00254                    000000018001f159     java.exp
 0002:0000719a       $N00255                    000000018001f19a     java.exp
 0002:000071da       $N00256                    000000018001f1da     java.exp
 0002:0000720a       $N00257                    000000018001f20a     java.exp
 0002:0000723e       $N00258                    000000018001f23e     java.exp
 0002:0000726f       $N00259                    000000018001f26f     java.exp
 0002:000072a1       $N00260                    000000018001f2a1     java.exp
 0002:000072e6       $N00261                    000000018001f2e6     java.exp
 0002:00007321       $N00262                    000000018001f321     java.exp
 0002:00007353       $N00263                    000000018001f353     java.exp
 0002:00007389       $N00264                    000000018001f389     java.exp
 0002:000073c2       $N00265                    000000018001f3c2     java.exp
 0002:000073f9       $N00266                    000000018001f3f9     java.exp
 0002:0000742c       $N00267                    000000018001f42c     java.exp
 0002:00007454       $N00268                    000000018001f454     java.exp
 0002:00007496       $N00269                    000000018001f496     java.exp
 0002:000074e1       $N00270                    000000018001f4e1     java.exp
 0002:00007532       $N00271                    000000018001f532     java.exp
 0002:00007588       $N00272                    000000018001f588     java.exp
 0002:000075d2       $N00273                    000000018001f5d2     java.exp
 0002:00007620       $N00274                    000000018001f620     java.exp
 0002:0000766f       $N00275                    000000018001f66f     java.exp
 0002:000076bf       $N00276                    000000018001f6bf     java.exp
 0002:0000770c       $N00277                    000000018001f70c     java.exp
 0002:00007759       $N00278                    000000018001f759     java.exp
 0002:0000779d       $N00279                    000000018001f79d     java.exp
 0002:000077ee       $N00280                    000000018001f7ee     java.exp
 0002:00007836       $N00281                    000000018001f836     java.exp
 0002:00007891       $N00282                    000000018001f891     java.exp
 0002:000078da       $N00283                    000000018001f8da     java.exp
 0002:00007932       $N00284                    000000018001f932     java.exp
 0002:00007978       $N00285                    000000018001f978     java.exp
 0002:000079bb       $N00286                    000000018001f9bb     java.exp
 0002:00007a08       $N00287                    000000018001fa08     java.exp
 0002:00007a4f       $N00288                    000000018001fa4f     java.exp
 0002:00007a96       $N00289                    000000018001fa96     java.exp
 0002:00007ae1       $N00290                    000000018001fae1     java.exp
 0002:00007b2e       $N00291                    000000018001fb2e     java.exp
 0002:00007b76       $N00292                    000000018001fb76     java.exp
 0002:00007bbf       $N00293                    000000018001fbbf     java.exp
 0002:00007c06       $N00294                    000000018001fc06     java.exp
 0002:00007c50       $N00295                    000000018001fc50     java.exp
 0002:00007c62       $N00296                    000000018001fc62     java.exp
 0002:00007c73       $N00297                    000000018001fc73     java.exp
 0002:00007c93       $N00298                    000000018001fc93     java.exp
 0002:00007ca9       $N00299                    000000018001fca9     java.exp
 0002:00007cb8       $N00300                    000000018001fcb8     java.exp
 0002:00007ccc       $N00301                    000000018001fccc     java.exp
 0002:00007cdf       $N00302                    000000018001fcdf     java.exp
 0002:00007ceb       $N00303                    000000018001fceb     java.exp
 0002:00007cf7       $N00304                    000000018001fcf7     java.exp
 0002:00007d02       $N00305                    000000018001fd02     java.exp
 0002:00007d0e       $N00306                    000000018001fd0e     java.exp
 0002:00007d1b       $N00307                    000000018001fd1b     java.exp
 0002:00007d36       $N00308                    000000018001fd36     java.exp
 0002:000095de       .idata$6                   00000001800215de     jvm:jvm.dll
 0002:0000963a       .idata$6                   000000018002163a     verify:verify.dll
 0002:00009768       .idata$6                   0000000180021768     advapi32:ADVAPI32.dll
 0002:000097b8       .idata$6                   00000001800217b8     version:VERSION.dll
 0002:00009ff0       .idata$6                   0000000180021ff0     kernel32:KERNEL32.dll
 0002:0000a07c       .idata$6                   000000018002207c     vcruntime:VCRUNTIME140.dll
 0002:0000a35a       .idata$6                   000000018002235a     ucrt:api-ms-win-crt-heap-l1-1-0.dll
 0002:0000a37a       .idata$6                   000000018002237a     ucrt:api-ms-win-crt-string-l1-1-0.dll
 0002:0000a39c       .idata$6                   000000018002239c     ucrt:api-ms-win-crt-stdio-l1-1-0.dll
 0002:0000a3bc       .idata$6                   00000001800223bc     ucrt:api-ms-win-crt-math-l1-1-0.dll
 0002:0000a3dc       .idata$6                   00000001800223dc     ucrt:api-ms-win-crt-convert-l1-1-0.dll
 0002:0000a3fe       .idata$6                   00000001800223fe     ucrt:api-ms-win-crt-runtime-l1-1-0.dll
 0002:0000a420       .idata$6                   0000000180022420     ucrt:api-ms-win-crt-filesystem-l1-1-0.dll
 0002:0000a446       .idata$6                   0000000180022446     ucrt:api-ms-win-crt-environment-l1-1-0.dll
 0003:00000000       methods                    0000000180023000     Class.obj
 0003:00000240       methods                    0000000180023240     ClassLoader.obj
 0003:00000258       hStdOut                    0000000180023258     Console_md.obj
 0003:00000260       hStdIn                     0000000180023260     Console_md.obj
 0003:00000920       methods                    0000000180023920     Object.obj
 0003:000009a0       methods                    00000001800239a0     System.obj
 0003:000009f0       methods                    00000001800239f0     Thread.obj
 0003:00000b70       keyNames                   0000000180023b70     TimeZone_md.obj
 0003:00000b90       methods                    0000000180023b90     VM.obj
 0003:00000ba8       MAX_INPUT_EVENTS           0000000180023ba8     io_util_md.obj
 0003:00000bac       ?curDirLenCached@?4??currentDirLength@@9@9 0000000180023bac     io_util_md.obj
 0003:00000bb0       cp1252c1chars              0000000180023bb0     jni_util.obj
 0003:00000c30       atanhi                     0000000180023c30     fdlibm:s_atan.obj
 0003:00000c50       atanlo                     0000000180023c50     fdlibm:s_atan.obj
 0003:00000c70       aT                         0000000180023c70     fdlibm:s_atan.obj
 0003:00000cc8       one                        0000000180023cc8     fdlibm:s_atan.obj
 0003:00000cd0       HUGE_NUMBER                0000000180023cd0     fdlibm:s_atan.obj
 0003:00000cd8       one                        0000000180023cd8     fdlibm:s_tanh.obj
 0003:00000ce0       two                        0000000180023ce0     fdlibm:s_tanh.obj
 0003:00000ce8       tiny                       0000000180023ce8     fdlibm:s_tanh.obj
 0003:00000cf0       one                        0000000180023cf0     fdlibm:s_expm1.obj
 0003:00000cf8       HUGE_NUMBER                0000000180023cf8     fdlibm:s_expm1.obj
 0003:00000d00       tiny                       0000000180023d00     fdlibm:s_expm1.obj
 0003:00000d08       o_threshold                0000000180023d08     fdlibm:s_expm1.obj
 0003:00000d10       ln2_hi                     0000000180023d10     fdlibm:s_expm1.obj
 0003:00000d18       ln2_lo                     0000000180023d18     fdlibm:s_expm1.obj
 0003:00000d20       invln2                     0000000180023d20     fdlibm:s_expm1.obj
 0003:00000d28       Q1                         0000000180023d28     fdlibm:s_expm1.obj
 0003:00000d30       Q2                         0000000180023d30     fdlibm:s_expm1.obj
 0003:00000d38       Q3                         0000000180023d38     fdlibm:s_expm1.obj
 0003:00000d40       Q4                         0000000180023d40     fdlibm:s_expm1.obj
 0003:00000d48       Q5                         0000000180023d48     fdlibm:s_expm1.obj
 0003:00000d50       ln2_hi                     0000000180023d50     fdlibm:s_log1p.obj
 0003:00000d58       ln2_lo                     0000000180023d58     fdlibm:s_log1p.obj
 0003:00000d60       two54                      0000000180023d60     fdlibm:s_log1p.obj
 0003:00000d68       Lp1                        0000000180023d68     fdlibm:s_log1p.obj
 0003:00000d70       Lp2                        0000000180023d70     fdlibm:s_log1p.obj
 0003:00000d78       Lp3                        0000000180023d78     fdlibm:s_log1p.obj
 0003:00000d80       Lp4                        0000000180023d80     fdlibm:s_log1p.obj
 0003:00000d88       Lp5                        0000000180023d88     fdlibm:s_log1p.obj
 0003:00000d90       Lp6                        0000000180023d90     fdlibm:s_log1p.obj
 0003:00000d98       Lp7                        0000000180023d98     fdlibm:s_log1p.obj
 0003:00000da0       one                        0000000180023da0     fdlibm:e_acos.obj
 0003:00000da8       pi                         0000000180023da8     fdlibm:e_acos.obj
 0003:00000db0       pio2_hi                    0000000180023db0     fdlibm:e_acos.obj
 0003:00000db8       pio2_lo                    0000000180023db8     fdlibm:e_acos.obj
 0003:00000dc0       pS0                        0000000180023dc0     fdlibm:e_acos.obj
 0003:00000dc8       pS1                        0000000180023dc8     fdlibm:e_acos.obj
 0003:00000dd0       pS2                        0000000180023dd0     fdlibm:e_acos.obj
 0003:00000dd8       pS3                        0000000180023dd8     fdlibm:e_acos.obj
 0003:00000de0       pS4                        0000000180023de0     fdlibm:e_acos.obj
 0003:00000de8       pS5                        0000000180023de8     fdlibm:e_acos.obj
 0003:00000df0       qS1                        0000000180023df0     fdlibm:e_acos.obj
 0003:00000df8       qS2                        0000000180023df8     fdlibm:e_acos.obj
 0003:00000e00       qS3                        0000000180023e00     fdlibm:e_acos.obj
 0003:00000e08       qS4                        0000000180023e08     fdlibm:e_acos.obj
 0003:00000e10       one                        0000000180023e10     fdlibm:e_asin.obj
 0003:00000e18       HUGE_NUMBER                0000000180023e18     fdlibm:e_asin.obj
 0003:00000e20       pio2_hi                    0000000180023e20     fdlibm:e_asin.obj
 0003:00000e28       pio2_lo                    0000000180023e28     fdlibm:e_asin.obj
 0003:00000e30       pio4_hi                    0000000180023e30     fdlibm:e_asin.obj
 0003:00000e38       pS0                        0000000180023e38     fdlibm:e_asin.obj
 0003:00000e40       pS1                        0000000180023e40     fdlibm:e_asin.obj
 0003:00000e48       pS2                        0000000180023e48     fdlibm:e_asin.obj
 0003:00000e50       pS3                        0000000180023e50     fdlibm:e_asin.obj
 0003:00000e58       pS4                        0000000180023e58     fdlibm:e_asin.obj
 0003:00000e60       pS5                        0000000180023e60     fdlibm:e_asin.obj
 0003:00000e68       qS1                        0000000180023e68     fdlibm:e_asin.obj
 0003:00000e70       qS2                        0000000180023e70     fdlibm:e_asin.obj
 0003:00000e78       qS3                        0000000180023e78     fdlibm:e_asin.obj
 0003:00000e80       qS4                        0000000180023e80     fdlibm:e_asin.obj
 0003:00000e88       tiny                       0000000180023e88     fdlibm:e_atan2.obj
 0003:00000e90       pi_o_4                     0000000180023e90     fdlibm:e_atan2.obj
 0003:00000e98       pi_o_2                     0000000180023e98     fdlibm:e_atan2.obj
 0003:00000ea0       pi                         0000000180023ea0     fdlibm:e_atan2.obj
 0003:00000ea8       pi_lo                      0000000180023ea8     fdlibm:e_atan2.obj
 0003:00000eb0       two_over_pi                0000000180023eb0     fdlibm:e_rem_pio2.obj
 0003:00000fb8       half                       0000000180023fb8     fdlibm:e_rem_pio2.obj
 0003:00000fc0       npio2_hw                   0000000180023fc0     fdlibm:e_rem_pio2.obj
 0003:00001040       two24                      0000000180024040     fdlibm:e_rem_pio2.obj
 0003:00001048       invpio2                    0000000180024048     fdlibm:e_rem_pio2.obj
 0003:00001050       pio2_1                     0000000180024050     fdlibm:e_rem_pio2.obj
 0003:00001058       pio2_1t                    0000000180024058     fdlibm:e_rem_pio2.obj
 0003:00001060       pio2_2                     0000000180024060     fdlibm:e_rem_pio2.obj
 0003:00001068       pio2_2t                    0000000180024068     fdlibm:e_rem_pio2.obj
 0003:00001070       pio2_3                     0000000180024070     fdlibm:e_rem_pio2.obj
 0003:00001078       pio2_3t                    0000000180024078     fdlibm:e_rem_pio2.obj
 0003:00001080       half                       0000000180024080     fdlibm:k_sin.obj
 0003:00001088       S1                         0000000180024088     fdlibm:k_sin.obj
 0003:00001090       S2                         0000000180024090     fdlibm:k_sin.obj
 0003:00001098       S3                         0000000180024098     fdlibm:k_sin.obj
 0003:000010a0       S4                         00000001800240a0     fdlibm:k_sin.obj
 0003:000010a8       S5                         00000001800240a8     fdlibm:k_sin.obj
 0003:000010b0       S6                         00000001800240b0     fdlibm:k_sin.obj
 0003:000010b8       one                        00000001800240b8     fdlibm:k_cos.obj
 0003:000010c0       C1                         00000001800240c0     fdlibm:k_cos.obj
 0003:000010c8       C2                         00000001800240c8     fdlibm:k_cos.obj
 0003:000010d0       C3                         00000001800240d0     fdlibm:k_cos.obj
 0003:000010d8       C4                         00000001800240d8     fdlibm:k_cos.obj
 0003:000010e0       C5                         00000001800240e0     fdlibm:k_cos.obj
 0003:000010e8       C6                         00000001800240e8     fdlibm:k_cos.obj
 0003:000010f0       one                        00000001800240f0     fdlibm:k_tan.obj
 0003:000010f8       pio4                       00000001800240f8     fdlibm:k_tan.obj
 0003:00001100       pio4lo                     0000000180024100     fdlibm:k_tan.obj
 0003:00001110       T                          0000000180024110     fdlibm:k_tan.obj
 0003:00001178       one                        0000000180024178     fdlibm:e_cosh.obj
 0003:00001180       half                       0000000180024180     fdlibm:e_cosh.obj
 0003:00001188       HUGE_NUMBER                0000000180024188     fdlibm:e_cosh.obj
 0003:00001190       one                        0000000180024190     fdlibm:e_sinh.obj
 0003:00001198       shuge                      0000000180024198     fdlibm:e_sinh.obj
 0003:000011a0       ln2_hi                     00000001800241a0     fdlibm:e_log.obj
 0003:000011a8       ln2_lo                     00000001800241a8     fdlibm:e_log.obj
 0003:000011b0       two54                      00000001800241b0     fdlibm:e_log.obj
 0003:000011b8       Lg1                        00000001800241b8     fdlibm:e_log.obj
 0003:000011c0       Lg2                        00000001800241c0     fdlibm:e_log.obj
 0003:000011c8       Lg3                        00000001800241c8     fdlibm:e_log.obj
 0003:000011d0       Lg4                        00000001800241d0     fdlibm:e_log.obj
 0003:000011d8       Lg5                        00000001800241d8     fdlibm:e_log.obj
 0003:000011e0       Lg6                        00000001800241e0     fdlibm:e_log.obj
 0003:000011e8       Lg7                        00000001800241e8     fdlibm:e_log.obj
 0003:000011f0       two54                      00000001800241f0     fdlibm:e_log10.obj
 0003:000011f8       ivln10                     00000001800241f8     fdlibm:e_log10.obj
 0003:00001200       log10_2hi                  0000000180024200     fdlibm:e_log10.obj
 0003:00001208       log10_2lo                  0000000180024208     fdlibm:e_log10.obj
 0003:00001210       one                        0000000180024210     fdlibm:e_sqrt.obj
 0003:00001218       tiny                       0000000180024218     fdlibm:e_sqrt.obj
 0003:00001220       init_jk                    0000000180024220     fdlibm:k_rem_pio2.obj
 0003:00001230       PIo2                       0000000180024230     fdlibm:k_rem_pio2.obj
 0003:00001270       one                        0000000180024270     fdlibm:k_rem_pio2.obj
 0003:00001278       two24                      0000000180024278     fdlibm:k_rem_pio2.obj
 0003:00001280       twon24                     0000000180024280     fdlibm:k_rem_pio2.obj
 0003:00001288       one                        0000000180024288     fdlibm:e_exp.obj
 0003:00001290       halF                       0000000180024290     fdlibm:e_exp.obj
 0003:000012a0       HUGE_NUMBER                00000001800242a0     fdlibm:e_exp.obj
 0003:000012a8       twom1000                   00000001800242a8     fdlibm:e_exp.obj
 0003:000012b0       o_threshold                00000001800242b0     fdlibm:e_exp.obj
 0003:000012b8       u_threshold                00000001800242b8     fdlibm:e_exp.obj
 0003:000012c0       ln2HI                      00000001800242c0     fdlibm:e_exp.obj
 0003:000012d0       ln2LO                      00000001800242d0     fdlibm:e_exp.obj
 0003:000012e0       invln2                     00000001800242e0     fdlibm:e_exp.obj
 0003:000012e8       P1                         00000001800242e8     fdlibm:e_exp.obj
 0003:000012f0       P2                         00000001800242f0     fdlibm:e_exp.obj
 0003:000012f8       P3                         00000001800242f8     fdlibm:e_exp.obj
 0003:00001300       P4                         0000000180024300     fdlibm:e_exp.obj
 0003:00001308       P5                         0000000180024308     fdlibm:e_exp.obj
 0003:00001310       one                        0000000180024310     fdlibm:e_fmod.obj
 0003:00001318       Zero                       0000000180024318     fdlibm:e_fmod.obj
 0003:00001328       HUGE_NUMBER                0000000180024328     fdlibm:s_floor.obj
 0003:00001330       two54                      0000000180024330     fdlibm:s_scalbn.obj
 0003:00001338       twom54                     0000000180024338     fdlibm:s_scalbn.obj
 0003:00001340       HUGE_NUMBER                0000000180024340     fdlibm:s_scalbn.obj
 0003:00001348       tiny                       0000000180024348     fdlibm:s_scalbn.obj
 0003:000013c0       handleID                   00000001800243c0     ClassLoader.obj
 0003:000013c8       jniVersionID               00000001800243c8     ClassLoader.obj
 0003:000013d0       procHandle                 00000001800243d0     ClassLoader.obj
 0003:000013e0       noSuchMethodErrCl          00000001800243e0     ObjectStreamClass.obj
 0003:000013e8       ProcessHandleImpl_Info_commandID 00000001800243e8     ProcessHandleImpl_win.obj
 0003:000013f0       ProcessHandleImpl_Info_commandLineID 00000001800243f0     ProcessHandleImpl_win.obj
 0003:000013f8       ProcessHandleImpl_Info_argumentsID 00000001800243f8     ProcessHandleImpl_win.obj
 0003:00001400       ProcessHandleImpl_Info_totalTimeID 0000000180024400     ProcessHandleImpl_win.obj
 0003:00001408       ProcessHandleImpl_Info_startTimeID 0000000180024408     ProcessHandleImpl_win.obj
 0003:00001410       ProcessHandleImpl_Info_userID 0000000180024410     ProcessHandleImpl_win.obj
 0003:00001418       ?initField@?1??check@@9@9  0000000180024418     SecurityManager.obj
 0003:00001420       ids                        0000000180024420     WinNTFileSystem_md.obj
 0003:00001428       GetFinalPathNameByHandle_func 0000000180024428     WinNTFileSystem_md.obj
 0003:00001430       ?u_path@?1??getHomeFromShell32@@9@9 0000000180024430     java_props_md.obj
 0003:00001440       ?sprops@?1??GetJavaProperties@@9@9 0000000180024440     java_props_md.obj
 0003:00001568       jvm_handle                 0000000180024568     jdk_util_md.obj
 0003:00001570       fastEncoding               0000000180024570     jni_util.obj
 0003:00001574       isJNUEncodingSupported     0000000180024574     jni_util.obj
 0003:00001578       jnuEncoding                0000000180024578     jni_util.obj
 0003:00001580       String_init_ID             0000000180024580     jni_util.obj
 0003:00001588       String_getBytes_ID         0000000180024588     jni_util.obj
 0003:00001590       String_coder_ID            0000000180024590     jni_util.obj
 0003:00001598       String_value_ID            0000000180024598     jni_util.obj
 0003:000015a0       ?cls@?1??JNU_ClassString@@9@9 00000001800245a0     jni_util.obj
 0003:000015a8       ?cls@?1??JNU_ClassClass@@9@9 00000001800245a8     jni_util.obj
 0003:000015b0       ?cls@?1??JNU_ClassObject@@9@9 00000001800245b0     jni_util.obj
 0003:000015b8       ?cls@?1??JNU_ClassThrowable@@9@9 00000001800245b8     jni_util.obj
 0003:000015c0       ?mid@?1??JNU_Equals@@9@9   00000001800245c0     jni_util.obj
 0003:000015c8       Object_waitMID             00000001800245c8     jni_util.obj
 0003:000015d0       Object_notifyMID           00000001800245d0     jni_util.obj
 0003:000015d8       Object_notifyAllMID        00000001800245d8     jni_util.obj
 0003:000015e0       zero                       00000001800245e0     fdlibm:s_log1p.obj
 0003:000015e8       zero                       00000001800245e8     fdlibm:e_atan2.obj
 0003:000015f0       zero                       00000001800245f0     fdlibm:e_rem_pio2.obj
 0003:000015f8       zero                       00000001800245f8     fdlibm:e_log.obj
 0003:00001600       zero                       0000000180024600     fdlibm:e_log10.obj
 0003:00001608       zero                       0000000180024608     fdlibm:e_remainder.obj
 0003:00001610       zero                       0000000180024610     fdlibm:k_rem_pio2.obj
 0003:00001650       GS_ExceptionRecord         0000000180024650     MSVCRT:gs_report.obj
 0003:000016f0       GS_ContextRecord           00000001800246f0     MSVCRT:gs_report.obj
 0003:00001bc0       ?__proc_attached@@3HA      0000000180024bc0     MSVCRT:dll_dllmain.obj
 0003:00001bf0       ?is_initialized_as_dll@@3_NA 0000000180024bf0     MSVCRT:utility.obj
 0003:00001bf1       ?module_local_atexit_table_initialized@@3_NA 0000000180024bf1     MSVCRT:utility.obj
 0003:00001bf8       ?module_local_atexit_table@@3U_onexit_table_t@@A 0000000180024bf8     MSVCRT:utility.obj
 0003:00001c10       ?module_local_at_quick_exit_table@@3U_onexit_table_t@@A 0000000180024c10     MSVCRT:utility.obj
 0005:00000060       $R000000                   0000000180026060     java.dll.res
